:020000040800F2
:1000000000060020E1010008E3010008E301000808
:10001000E3010008E3010008E3010008E301000830
:10002000E3010008E3010008E30100086D2F000868
:10003000E3010008E3010008E3010008E301000810
:10004000E3010008E3010008E3010008E301000800
:10005000E3010008E3010008153200083D32000802
:10006000653200088D320008B5320008E30100084F
:10007000E3010008E3010008E3010008E3010008D0
:10008000E3010008E3010008E3010008E3010008C0
:10009000E3010008E3010008E3010008DD32000885
:1000A000E3010008E3010008E3010008E3010008A0
:1000B000B1330008E3010008E3010008E301000890
:1000C000E3010008E3010008E3010008E301000880
:1000D000E3010008E3010008E3010008E301000870
:1000E00041330008E3010008E3010008E3010008D0
:1000F000E3010008E3010008E3010008E301000850
:10010000E3010008E3010008E3010008E30100083F
:10011000E3010008E3010008E3010008E30100082F
:10012000E3010008E3010008E3010008E30100081F
:10013000E3010008E3010008E3010008E30100080F
:10014000E3010008E3010008E3010008212700089B
:10015000E3010008E3010008E3010008E3010008EF
:10016000E3010008E3010008E3010008E3010008DF
:10017000E3010008E3010008E3010008E3010008CF
:10018000E3010008E3010008E3010008E3010008BF
:10019000E3010008E3010008E3010008E3010008AF
:1001A000E3010008E3010008E3010008E30100089F
:1001B000E3010008E3010008E3010008E30100088F
:1001C000E3010008E3010008E3010008E30100087F
:1001D000E3010008E3010008E3010008E30100086F
:1001E00002E000F000F8FEE772B6374880F30888B6
:1001F000364880F3098836483649086040F20000E6
:10020000CCF200004EF63471CEF200010860BFF36C
:100210004F8FBFF36F8F40F20000C0F2F0004EF638
:100220008851CEF200010860BFF34F8FBFF36F8F8C
:100230004FF00000E1EE100A4EF63C71CEF20001E4
:100240000860062080F31488BFF36F8F01F030FF41
:1002500002F02AFE4FF055301F491B4A91423CBF25
:1002600041F8040BFAE71D49184A91423CBF41F896
:10027000040BFAE71A491B4A1B4B9A423EBF51F83E
:10028000040B42F8040BF8E700201849184A914281
:100290003CBF41F8040BFAE701F00EFF02F058FEF4
:1002A000144C154DAC4203DA54F8041B8847F9E7A7
:1002B00000F042F8114C124DAC4203DA54F8041B22
:1002C0008847F9E701F0F6BE000600200022002072
:1002D0000000000808ED00E00000002000060020FB
:1002E0007837000800220020402200204022002011
:1002F000602E0020E0010008E0010008E001000895
:10030000E00100082DE9F04F2DED108AC1F80CD066
:10031000C3689D46BDEC108ABDE8F08F002383F3CF
:1003200011882846A047002001F072FAFEE701F08C
:1003300001FA00DFFEE7000038B500F0BBFB01F07A
:1003400087FE054601F0AAFE0446C8B90E4B9D4241
:1003500018D001339D4218BF044641F2883504BFCE
:1003600001240025002001F07DFE0CB100F074F89E
:1003700000F000FD284600F0BFF800F06DF8F9E746
:100380000025EFE70546EDE7010007B008B500F0EE
:1003900063FBA0F120035842584108BD07B541F264
:1003A0001203022101A8ADF8043000F073FB03B082
:1003B0005DF804FB38B5302383F3118817480368D0
:1003C0000BB101F0F1FA164A144800234FF47A7188
:1003D00001F0E0FA002383F31188124C236813B173
:1003E0002368013B2360636813B16368013B63606A
:1003F0000D4D2B7833B963687BB9022000F024FCE3
:10040000322363602B78032B07D163682BB902205A
:1004100000F01AFC4FF47A73636038BD402200206C
:10042000B50300086023002058220020084B1870F4
:1004300003280CD8DFE800F008050208022000F0CD
:10044000F9BB022000F0ECBB024B00225A6070475F
:100450005822002060230020234B244A10B51C465C
:10046000196801313FD004339342F9D16268A24246
:1004700039D31F4B9B6803F1006303F540439A4255
:1004800031D2002000F030FB0220FFF7CFFF194BE4
:100490001A6C00221A64196E1A66196E596C5A6425
:1004A000596E5A665A6E5A6942F080025A615A6908
:1004B00022F080025A615A691A6942F000521A61A8
:1004C0001A6922F000521A611B6972B64FF0E023DC
:1004D0003021C3F8084DD4E9003281F311889D46DC
:1004E00083F30888104710BD00C0000820C0000832
:1004F00000220020003802402DE9F04F93B0AA4BB3
:1005000000902022FF210AA89D6800F0DDFBA74A89
:100510001378A3B9A648012103601170302383F337
:10052000118803680BB101F03FFAA24AA0480023EA
:100530004FF47A7101F02EFA002383F31188009BA7
:1005400013B19D4B009A1A609C4A009C1378032BB0
:100550001EBF00231370984A4FF0000A18BF536063
:10056000D3465646D146012000F064FB24B1924B9D
:100570001B68002B00F01182002000F06DFA039040
:10058000039B002BF2DB012000F04AFB039B213B85
:10059000162BE8D801A252F823F000BFF905000895
:1005A00021060008B5060008670500086705000871
:1005B000670500083F0700080F0900082908000820
:1005C0008B080008B3080008D90800086705000870
:1005D000EB080008670500085D0900089906000897
:1005E00067050008A109000805060008990600082B
:1005F000670500088B0800080220FFF7C7FE0028E7
:1006000040F0F581009B0221BAF1000F08BF1C46A3
:1006100005A841F21233ADF8143000F03BFAA2E71E
:100620004FF47A7000F018FA071EEBDB0220FFF798
:10063000ADFE0028E6D0013F052F00F2DA81DFE8A9
:1006400007F0030A0D10133605230593042105A8AE
:1006500000F020FA17E054480421F9E75848042133
:10066000F6E758480421F3E74FF01C08404600F035
:100670003DFA08F104080590042105A800F00AFAE3
:10068000B8F12C0FF2D1012000FA07F747EA0B0B63
:100690005FFA8BFB4FF0000900F062FB26B10BF014
:1006A0000B030B2B08BF0024FFF778FE5BE74648DF
:1006B0000421CDE7002EA5D00BF00B030B2BA1D10D
:1006C0000220FFF763FE074600289BD0012000F0C0
:1006D0000BFA0220FFF7AAFE00261FFA86F8404612
:1006E00000F012FA044690B10021404600F01CFAD6
:1006F00001360028F1D1BA46044641F21213022114
:1007000005A8ADF814303E4600F0C4F92BE70120EF
:10071000FFF78CFE2546244B9B68AB4207D9284641
:1007200000F0E4F9013040F067810435F3E7234B32
:1007300000251D70204BBA465D603E46ACE7002E9A
:100740003FF460AF0BF00B030B2B7FF45BAF022089
:10075000FFF76CFE322000F07FF9B0F10008FFF6E1
:1007600051AF18F003077FF44DAF0F4A926808EBC2
:10077000050393423FF646AFB8F5807F3FF742AF9F
:10078000124B0193B84523DD4FF47A7000F064F901
:100790000390039A002AFFF635AF019B039A03F8F2
:1007A000012B0137EDE700BF002200205C23002071
:1007B00040220020B50300086023002058220020BA
:1007C00004220020082200200C2200205C220020AD
:1007D000C820FFF7DBFD074600283FF413AF1F2DAD
:1007E00011D8C5F1200242450AAB25F0030028BF0D
:1007F000424683490192184400F040FA019A804829
:10080000FF2100F061FA4FEAA8037D490193C8F384
:100810008702284600F060FA064600283FF46DAFD4
:10082000019B05EB830537E70220FFF7AFFD0028AA
:100830003FF4E8AE00F0A4F900283FF4E3AE00274F
:10084000B846704B9B68BB4218D91F2F11D80A9B22
:1008500001330ED027F0030312AA134453F8203CAF
:1008600005934046042205A900F0AEFA04378046FD
:10087000E7E7384600F03AF90590F2E7CDF8148042
:10088000042105A800F006F906E70023642104A866
:10089000049300F0F5F800287FF4B4AE0220FFF7CF
:1008A00075FD00283FF4AEAE049800F051F90590B4
:1008B000E6E70023642104A8049300F0E1F800288F
:1008C0007FF4A0AE0220FFF761FD00283FF49AAE4E
:1008D000049800F04DF9EAE70220FFF757FD0028E1
:1008E0003FF490AE00F05CF9E1E70220FFF74EFD27
:1008F00000283FF487AE05A9142000F057F9042121
:100900000746049004A800F0C5F83946B9E732203C
:1009100000F0A2F8071EFFF675AEBB077FF472AEBB
:10092000384A926807EB090393423FF66BAE022008
:10093000FFF72CFD00283FF465AE27F003074F4476
:10094000B9453FF4A9AE484600F0D0F8042105901F
:1009500005A800F09FF809F10409F1E74FF47A7057
:10096000FFF714FD00283FF44DAE00F009F9002810
:1009700044D00A9B01330BD008220AA9002000F0C2
:10098000ABF900283AD02022FF210AA800F09CF9F8
:10099000FFF704FD1C4800F041FF13B0BDE8F08FE5
:1009A000002E3FF42FAE0BF00B030B2B7FF42AAE7F
:1009B0000023642105A8059300F062F8074600288B
:1009C0007FF420AE0220FFF7E1FC804600283FF4D0
:1009D00019AEFFF7E3FC41F2883000F01FFF0598E5
:1009E00000F0F0F9464600F0BBF93C46BBE5064690
:1009F00052E64FF0000905E6BA467EE637467CE649
:100A00005C22002000220020A086010070B50F4B60
:100A10001B780133DBB2012B0C4611D80C4D296831
:100A20004FF47A730E6AA2FB03320146224628462F
:100A3000B047844204D1074B00221A70012070BDD8
:100A40004FF4FA7000F0EAFE0020F8E710220020D0
:100A5000082600209423002007B500230246012128
:100A60000DF107008DF80730FFF7D0FF20B19DF89A
:100A7000070003B05DF804FB4FF0FF30F9E700001A
:100A80000A4608B50421FFF7C1FF80F00100C0B29B
:100A9000404208BD30B4054C2368DD69044B0A466A
:100AA000AC460146204630BC604700BF0826002007
:100AB000A086010070B501F0D1F9094E094D3080D2
:100AC000002428683388834208D901F0C1F92B68D3
:100AD00004440133B4F5404F2B60F2D370BD00BF26
:100AE000962300206823002001F066BA00F1006020
:100AF00000F540400068704700F10060920000F58A
:100B0000404001F0F1B90000054B1A68054B1B8805
:100B10009B1A834202D9104401F09AB90020704711
:100B2000682300209623002038B5084D044629B1DB
:100B300028682044BDE8384001F0AAB9286820445C
:100B400001F08EF90028F3D038BD00BF68230020E3
:100B500010F003030AD1B0F5047F05D200F1005074
:100B6000A0F51040D0F80038184670470023FBE786
:100B700000F10050A0F51040D0F8100A70470000B6
:100B8000064991F8243033B10023086A81F82430F3
:100B90000822FFF7B1BF0120704700BF6C2300207F
:100BA000014B1868704700BF002004E070B5194B76
:100BB0001D68194B0138C5F30B0408442D0C0422A1
:100BC0001E88A6420BD15C680A46013C824213464D
:100BD0000FD214F9016F4EB102F8016BF6E7013A3A
:100BE00003F10803ECD181420B4602D22C2203F818
:100BF000012B0A4A05241688AE4204D1984284BFCC
:100C0000967803F8016B013C02F10402F3D1581A03
:100C100070BD00BF002004E0943400088034000858
:100C2000022802BF024B4FF480429A61704700BF16
:100C300000080240022802BF024B4FF080429A6136
:100C4000704700BF00080240022801BF024A5369F2
:100C500083F48043536170470008024070B5044636
:100C60004FF47A764CB1412C254628BF412506FB2E
:100C700005F000F0D3FD641BF4E770BD10B5002350
:100C8000934203D0CC5CC4540133F9E710BD00009B
:100C900010B5013810F9013F3BB191F900409C4279
:100CA00003D11AB10131013AF4E71AB191F90020E8
:100CB000981A10BD1046FCE703460246D01A12F9F6
:100CC000011B0029FAD1704702440346934202D027
:100CD00003F8011BFAE770472DE9F8431F4D14464E
:100CE00095F824200746884652BBDFF870909CB3E5
:100CF00095F824302BB92022FF2148462F62FFF7B8
:100D0000E3FF95F82400C0F10802A24228BF224662
:100D1000D6B24146920005EB8000FFF7AFFF95F891
:100D20002430A41B1E44F6B2082E17449044E4B2AB
:100D300085F82460DBD1FFF723FF0028D7D108E036
:100D40002B6A03EB82038342CFD0FFF719FF002801
:100D5000CBD10020BDE8F8830120FBE76C23002005
:100D6000024B1A78024B1A70704700BF9423002080
:100D70001022002010B5104C104800F0B5F82146A4
:100D80000E4800F0DDF82468626DD2F8043843F0B4
:100D90000203C2F804384FF47A70FFF75FFF084986
:100DA000204600F0D3F9626DD2F8043823F0020334
:100DB000C2F8043810BD00BF6035000808260020C6
:100DC000683500087047000030B5094D0A4491426B
:100DD0000DD011F8013B5840082340F30004013BBB
:100DE0002C4013F0FF0384EA5000F6D1EFE730BD4A
:100DF0002083B8ED026843681143016003B11847CE
:100E00007047000013B5446BD4F894341A68117815
:100E1000042915D1217C022912D1197912890123C3
:100E20008B4013420CD101A904F14C0001F0F8FEF3
:100E3000D4F89444019B21790246206800F0D0F94F
:100E400002B010BD143001F07BBE00004FF0FF3344
:100E5000143001F075BE00004C3001F04DBF0000B1
:100E60004FF0FF334C3001F047BF0000143001F069
:100E700049BE00004FF0FF31143001F043BE0000C6
:100E80004C3001F019BF00004FF0FF324C3001F040
:100E900013BF00000020704710B5D0F894341A68D2
:100EA00011780429044617D1017C022914D15979FB
:100EB000528901238B4013420ED1143001F0DCFD26
:100EC000024648B1D4F894444FF4807361792068A5
:100ED000BDE8104000F072B910BD0000406BFFF794
:100EE000DBBF0000704700007FB5124B036000239A
:100EF0004360C0E90233012502260F4B0574044606
:100F00000290019300F18402294600964FF4807309
:100F1000143001F08DFD094B0294CDE9006304F516
:100F200023724FF48073294604F14C0001F054FE03
:100F300004B070BDB4340008DD0E0008050E0008D2
:100F40000B68302282F311880A7903EB82029061E8
:100F50004A79093243F822008A7912B103EB8203FD
:100F600098610223C0F894140374002080F3118860
:100F70007047000038B5037F044613B190F8543031
:100F8000ABB9201D01250221FFF734FF04F1140045
:100F900025776FF0010100F069FC84F8545004F1EA
:100FA0004C006FF00101BDE8384000F05FBC38BD77
:100FB00010B5012104460430FFF71CFF00232377FE
:100FC00084F8543010BD000038B5044600251430B4
:100FD00001F046FD04F14C00257701F015FE201DBF
:100FE00084F854500121FFF705FF2046BDE8384042
:100FF000FFF752BF90F8443003F06003202B07D175
:1010000090F84520212A4FF0000303D81F2A06D864
:1010100000207047222AFBD1C0E90E3303E0034AC7
:1010200082630722C26303640120704711220020FB
:1010300037B5D0F894341A681178042904461AD1C7
:10104000017C022917D11979128901238B4013429F
:1010500011D100F14C05284601F096FE58B101A9C6
:10106000284601F0DDFDD4F89444019B2179024625
:10107000206800F0B5F803B030BD0000F0B500EB1B
:10108000810385B09E6904460D46FEB1302383F38B
:10109000118804EB8507301D0821FFF7ABFEFB68C4
:1010A0005B691B6806F14C001BB1019001F0C6FDA5
:1010B000019803A901F0B4FD024648B1039B2946FB
:1010C000204600F08DF8002383F3118805B0F0BDB1
:1010D000FB685A691268002AF5D01B8A013B13404D
:1010E000F1D104F14402EAE7093138B550F8214062
:1010F000DCB1302383F31188D4F894241368527937
:1011000003EB8203DB689B695D6845B104216018CD
:10111000FFF770FE294604F1140001F0B7FC2046E9
:10112000FFF7BAFE002383F3118838BD7047000033
:1011300001F016B8012303700023C0E90133C36135
:1011400083620362C36243620363704738B5044637
:10115000302383F311880025C0E90355C0E9055504
:10116000416001F00DF80223237085F311882846B1
:1011700038BD000070B500EB810305465069DA60A8
:101180000E46144618B110220021FFF79DFDA069FC
:1011900018B110220021FFF797FD31462846BDE81F
:1011A000704001F0B7B80000826802F0011282605E
:1011B0000022C0E90422826101F038B9F0B400EBEA
:1011C00081044789E4680125A4698D403D43458138
:1011D00023600023A2606360F0BC01F053B90000FB
:1011E000F0B400EB81040789E468012564698D404F
:1011F0003D43058123600023A2606360F0BC01F0E1
:10120000CDB9000070B50223002504460370C0E983
:101210000255C0E90455C564856180F8345001F079
:1012200015F863681B6823B129462046BDE8704065
:10123000184770BD0378052B10B504460AD080F816
:1012400050300523037043681B680BB10421984795
:101250000023A36010BD00000178052906D190F895
:101260005020436802701B6803B1184770470000A4
:1012700070B590F83430044613B1002380F8343050
:1012800004F14402204601F0F3F863689B68B3B9A7
:1012900094F8443013F0600535D00021204601F069
:1012A00093FB0021204601F085FB63681B6813B1A6
:1012B000062120469847062384F8343070BD204626
:1012C00098470028E4D0B4F84A30E26B9A4288BFCD
:1012D000E36394F94430E56B002B4FF0300380F268
:1012E0000381002D00F0F280092284F8342083F37A
:1012F00011880021D4E90E232046FFF771FF002357
:1013000083F31188DAE794F8452003F07F0343EA7A
:10131000022340F20232934200F0C58021D8B3F597
:10132000807F48D00DD8012B3FD0022B00F0938056
:10133000002BB2D104F14C02A2630222E2632364C7
:10134000C1E7B3F5817F00F09B80B3F5407FA4D166
:1013500094F84630012BA0D1B4F84C3043F002038E
:1013600032E0B3F5006F4DD017D8B3F5A06F31D090
:10137000A3F5C063012B90D8636894F846205E689B
:1013800094F84710B4F848302046B047002884D07D
:101390004368A3630368E3631AE0B3F5106F36D0C4
:1013A00040F6024293427FF478AF5C4BA363022382
:1013B000E3630023C3E794F84630012B7FF46DAF5D
:1013C000B4F84C3023F00203C4E90E55A4F84C30B5
:1013D000256478E7B4F84430B3F5A06F0ED194F8E3
:1013E000463084F84E30204600F088FF63681B6862
:1013F00013B1012120469847032323700023C4E939
:101400000E339CE704F14F03A3630123C3E7237862
:10141000042B10D1302383F311882046FFF7C4FE3C
:1014200085F311880321636884F84F5021701B688D
:101430000BB12046984794F84630002BDED084F854
:101440004F300423237063681B68002BD6D0022121
:1014500020469847D2E794F848301D0603F00F0164
:1014600020460AD500F0F6FF012804D002287FF4B8
:1014700014AF2B4B9AE72B4B98E700F0DDFFF3E717
:1014800094F84630002B7FF408AF94F8483013F0FE
:101490000F01B3D01A06204602D501F0A9FAADE734
:1014A00001F09CFAAAE794F84630002B7FF4F5AEE1
:1014B00094F8483013F00F01A0D01B06204602D547
:1014C00001F082FA9AE701F075FA97E7142284F89E
:1014D000342083F311882B462A4629462046FFF7FD
:1014E0006DFE85F31188E9E65DB1152284F834209C
:1014F00083F311880021D4E90E232046FFF75EFE16
:10150000FDE60B2284F8342083F311882B462A460B
:1015100029462046FFF764FEE3E700BFE4340008F5
:10152000DC340008E034000838B590F83430044664
:10153000002B3ED0063BDAB20F2A34D80F2B32D81C
:10154000DFE803F0373131082232313131313131C6
:1015500031313737C56BB0F84A309D4214D2C36879
:101560001B8AB5FBF3F203FB12556DB9302383F3ED
:1015700011882B462A462946FFF732FE85F311884B
:101580000A2384F834300EE0142384F834303023F6
:1015900083F3118800231A4619462046FFF70EFEF2
:1015A000002383F3118838BD036C03B198470023EF
:1015B000E7E70021204601F007FA0021204601F06C
:1015C000F9F963681B6813B1062120469847062382
:1015D000D7E7000010B590F83430142B044629D01A
:1015E00017D8062B05D001D81BB110BD093B022B23
:1015F000FBD80021204601F0E7F90021204601F048
:10160000D9F963681B6813B1062120469847062361
:1016100019E0152BE9D10B2380F83430302383F304
:10162000118800231A461946FFF7DAFD002383F3D9
:101630001188DAE7C3689B695B68002BD5D1036C1E
:1016400003B19847002384F83430CEE700230375B4
:10165000826803691B6899689142FBD25A680360EB
:101660004260106058607047002303758268036908
:101670001B6899689142FBD85A6803604260106009
:101680005860704708B50846302383F311880B7DF6
:10169000032B05D0042B0DD02BB983F3118808BD83
:1016A0008B6900221A604FF0FF338361FFF7CEFF92
:1016B0000023F2E7D1E9003213605A60F3E700003B
:1016C000FFF7C4BF054BD9680875186802681A602F
:1016D000536001220275D860FEF714BE98230020E3
:1016E00030B50C4BDD684B1C87B004460FD02B4641
:1016F000094A684600F04EF92046FFF7E3FF009BD9
:1017000013B1684600F050F9A86907B030BDFFF783
:10171000D9FFF9E79823002085160008044B1A68C2
:10172000DB6890689B68984294BF00200120704756
:1017300098230020084B10B51C68D86822681A60EE
:10174000536001222275DC60FFF78EFF01462046C0
:10175000BDE81040FEF7D6BD9823002038B5074CF1
:1017600007490848012300252370656001F044FB08
:101770000223237085F3118838BD00BF00260020A6
:10178000EC3400089823002000F044B9034A516863
:1017900053685B1A9842FBD8704700BF001000E006
:1017A0008B60022308618B82084670478368A3F12F
:1017B000840243F8142C026943F8442C426943F82C
:1017C000402C094A43F8242CC26843F8182C022202
:1017D00003F80C2C002203F80B2C044A43F8102CBD
:1017E000A3F12000704700BF1D03000898230020CC
:1017F00008B5FFF7DBFFBDE80840FFF761BF000059
:10180000024BDB6898610F20FFF75CBF9823002034
:10181000302383F31188FFF7F3BF000008B50146BA
:10182000302383F311880820FFF75AFF002383F346
:10183000118808BD064BDB6839B1426818605A60F0
:10184000136043600420FFF74BBF4FF0FF30704739
:10185000982300200368984206D01A6802605060FE
:1018600099611846FFF72CBF7047000038B5044651
:101870000D462068844200D138BD036823605C6057
:101880008561FFF71DFFF4E710B503689C68A2426D
:101890000CD85C688A600B604C6021605960996864
:1018A0008A1A9A604FF0FF33836010BD1B68121BC9
:1018B000ECE700000A2938BF0A2170B504460D463E
:1018C0000A26601901F092FA01F07EFA041BA54283
:1018D00003D8751C2E460446F3E70A2E04D9BDE84A
:1018E0007040012001F0C8BA70BD0000F8B5144B7B
:1018F0000D46D96103F1100141600A2A196982601D
:1019000038BF0A22016048601861A818144601F027
:101910005FFA0A2701F058FA431BA342064606D392
:101920007C1C281901F062FA27463546F2E70A2F97
:1019300004D9BDE8F840012001F09EBAF8BD00BF0F
:1019400098230020F8B506460D4601F03DFA0F4AEF
:10195000134653F8107F9F4206D12A46014630466F
:10196000BDE8F840FFF7C2BFD169BB68441A2C1923
:1019700028BF2C46A34202D92946FFF79BFF2246E7
:1019800031460348BDE8F840FFF77EBF98230020AA
:10199000A823002010B4C0E9032300235DF8044B02
:1019A0004361FFF7CFBF000010B5194C236998427F
:1019B0000DD0D0E90032816813605A609A680A44F9
:1019C0009A60002303604FF0FF33A36110BD2346EC
:1019D000026843F8102F53600022026022699A4285
:1019E00003D1BDE8104001F0FBB9936881680B4456
:1019F000936001F0E9F92269E1699268441AA24210
:101A0000E4D91144BDE81040091AFFF753BF00BFE5
:101A1000982300202DE9F047DFF8BC8008F110077B
:101A20002C4ED8F8105001F0CFF9D8F81C40AA6815
:101A3000031B9A423ED81444D5E900324FF0000906
:101A4000C8F81C4013605A60C5F80090D8F81030F0
:101A5000B34201D101F0C4F989F31188D5E903310A
:101A600028469847302383F311886B69002BD8D020
:101A700001F0AAF96A69A0EB04094A4582460DD231
:101A8000022001F0F9F90022D8F81030B34208D151
:101A900051462846BDE8F047FFF728BF121A2244F6
:101AA000F2E712EB090938BF4A4629463846FFF7E4
:101AB000EBFEB5E7D8F81030B34208D01444211A31
:101AC000C8F81C00A960BDE8F047FFF7F3BEBDE809
:101AD000F08700BFA8230020982300200020704733
:101AE000FEE70000704700004FF0FF307047000035
:101AF00002290CD0032904D00129074818BF00206F
:101B00007047032A05D8054800EBC2007047044817
:101B100070470020704700BFC43500082022002015
:101B20007835000870B59AB00546084601A91446F4
:101B300000F0C2F801A8FFF7BFF8431C5B00C5E93D
:101B400000340022237003236370C6B201AB023459
:101B50001046D1B28E4204F1020401D81AB070BD11
:101B600013F8011B04F8021C04F8010C0132F0E721
:101B700008B5302383F311880348FFF759FA00238F
:101B800083F3118808BD00BF0826002090F8443078
:101B900003F01F02012A07D190F845200B2A03D138
:101BA0000023C0E90E3315E003F06003202B08D1B9
:101BB000B0F848302BB990F84520212A03D81F2AC5
:101BC00004D8FFF717BA222AEBD0FAE7034A826358
:101BD0000722C26303640120704700BF182200205F
:101BE00007B5052917D8DFE801F0191603191920E0
:101BF000302383F31188104A01900121FFF7BAFACC
:101C000001980E4A0221FFF7B5FA0D48FFF7DCF9FB
:101C1000002383F3118803B05DF804FB302383F3C2
:101C200011880748FFF7A6F9F2E7302383F31188FC
:101C30000348FFF7BDF9EBE7183500083C3500080D
:101C40000826002038B50C4D0C4C0D492A4604F1ED
:101C50000800FFF767FF05F1CA0204F11000094907
:101C6000FFF760FF05F5CA7204F118000649BDE8E8
:101C70003840FFF757BF00BFD02A002020220020A5
:101C8000F8340008023500080D35000870B5044628
:101C900008460D46FFF710F8C6B220460134037817
:101CA0000BB9184670BD32462946FEF7F1FF0028F1
:101CB000F3D10120F6E700002DE9F04705460C4678
:101CC000FEF7FAFF2B49C6B22846FFF7DFFF08B13F
:101CD0000636F6B228492846FFF7D8FF08B1103675
:101CE000F6B2632E0BD8DFF88C80DFF88C90234F90
:101CF000DFF894A02E7846B92670BDE8F087294613
:101D00002046BDE8F04701F09DBB252E2ED10722CD
:101D100041462846FEF7BCFF70B9194B224603F135
:101D20000C0153F8040B42F8040B8B42F9D11B78D9
:101D3000137007350D34DDE7082249462846FEF7C3
:101D4000A7FF98B90F4BA21C197809090232C95D87
:101D500002F8041C13F8011B01F00F015345C95D83
:101D600002F8031CF0D118340835C3E704F8016BFE
:101D70000135BFE7E43500080D350008FA350008E5
:101D8000EC350008107AFF1F1C7AFF1FBFF34F8F3E
:101D9000024AD368DB03FCD4704700BF003C02401A
:101DA00008B5094B1B7873B9FFF7F0FF074B1A69A9
:101DB000002ABFBF064A5A6002F188325A601A6888
:101DC00022F480621A6008BD2E2D0020003C0240E3
:101DD0002301674508B50B4B1B7893B9FFF7D6FF76
:101DE000094B1A6942F000421A611A6842F48052A3
:101DF0001A601A6822F480521A601A6842F48062EB
:101E00001A6008BD2E2D0020003C02400B28F0B5C2
:101E100016D80C4C0C4923787BB90C4D0E460C237C
:101E20004FF0006255F8047B46F8042B013B13F099
:101E3000FF033A44F6D10123237051F82000F0BD8E
:101E40000020FCE7602D0020302D00200C3600081B
:101E5000014B53F8200070470C3600080C207047E7
:101E60000B2810B5044601D9002010BDFFF7CEFFA6
:101E7000064B53F824301844C21A0BB90120F4E77A
:101E800012680132F0D1043BF6E700BF0C360008BF
:101E90000B2810B5044621D8FFF778FFFFF780FF25
:101EA0000F4AF323D360C300DBB243F4007343F063
:101EB00002031361136943F480331361FFF766FF74
:101EC000FFF7A4FF074B53F8241000F0D9F8FFF7F1
:101ED00081FF2046BDE81040FFF7C2BF002010BDC3
:101EE000003C02400C360008F8B512F0010314461D
:101EF00042D18218B2F1016F57D82D4B1B6813F0F5
:101F0000010352D02B4DFFF74BFFF323EB60FFF79C
:101F10003DFF40F20127032C15D824F00104661878
:101F2000244C401A40F20117B142236900EB01052D
:101F300024D123F001032361FFF74CFF0120F8BDFA
:101F4000043C0430E7E78307E7D12B6923F44073AF
:101F50002B612B693B432B6151F8046B0660BFF387
:101F60004F8FFFF713FF03689E42E9D02B6923F0E0
:101F700001032B61FFF72EFF0020E0E723F44073FD
:101F8000236123693B4323610B882B80BFF34F8F71
:101F9000FFF7FCFE2D8831F8023BADB2AB42C3D057
:101FA000236923F001032361E4E71846C7E700BF74
:101FB00000380240003C0240084908B50B7828B1BF
:101FC0001BB9FFF7EDFE01230B7008BD002BFCD001
:101FD000BDE808400870FFF7FDBE00BF2E2D0020B1
:101FE00010B50244064BD2B2904200D110BD441C41
:101FF00000B253F8200041F8040BE0B2F4E700BF50
:10200000502800400F4B30B51C6F240407D41C6FC0
:1020100044F400741C671C6F44F400441C670A4CB1
:10202000236843F4807323600244084BD2B2904289
:1020300000D130BD441C00B251F8045B43F820507D
:10204000E0B2F4E700380240007000405028004041
:1020500007B5012201A90020FFF7C2FF019803B0D4
:102060005DF804FB13B50446FFF7F2FFA04205D06C
:10207000012201A900200194FFF7C4FF02B010BDA6
:1020800070470000034B1A681AB9034AD2F8742843
:102090001A607047642D00200030024008B5FFF739
:1020A000F1FF024B1868C0F3407008BD642D00209A
:1020B00070470000FEE700000A4B0B480B4A9042B5
:1020C0000BD30B4BDA1C121AC11E22F003028B42F7
:1020D00038BF00220021FEF7F7BD53F8041B40F87B
:1020E000041BECE7B8370008602E0020602E0020AB
:1020F000602E002070B5D0E915439E6800224FF095
:10210000FF3504EB42135101D3F800090028BEBF8C
:10211000D3F8000940F08040C3F80009D3F8000B61
:102120000028BEBFD3F8000B40F08040C3F8000B7E
:10213000013263189642C3F80859C3F8085BE0D22D
:102140004FF00113C4F81C3870BD0000890141F044
:102150002001016103699B06FCD41220FFF716BB26
:1021600010B5054C2046FEF7E5FF4FF0A043636530
:10217000024BA36510BD00BF682D0020603600082B
:1021800070B50378012B054650D12A4B446D984217
:102190001BD1294B5A6B42F080025A635A6D42F0B0
:1021A00080025A655A6D5A6942F080025A615A6932
:1021B00022F080025A610E2143205B6900F022FC6C
:1021C0001E4BE3601E4BC4F800380023C4F8003EE9
:1021D000C02323606E6D4FF40413A3633369002B97
:1021E000FCDA012333610C20FFF7D0FA3369DB07F7
:1021F000FCD41220FFF7CAFA3369002BFCDA002660
:10220000A6602846FFF776FF6B68C4F81068DB68A5
:10221000C4F81468C4F81C684BB90A4BA3614FF0AA
:10222000FF336361A36843F00103A36070BD064BF5
:10223000F4E700BF682D0020003802404014004041
:1022400003002002003C30C0083C30C0F8B5446DAB
:10225000054600212046FFF779FFA96D00234FF0C6
:1022600001128F68C4F834384FF00066C4F81C2897
:102270004FF0FF3004EB431201339F42C2F8006974
:10228000C2F8006BC2F80809C2F8080BF2D20B685A
:102290006A6DEB65636210231361166916F0100610
:1022A000FBD11220FFF772FAD4F8003823F4FE6352
:1022B000C4F80038A36943F4402343F01003A3613A
:1022C0000923C4F81038C4F814380A4BEB604FF0F7
:1022D000C043C4F8103B084BC4F8003BC4F8106975
:1022E000C4F80039EB6D03F1100243F48013EA6582
:1022F000A362F8BD3C36000840800010426D90F8A3
:102300004E10D2F8003823F4FE6343EA0113C2F8FA
:10231000003870472DE9F84300EB8103456DDA681A
:10232000166806F00306731E022B05EB41130C46DC
:1023300080460FFA81F94FEA41104FF00001C3F8CF
:10234000101B4FF0010104F1100398BFB60401FA0D
:1023500003F391698EBF334E06F1805606F50046B1
:1023600000293AD0578A04F15801490137436F5088
:10237000D5F81C180B43C5F81C382B180021C3F8DE
:10238000101953690127611EA7409BB3138A928BD2
:102390009B08012A88BF5343D8F85C20981842EA6A
:1023A000034301F1400205EB8202C8F85C002146BC
:1023B00053602846FFF7CAFE08EB8900C3681B8AF2
:1023C00043EA8453483464011E432E51D5F81C3827
:1023D0001F43C5F81C78BDE8F88305EB4917D7F80B
:1023E000001B21F40041C7F8001BD5F81C1821EA96
:1023F0000303C0E704F13F0305EB83030A4A5A6075
:1024000028462146FFF7A2FE05EB4910D0F8003917
:1024100023F40043C0F80039D5F81C3823EA070735
:10242000D7E700BF0080001000040002826D126830
:10243000C265FFF75FBE00005831436D49015B582C
:1024400013F4004004D013F4001F0CBF022001203D
:10245000704700004831436D49015B5813F4004058
:1024600004D013F4001F0CBF0220012070470000AD
:1024700000EB8101CB68196A0B6813604B685360ED
:102480007047000000EB810330B5DD68AA6913686E
:10249000D36019B9402B84BF402313606B8A146842
:1024A000426D1C44013CB4FBF3F46343033323F05B
:1024B000030302EB411043EAC44343F0C043C0F8B6
:1024C000103B2B6803F00303012B09B20ED1D2F8A5
:1024D000083802EB411013F4807FD0F8003B14BFA2
:1024E00043F0805343F00053C0F8003B02EB41122D
:1024F000D2F8003B43F00443C2F8003B30BD00007B
:102500002DE9F041244D6E6D06EB40130446D3F8DF
:10251000087BC3F8087B38070AD5D6F814381907A2
:1025200006D505EB84032146DB6828465B6898479F
:10253000FA071FD5D6F81438DB071BD505EB840343
:10254000D968CCB98B69488A5A68B2FBF0F600FBAF
:1025500016228AB91868DA6890420DD2121AC3E9B5
:102560000024302383F311880B482146FFF78AFFAC
:1025700084F31188BDE8F081012303FA04F26B892A
:1025800023EA02036B81CB68002BF3D0214602487B
:10259000BDE8F041184700BF682D002000EB810323
:1025A00070B5DD68436D6C692668E6604A0156BB0C
:1025B0001A444FF40020C2F810092A6802F00302FE
:1025C000012A0AB20ED1D3F8080803EB421410F422
:1025D000807FD4F8000914BF40F0805040F00050D4
:1025E000C4F8000903EB4212D2F8000940F004409D
:1025F000C2F80009D3F83408012202FA01F10143BC
:10260000C3F8341870BD19B9402E84BF4020206033
:1026100020682E8A8419013CB4FBF6F440EAC440D9
:1026200040F000501A44C6E72DE9F8433B4D6E6D6B
:1026300006EB40130446D3F80889C3F8088918F05C
:10264000010F4FEA40171AD0D6F81038DB0716D51D
:1026500005EB8003D9684B691868DA68904230D27C
:10266000121A4FF000091A60C3F80490302383F364
:10267000118821462846FFF791FF89F3118818F049
:10268000800F1CD0D6F834380126A640334216D02D
:1026900005EB84036D6DD3F80CC0DCF81420013415
:1026A000E4B2D2F800E005EB04342F4451687145E0
:1026B00015D3D5F8343823EA0606C5F83468BDE8E2
:1026C000F883012303FA04F22B8923EA02032B8106
:1026D0008B68002BD3D0214628469847CFE7BCF81B
:1026E0001000AEEB0103834228BF0346D7F8180958
:1026F00080B2B3EB800FE2D89068A0F1040959F8DA
:10270000048FC4F80080A0EB09089844B8F1040FC6
:10271000F5D818440B4490605360C7E7682D00203B
:102720002DE9F74FA24C656D6E69AB691E4016F43A
:1027300080586E6107D02046FEF764FD03B0BDE807
:10274000F04F00F047BC002E12DAD5F8003E984852
:102750009B071EBFD5F8003E23F00303C5F8003EDB
:10276000D5F8043823F00103C5F80438FEF774FDEA
:10277000370505D58E48FFF7BDFC8D48FEF75AFD9D
:10278000B0040CD5D5F8083813F0060FEB6823F425
:1027900070530CBF43F4105343F4A053EB60310764
:1027A0001BD56368DB681BB9AB6923F00803AB6119
:1027B0002378052B0CD1D5F8003E7D489A071EBF23
:1027C000D5F8003E23F00303C5F8003EFEF744FDB4
:1027D0006368DB680BB176489847F30274D4B7029C
:1027E00027D5D4F85490DFF8C8B100274FF0010A7C
:1027F00009EB4712D2F8003B03F44023B3F5802FD6
:1028000011D1D2F8003B002B0DDA62890AFA07F3E6
:1028100022EA0303638104EB8703DB68DB6813B1FF
:10282000394658469847A36D01379B68FFB29F42CF
:10283000DED9F00617D5676D3A6AC2F30A1002F0C6
:102840000F0302F4F012B2F5802F00F08580B2F58C
:10285000402F08D104EB83030022DB681B6A07F5D5
:10286000805790426AD13003D5F8184813D5E10358
:1028700002D50020FFF744FEA20302D50120FFF796
:102880003FFE630302D50220FFF73AFE270302D57D
:102890000320FFF735FE75037FF550AFE00702D543
:1028A0000020FFF7C1FEA10702D50120FFF7BCFE03
:1028B000620702D50220FFF7B7FE23077FF53EAF80
:1028C0000320FFF7B1FE39E7636DDFF8E4A0019361
:1028D00000274FF00109A36D9B685FFA87FB9B45BA
:1028E0003FF67DAF019B03EB4B13D3F8001901F4C6
:1028F0004021B1F5802F1FD1D3F8001900291BDA30
:10290000D3F8001941F09041C3F80019D3F8001929
:102910000029FBDB5946606DFFF718FC218909FA95
:102920000BF321EA0303238104EB8B03DB689B6831
:1029300013B15946504698470137CCE7910708BF75
:10294000D7F80080072A98BF03F8018B02F1010233
:1029500098BF4FEA182884E7023304EB830207F597
:1029600080575268D2F818C0DCF80820DCE9001C57
:10297000A1EB0C0C002188420AD104EB83046368AC
:102980009B699A6802449A605A6802445A606AE7EE
:1029900011F0030F08BFD7F800808C4588BF02F8FC
:1029A000018B01F1010188BF4FEA1828E3E700BF5E
:1029B000682D0020436D03EB4111D1F8003B43F437
:1029C0000013C1F8003B7047436D03EB4111D1F890
:1029D000003943F40013C1F800397047436D03EB2D
:1029E0004111D1F8003B23F40013C1F8003B7047BC
:1029F000436D03EB4111D1F8003923F40013C1F802
:102A00000039704700F1604303F561430901C9B221
:102A100083F80013012200F01F039A4043099B0032
:102A200003F1604303F56143C3F880211A607047E6
:102A300030B5039C0172043304FB0325C0E906533F
:102A4000049B03630021059BC160C0E90000C0E94D
:102A50000422C0E90842C0E90A11436330BD000006
:102A6000416A0022C0E90411C0E90A22C2606FF085
:102A70000101FEF7FBBE0000D0E90432934201D110
:102A8000C2680AB9181D70470020704703691960B1
:102A9000C2680132C260C269134482690361934211
:102AA00024BF436A03610021FEF7D4BE38B5044653
:102AB0000D46E3683BB16269131D1268A3621344BB
:102AC000E362002007E0237A33B929462046FEF767
:102AD000B1FE0028EDDA38BD6FF00100FBE7000021
:102AE000C368C269013BC36043691344826943619F
:102AF000934224BF436A436100238362036B03B1A3
:102B00001847704770B53023044683F31188866AEE
:102B10003EB9FFF7CBFF054618B186F3118828466A
:102B200070BDA36AE26A13F8015BA362934202D309
:102B30002046FFF7D5FF002383F31188EFE700005D
:102B40002DE9F84F04460E46174698464FF03009D7
:102B500089F311880025AA46D4F828B0BBF1000FEC
:102B600009D141462046FFF7A1FF20B18BF3118820
:102B70002846BDE8F88FD4E90A12A7EB050B521AD4
:102B8000934528BF9346BBF1400F1BD9334601F153
:102B9000400251F8040B43F8040B9142F9D1A36AA7
:102BA00040334036A3624035D4E90A239A4202D327
:102BB0002046FFF795FF8AF31188BD42D8D289F3EA
:102BC0001188C9E730465A46FEF758F8A36A5B44B5
:102BD0005E44A3625D44E7E710B5029C01720433D2
:102BE00003FB0421C0E906130023C0E90A33039B59
:102BF0000363049BC460C0E90000C0E90422C0E98B
:102C00000842436310BD0000026AC260426AC0E924
:102C100004220022C0E90A226FF00101FEF726BE5D
:102C2000D0E904239A4201D1C26822B9184650F86B
:102C3000043B0B60704700231846FAE7C368C2697B
:102C40000133C3604369134482694361934224BFE3
:102C5000436A43610021FEF7FDBD000038B504461C
:102C60000D46E3683BB123691A1DA262E269134471
:102C7000E362002007E0237A33B929462046FEF7B5
:102C8000D9FD0028EDDA38BD6FF00100FBE7000048
:102C900003691960C268013AC260C269134482695B
:102CA0000361934224BF436A036100238362036B81
:102CB00003B118477047000070B530230D46044635
:102CC000114683F31188866A2EB9FFF7C7FF10B14A
:102CD00086F3118870BDA36A1D70A36AE26A01338E
:102CE0009342A36204D3E16920460439FFF7D0FF81
:102CF000002080F31188EDE72DE9F84F04460D46DA
:102D0000904699464FF0300A8AF311880026B34660
:102D1000A76A4FB949462046FFF7A0FF20B187F3C5
:102D200011883046BDE8F88FD4E90A073A1AA8EBB3
:102D30000607974228BF1746402F1BD905F14003CD
:102D400055F8042B40F8042B9D42F9D1A36A403377
:102D5000A3624036D4E90A239A4204D3E1692046AB
:102D60000439FFF795FF8BF311884645D9D28AF3D2
:102D70001188CDE729463A46FDF780FFA36A3B4418
:102D80003D44A3623E44E5E7D0E904239A4217D1CB
:102D9000C3689BB1836A8BB1043B9B1A0ED013604E
:102DA000C368013BC360C3691A44836902619A42E4
:102DB00024BF436A036100238362012318467047DE
:102DC0000023FBE700F030B94FF08043586A7047AA
:102DD0004FF08043002258631A610222DA60704784
:102DE0004FF080430022DA60704700004FF08043CC
:102DF00058637047FEE7000070B51B4B0163002568
:102E0000044686B0586085620E4600F0BFF804F1B3
:102E10001003C4E904334FF0FF33C4E90635C4E9B5
:102E20000044A560E562FFF7CFFF2B460246C4E9E8
:102E3000082304F134010D4A256580232046FEF75E
:102E4000AFFC0123E0600A4A0375009272680192A8
:102E5000B268CDE90223074B6846CDE90435FEF799
:102E6000C7FC06B070BD00BF002600206C3600080D
:102E700071360008F52D0008024AD36A1843D06263
:102E8000704700BF982300204B6843608B688360C5
:102E9000CB68C3600B6943614B6903628B69436212
:102EA0000B6803607047000008B5264B26481A6976
:102EB00040F2FF110A431A611A6922F4FF7222F0EC
:102EC00001021A611A691A6B0A431A631A6D0A43DE
:102ED0001A651E4A1B6D1146FFF7D6FF02F11C0151
:102EE00000F58060FFF7D0FF02F1380100F5806047
:102EF000FFF7CAFF02F1540100F58060FFF7C4FF3D
:102F000002F1700100F58060FFF7BEFF02F18C0155
:102F100000F58060FFF7B8FF02F1A80100F58060BE
:102F2000FFF7B2FF02F1C40100F58060FFF7ACFFCC
:102F300002F1E00100F58060FFF7A6FFBDE8084060
:102F400000F0EEB800380240000002407836000879
:102F500008B500F059FAFEF701FCFFF793F8BDE859
:102F60000840FEF76FBE000070470000EFF30983D2
:102F700005494A6B22F001024A63683383F30988EA
:102F8000002383F31188704700EF00E0302080F3C6
:102F9000118862B60C4B0D4AD96821F4E06109042E
:102FA000090C0A43DA60D3F8FC20094942F0807228
:102FB000C3F8FC200A6842F001020A602022DA7796
:102FC00083F82200704700BF00ED00E00003FA051F
:102FD000001000E010B5302383F311880E4B5B68BE
:102FE00013F4006314D0F1EE103AEFF30984683C57
:102FF0004FF08073E361094BDB6B236684F3098830
:10300000FEF78CFB10B1064BA36110BD054BFBE72F
:1030100083F31188F9E700BF00ED00E000EF00E066
:103020002F030008320300080F4B1A6C42F0010214
:103030001A641A6E42F001021A660C4A1B6E9368FB
:1030400043F0010393604FF0804353229A624FF0A4
:10305000FF32DA6200229A615A63DA605A60012212
:103060005A611A60704700BF00380240002004E037
:103070004FF0804208B51169D3680B40D9B2C943FB
:103080009B07116107D5302383F31188FEF77CFB82
:10309000002383F3118808BD1F4B1A696FEAC252DF
:1030A0006FEAD2521A611A69C2F308021A614FF02C
:1030B000FF301A695A69586100215A6959615A6981
:1030C0001A6A62F080521A621A6A02F080521A6218
:1030D0001A6A5A6A58625A6A59625A6A1A6C42F0F3
:1030E00080521A641A6E42F080521A661A6E0B4AA7
:1030F000106840F480701060186F00F44070B0F5F4
:10310000007F1EBF4FF4803018671967536823F49F
:103110000073536000F054B9003802400070004062
:10312000334B4FF080521A64324A4FF440411160E1
:103130001A6842F001021A601A689107FCD59A6871
:1031400022F003029A602A4B9A6812F00C02FBD11B
:10315000196801F0F90119609A601A6842F4803226
:103160001A601A689203FCD55A6F42F001025A673E
:103170001F4B5A6F9007FCD51F4A5A601A6842F0DD
:1031800080721A601B4A53685904FCD5184B1A68A0
:103190009201FCD5194A9A60194B1A68194B9A4248
:1031A000194B21D1194A1168194A91421CD140F298
:1031B00005121A60144A136803F00F03052BFAD1A5
:1031C0000B4B9A6842F002029A609A6802F00C0275
:1031D000082AFAD15A6C42F480425A645A6E42F478
:1031E00080425A665B6E704740F20572E1E700BFAD
:1031F00000380240007000400854400700948838AE
:10320000002004E011640020003C024000ED00E0DA
:1032100041C20F41074A08B5536903F001035361E6
:1032200023B1054A13680BB150689847BDE80840C0
:10323000FFF7D0BE003C0140E02D0020074A08B552
:10324000536903F00203536123B1054A93680BB13C
:10325000D0689847BDE80840FFF7BCBE003C01407D
:10326000E02D0020074A08B5536903F004035361B9
:1032700023B1054A13690BB150699847BDE808406E
:10328000FFF7A8BE003C0140E02D0020074A08B52A
:10329000536903F00803536123B1054A93690BB1E5
:1032A000D0699847BDE80840FFF794BE003C014054
:1032B000E02D0020074A08B5536903F0100353615D
:1032C00023B1054A136A0BB1506A9847BDE808401C
:1032D000FFF780BE003C0140E02D0020164B10B5EA
:1032E0005C6904F478725A61A30604D5134A936AA0
:1032F0000BB1D06A9847600604D5104A136B0BB126
:10330000506B9847210604D50C4A936B0BB1D06BD8
:103310009847E20504D5094A136C0BB1506C9847E5
:10332000A30504D5054A936C0BB1D06C9847BDE852
:103330001040FFF74FBE00BF003C0140E02D0020D1
:10334000194B10B55C6904F47C425A61620504D5DE
:10335000164A136D0BB1506D9847230504D5134AD7
:10336000936D0BB1D06D9847E00404D50F4A136EEE
:103370000BB1506E9847A10404D50C4A936E0BB163
:10338000D06E9847620404D5084A136F0BB1506F92
:103390009847230404D5054A936F0BB1D06F984723
:1033A000BDE81040FFF716BE003C0140E02D0020B4
:1033B00008B5FFF75DFEBDE80840FFF70BBE000053
:1033C000062108B50846FFF71DFB06210720FFF779
:1033D00019FB06210820FFF715FB06210920FFF73E
:1033E00011FB06210A20FFF70DFB06211720FFF72E
:1033F00009FB06212820FFF705FBBDE8084007214F
:103400001C20FFF7FFBA000008B5FFF745FE00F0EB
:103410000BF8FDF78DFEFDF765FDFFF7A5FDBDE897
:103420000840FFF7CFBC00000023054A19460133CE
:10343000102BC2E9001102F10802F8D1704700BF59
:10344000E02D0020034611F8012B03F8012B002A80
:10345000F9D1704753544D3332463F3F3F005354E8
:103460004D3332463430780053544D333246343283
:10347000780053544D3332463434365858000000E7
:10348000012033000010410001105A0003105900C0
:10349000071031000000000054340008130400003D
:1034A0005E3400081904000068340008210400009C
:1034B0007234000800000000610E00084D0E000884
:1034C000890E0008750E0008810E00086D0E0008B8
:1034D000590E0008450E0008950E00080000000077
:1034E000010000000000000063300000E834000824
:1034F000F0230020002600204172647550696C6F33
:10350000740025424F415244252D424C002553451D
:103510005249414C2500000002000000000000005C
:103520007D100008E910000840004000A02A00209B
:10353000B02A00200200000000000000030000008C
:10354000000000002D110008000000001000000025
:10355000C02A002000000000010000000000000060
:10356000682D002001010200E11B0008F11A00088B
:103570008D1B0008711B0008430000008035000807
:1035800009024300020100C03209040000010202E6
:103590000100052400100105240100010424020299
:1035A0000524060001070582030800FF0904010045
:1035B000020A000000070501024000000705810221
:1035C0004000000012000000CC350008120110017C
:1035D00002000040091241570002010203010000ED
:1035E0000403090425424F41524425005442535FCD
:1035F0004C554349445F50524F00303132333435DB
:103600003637383941424344454600000040000007
:1036100000400000004000000040000000000100E9
:103620000000020000000200000002000000020092
:103630000000020000000200000002000000000084
:103640007112000829150008D51500084000400037
:10365000C82D0020C82D002001000000D82D00201A
:103660008000000040010000030000006D61696EF1
:103670000069646C650000000001806A00000000C1
:10368000AAAAAAAA00010064FFFF0000000000002F
:1036900000A00A000000000100000000AAAAAAAAD7
:1036A00000000001FFFF000000000000000000001B
:1036B0000000001000000000AAAAAAAA0000000052
:1036C000FFBF00000000000000000000000000003C
:1036D00000000000AAAAAAAA00000000FFFF000044
:1036E00000000000000000000000000000000000DA
:1036F000AAAAAAAA00000000FFFF00000000000024
:10370000000000000000000000000000AAAAAAAA11
:1037100000000000FFFF00000000000000000000AB
:103720000000000000000000AAAAAAAA00000000F1
:10373000FFFF00000000000000000000000000008B
:10374000000000000A00000000000000030000006C
:103750000000000000000000000000000000000069
:103760000000000000000000000000000000000059
:1037700000000000000000008314000000000000B2
:1037800000400F0000000000FF009600000000084D
:10379000009600000000080004000000E03500086A
:1037A0000000000000000000000000000000000019
:1037B0000000000000000000FFFFFFFFFFFFFFFF11
:1037C000FFFFFFFFFFFFFFFFFFFFFFFFFFFFFFFF09
:1037D000FFFFFFFFFFFFFFFFFFFFFFFFFFFFFFFFF9
:1037E000FFFFFFFFFFFFFFFFFFFFFFFFFFFFFFFFE9
:1037F000FFFFFFFFFFFFFFFFFFFFFFFFFFFFFFFFD9
:10C000000006002099D200085DA20608B9A1060822
:10C0100025A20608B9A10608F1A106089BD20008CE
:10C020009BD200089BD200089BD2000835CA0808A2
:10C030009BD200089BD200089BD200089BD200082C
:10C040009BD200089BD200089BD200089BD200081C
:10C050009BD200089BD2000851DC080879DC080854
:10C06000A1DC0808C9DC0808F1DC080849890808CF
:10C07000718908089D890808C9890808F589080890
:10C080001D8A0808498A0808CD8808089BD200083C
:10C090009BD200089BD200089BD2000819DD08083B
:10C0A00065DE080869DE08087DDE080881DE08080C
:10C0B0009BD2000885DE080899DE0808D58F08089D
:10C0C0007D9108089BD200089BD200089BD20008F3
:10C0D0009BD20008EDDD080801DE080815DE08081F
:10C0E0007DDD08089BD200089BD200089BD2000887
:10C0F0009BD200089BD200089BD20008758A0808D2
:10C100009BD200089BD20008ADDE08089BD2000835
:10C1100029DE08083DDE08089BD200089BD20008F3
:10C12000A18A0808C98A0808F58A0808218B080826
:10C130004D8B08089BD200089BD200089BD20008B8
:10C140009BD200089BD200089BD2000861D108084E
:10C15000758B0808A18B0808CD8B080851DE0808EC
:10C160009BD200089BD200089BD200089BD20008FB
:10C170009BD200089BD200089BD200089BD20008EB
:10C180009BD200089BD200089BD200089BD20008DB
:10C190009BD200089BD200089BD200089BD20008CB
:10C1A0009BD200089BD200089BD200089BD20008BB
:10C1B0009BD200089BD200089BD200089BD20008AB
:10C1C0009BD200089BD200089BD200089BD200089B
:10C1D0009BD200089BD200089BD200089BD200088B
:10C1E000B1E7000809F8000879530108C5B802084A
:10C1F000956704081D820408A1CF040865D70408C8
:10C200009DDA0408153F0508995B0508E1E4050877
:10C21000C9F90508159B0608917B0708E5AC0708D6
:10C2200079FA07085121080811370808D16408086D
:10C23000996A0808000000000000000000000000EB
:10C2400081F0004102E000BF83F0004330B54FEAC7
:10C2500041044FEA430594EA050F08BF90EA020F34
:10C260001FBF54EA000C55EA020C7FEA645C7FEAC7
:10C27000655C00F0E2804FEA5454D4EB5555B8BFEA
:10C280006D420CDD2C4480EA020281EA030382EA5B
:10C29000000083EA010180EA020281EA0303362DED
:10C2A00088BF30BD11F0004F4FEA01314FF4801CC0
:10C2B0004CEA113102D0404261EB410113F0004FD2
:10C2C0004FEA03334CEA133302D0524263EB430389
:10C2D00094EA050F00F0A780A4F10104D5F1200E27
:10C2E0000DDB02FA0EFC22FA05F2801841F1000182
:10C2F00003FA0EF2801843FA05F359410EE0A5F156
:10C3000020050EF1200E012A03FA0EFC28BF4CF086
:10C31000020C43FA05F3C01851EBE37101F000453C
:10C3200007D54FF0000EDCF1000C7EEB00006EEB49
:10C330000101B1F5801F1BD3B1F5001F0CD34908D3
:10C340005FEA30004FEA3C0C04F101044FEA44522A
:10C3500012F5800F80F09A80BCF1004F08BF5FEAB1
:10C36000500C50F1000041EB045141EA050130BD91
:10C370005FEA4C0C404141EB0101013C28BFB1F5A3
:10C38000801FE9D291F0000F04BF01460020B1FAEE
:10C3900081F308BF2033A3F10B03B3F120020CDAC1
:10C3A0000C3208DD02F1140CC2F10C0201FA0CF09F
:10C3B00021FA02F10CE002F11402D8BFC2F1200C04
:10C3C00001FA02F120FA0CFCDCBF41EA0C019040BA
:10C3D000E41AA2BF01EB0451294330BD6FEA040403
:10C3E0001F3C1CDA0C340EDC04F11404C4F12002EE
:10C3F00020FA04F001FA02F340EA030021FA04F300
:10C4000045EA030130BDC4F10C04C4F1200220FA56
:10C4100002F001FA04F340EA0300294630BD21FA94
:10C4200004F0294630BD94F0000F83F4801306BF5A
:10C4300081F480110134013D4EE77FEA645C18BF4E
:10C440007FEA655C29D094EA050F08BF90EA020FE5
:10C4500005D054EA000C04BF1946104630BD91EADD
:10C46000030F1EBF0021002030BD5FEA545C05D1E0
:10C470004000494128BF41F0004130BD14F580041F
:10C480003CBF01F5801130BD01F0004545F0FE4193
:10C4900041F470014FF0000030BD7FEA645C1ABFC8
:10C4A000194610467FEA655C1CBF0B46024650EAFF
:10C4B000013406BF52EA033591EA030F41F400212B
:10C4C00030BD00BF90F0000F04BF0021704730B5B1
:10C4D0004FF4806404F132044FF000054FF0000186
:10C4E00050E700BF90F0000F04BF0021704730B547
:10C4F0004FF4806404F1320410F0004548BF40421C
:10C500004FF000013EE700BF42004FEAE2014FEA70
:10C5100031014FEA02701FBF12F07F4393F07F4F4B
:10C5200081F06051704732F07F4208BF704793F04E
:10C530007F4F04BF41F40021704730B54FF4607461
:10C5400001F0004521F000411CE700BF50EA010264
:10C5500008BF704730B54FF000050AE050EA01020D
:10C5600008BF704730B511F0004502D5404261EB7D
:10C5700041014FF4806404F132045FEA915C3FF4BE
:10C58000D8AE4FF003025FEADC0C18BF03325FEA5B
:10C59000DC0C18BF033202EBDC02C2F1200300FA0C
:10C5A00003FC20FA02F001FA03FE40EA0E0021FA31
:10C5B00002F11444BDE600BF70B54FF0FF0C4CF41F
:10C5C000E06C1CEA11541DBF1CEA135594EA0C0FD1
:10C5D00095EA0C0F00F0DEF82C4481EA030621EA0C
:10C5E0004C5123EA4C5350EA013518BF52EA033547
:10C5F00041F4801143F4801338D0A0FB02CE4FF0F9
:10C600000005E1FB02E506F00042E0FB03E54FF028
:10C610000006E1FB03569CF0000F18BF4EF0010E20
:10C62000A4F1FF04B6F5007F64F5407404D25FEA1C
:10C630004E0E6D4146EB060642EAC62141EA5551CF
:10C640004FEAC52040EA5E504FEACE2EB4F1FD0C11
:10C6500088BFBCF5E06F1ED8BEF1004F08BF5FEA8F
:10C66000500E50F1000041EB045170BD06F0004641
:10C6700046EA010140EA020081EA0301B4EB5C04EE
:10C68000C2BFD4EB0C0541EA045170BD41F48011E6
:10C690004FF0000E013C00F3AB8014F1360FDEBF0B
:10C6A000002001F0004170BDC4F10004203C35DAE7
:10C6B0000C341BDC04F11404C4F1200500FA05F36A
:10C6C00020FA04F001FA05F240EA020001F000420B
:10C6D00021F0004110EBD37021FA04F642EB060181
:10C6E0005EEA430E08BF20EAD37070BDC4F10C04AB
:10C6F000C4F1200500FA04F320FA05F001FA04F26F
:10C7000040EA020001F0004110EBD37041F100015A
:10C710005EEA430E08BF20EAD37070BDC4F1200565
:10C7200000FA05F24EEA020E20FA04F301FA05F2CD
:10C7300043EA020321FA04F001F0004121FA04F275
:10C7400020EA020000EBD3705EEA430E08BF20EA45
:10C75000D37070BD94F0000F0FD101F0004640007F
:10C7600041EB010111F4801F08BF013CF7D041EA01
:10C77000060195F0000F18BF704703F00046520005
:10C7800043EB030313F4801F08BF013DF7D043EAD6
:10C790000603704794EA0C0F0CEA135518BF95EA8C
:10C7A0000C0F0CD050EA410618BF52EA4306D1D113
:10C7B00081EA030101F000414FF0000070BD50EA32
:10C7C000410606BF1046194652EA430619D094EABC
:10C7D0000C0F02D150EA013613D195EA0C0F05D1A6
:10C7E00052EA03361CBF104619460AD181EA0301FA
:10C7F00001F0004141F0FE4141F470014FF00000B2
:10C8000070BD41F0FE4141F4780170BD70B54FF04C
:10C81000FF0C4CF4E06C1CEA11541DBF1CEA1355CC
:10C8200094EA0C0F95EA0C0F00F0A7F8A4EB0504AE
:10C8300081EA030E52EA03354FEA013100F08880A5
:10C840004FEA03334FF0805545EA131343EA12636E
:10C850004FEA022245EA111545EA10654FEA002623
:10C860000EF000419D4208BF964244F1FD0404F5DC
:10C87000407402D25B084FEA3202B61A65EB030538
:10C880005B084FEA32024FF480104FF4002CB6EBF5
:10C89000020E75EB030E22BFB61A754640EA0C0075
:10C8A0005B084FEA3202B6EB020E75EB030E22BFB5
:10C8B000B61A754640EA5C005B084FEA3202B6EBF6
:10C8C000020E75EB030E22BFB61A754640EA9C00B5
:10C8D0005B084FEA3202B6EB020E75EB030E22BF85
:10C8E000B61A754640EADC0055EA060E18D04FEA43
:10C8F000051545EA16754FEA06164FEAC30343EAE3
:10C9000052734FEAC2025FEA1C1CC0D111F4801FAF
:10C910000BD141EA00014FF000004FF0004CB6E7A8
:10C9200011F4801F04BF01430020B4F1FD0C88BF47
:10C93000BCF5E06F3FF6AFAEB5EB030C04BFB6EB52
:10C94000020C5FEA500C50F1000041EB045170BD45
:10C950000EF0004E4EEA113114EB5C04C2BFD4EB72
:10C960000C0541EA045170BD41F480114FF0000EF6
:10C97000013C90E645EA060E8DE60CEA135594EA72
:10C980000C0F08BF95EA0C0F3FF43BAF94EA0C0F75
:10C990000AD150EA01347FF434AF95EA0C0F7FF4EA
:10C9A00025AF104619462CE795EA0C0F06D152EA3E
:10C9B00003353FF4FDAE1046194622E750EA410622
:10C9C00018BF52EA43067FF4C5AE50EA41047FF433
:10C9D0000DAF52EA43057FF4EBAE12E74FF0FF3C98
:10C9E00006E000BF4FF0010C02E000BF4FF0010C69
:10C9F0004DF804CD4FEA410C7FEA6C5C4FEA430CE2
:10CA000018BF7FEA6C5C1BD001B050EA410C0CBF30
:10CA100052EA430C91EA030F02BF90EA020F002092
:10CA2000704710F1000F91EA030F58BF994208BFF9
:10CA300090422CBFD8176FEAE37040F001007047B6
:10CA40004FEA410C7FEA6C5C02D150EA013C07D10D
:10CA50004FEA430C7FEA6C5CD6D152EA033CD3D058
:10CA60005DF8040B704700BF8446104662468C4652
:10CA70001946634600E000BF01B5FFF7B7FF002885
:10CA800048BF10F1000F01BD4DF808EDFFF7F4FFAE
:10CA90000CBF012000205DF808FB00BF4DF808ED39
:10CAA000FFF7EAFF34BF012000205DF808FB00BF5C
:10CAB0004DF808EDFFF7E0FF94BF012000205DF87E
:10CAC00008FB00BF4DF808EDFFF7CEFF94BF012033
:10CAD00000205DF808FB00BF4DF808EDFFF7C4FF2C
:10CAE00034BF012000205DF808FB00BF4FEA410C75
:10CAF0007FEA6C5C02D150EA013C0AD14FEA430C58
:10CB00007FEA6C5C02D152EA033C02D14FF0000094
:10CB100070474FF0010070474FEA410212F50012D2
:10CB200015D211D56FF47873B3EB625212D94FEA74
:10CB3000C12343F0004343EA505311F0004F23FA5E
:10CB400002F018BF404270474FF00000704750EAB3
:10CB5000013005D111F0004008BF6FF00040704770
:10CB60004FF00000704700BF4A0011D212F50012CA
:10CB700011D20DD56FF47873B3EB62520ED44FEA35
:10CB8000C12343F0004343EA505323FA02F07047B5
:10CB90004FF00000704750EA013002D14FF0FF30F3
:10CBA00070474FF0000070474FEA4102B2F1E04396
:10CBB00024BFB3F5001CDCF1FE5C0DD901F0004C84
:10CBC0004FEAC0024CEA5070B2F1004F40EB8300D4
:10CBD00008BF20F00100704711F0804F21D113F100
:10CBE0003872BCBF01F00040704741F480114FEA39
:10CBF0005252C2F11802C2F1200C10FA0CF320FAC2
:10CC000002F018BF40F001004FEAC1234FEAD323DE
:10CC100003FA0CFC40EA0C0023FA02F34FEA430348
:10CC2000CCE77FEA625307D150EA01331EBF4FF0D1
:10CC3000FE4040F44000704701F0004040F0FE40EC
:10CC400040F40000704700BF80F0004002E000BFE9
:10CC500081F0004142001FBF5FEA410392EA030FE7
:10CC60007FEA226C7FEA236C6AD04FEA1262D2EB31
:10CC70001363C1BFD218414048404140B8BF5B4236
:10CC8000192B88BF704710F0004F40F4000020F0CF
:10CC90007F4018BF404211F0004F41F4000121F0E5
:10CCA0007F4118BF494292EA030F3FD0A2F101022F
:10CCB00041FA03FC10EB0C00C3F1200301FA03F16D
:10CCC00000F0004302D5494260EB4000B0F5000F90
:10CCD00013D3B0F1807F06D340084FEA310102F14F
:10CCE0000102FE2A51D2B1F1004F40EBC25008BF01
:10CCF00020F0010040EA03007047490040EB0000CB
:10CD0000013A28BFB0F5000FEDD2B0FA80FCACF1CB
:10CD1000080CB2EB0C0200FA0CF0AABF00EBC250F8
:10CD200052421843BCBFD0401843704792F0000FE6
:10CD300081F4000106BF80F400000132013BB5E739
:10CD40004FEA41037FEA226C18BF7FEA236C21D0AF
:10CD500092EA030F04D092F0000F08BF0846704714
:10CD600090EA010F1CBF0020704712F07F4F04D1E2
:10CD7000400028BF40F00040704712F100723CBFF5
:10CD800000F50000704700F0004343F0FE4040F41F
:10CD9000000070477FEA226216BF08467FEA2363DD
:10CDA0000146420206BF5FEA412390EA010F40F4C8
:10CDB000800070474FF0000304E000BF10F0004314
:10CDC00048BF40425FEA000C08BF704743F09643FB
:10CDD00001464FF000001CE050EA010208BF704716
:10CDE0004FF000030AE000BF50EA010208BF70479D
:10CDF00011F0004302D5404261EB41015FEA010CB2
:10CE000002BF84460146002043F0B64308BFA3F1A9
:10CE10008053A3F50003BCFA8CF2083AA3EBC2538B
:10CE200010DB01FA02FC634400FA02FCC2F12002AA
:10CE3000BCF1004F20FA02F243EB020008BF20F0E1
:10CE40000100704702F1200201FA02FCC2F1200247
:10CE500050EA4C0021FA02F243EB020008BF20EA3C
:10CE6000DC7070477BB972B90029BEBF00204FF05B
:10CE7000004106E008BF00281CBF6FF000414FF0E2
:10CE8000FF3000F007BAADF1080C6DE904CE0029BF
:10CE900009DB002B1ADB00F095F8DDF804E0DDE992
:10CEA000022304B07047404261EB4101002B1BDBC1
:10CEB00000F088F8DDF804E0DDE9022304B0404228
:10CEC00061EB4101524263EB43037047524263EB13
:10CED000430300F077F8DDF804E0DDE9022304B055
:10CEE000404261EB41017047524263EB430300F063
:10CEF00069F8DDF804E0DDE9022304B0524263EB97
:10CF00004303704753B94AB9002908BF00281CBF22
:10CF10004FF0FF314FF0FF3000F0BCB9ADF1080C1D
:10CF20006DE904CE00F04EF8DDF804E0DDE90223FF
:10CF300004B07047430803F05533C01A830803F068
:10CF4000333300F03330184400EB101000F00F3092
:10CF500000EB002000EB0040000E704707EE900A47
:10CF6000F5EEC07AF1EE10FA01D400F00BB8F1EE54
:10CF7000677A08B517EE900A00F004F8404261EBBA
:10CF8000410108BDD0B5FFF7BFFA0C4B00220646A1
:10CF90000F46FFF711FBFFF7E7FD0446FFF792FA94
:10CFA000074B0022FFF708FB02460B463046394686
:10CFB000FFF74AF9FFF7D8FD2146D0BD0000F03D4C
:10CFC0000000F0412DE9F047089D04468E46002BF5
:10CFD0004DD18A42944669D9B2FA82F252B101FA2D
:10CFE00002F3C2F1200120FA01F10CFA02FC41EA3D
:10CFF000030E94404FEA1C48210CBEFBF8F61FFAC2
:10D000008CF708FB16E341EA034306FB07F199425C
:10D010000AD91CEB030306F1FF3080F01F8199420F
:10D0200040F21C81023E63445B1AA4B2B3FBF8F0E9
:10D0300008FB103344EA034400FB07F7A7420AD970
:10D040001CEB040400F1FF3380F00A81A74240F298
:10D0500007816444023840EA0640E41B00261DB103
:10D06000D4400023C5E900433146BDE8F0878B4238
:10D0700009D9002D00F0EF800026C5E900013046F7
:10D080003146BDE8F087B3FA83F6002E4AD18B42D1
:10D0900002D3824200F2F980841A61EB030301207B
:10D0A0009E46002DE0D0C5E9004EDDE702B9FFDE67
:10D0B000B2FA82F2002A40F09280A1EB0C014FEA12
:10D0C0001C471FFA8CFE0126200CB1FBF7F307FB6F
:10D0D000131140EA01410EFB03F0884208D91CEB12
:10D0E000010103F1FF3802D2884200F2CB804346AF
:10D0F000091AA4B2B1FBF7F007FB101144EA01448E
:10D100000EFB00FEA64508D91CEB040400F1FF311C
:10D1100002D2A64500F2BB800846A4EB0E0440EA0A
:10D1200003409CE7C6F12007B34022FA07FC4CEA13
:10D13000030C20FA07F401FA06F31C43F9404FEA06
:10D140001C4900FA06F3B1FBF9F8200C1FFA8CFE1B
:10D1500009FB181140EA014108FB0EF0884202FA6F
:10D1600006F20BD91CEB010108F1FF3A80F0888030
:10D17000884240F28580A8F102086144091AA4B2ED
:10D18000B1FBF9F009FB101144EA014100FB0EFE6E
:10D190008E4508D91CEB010100F1FF346CD28E459D
:10D1A0006AD90238614440EA0840A0FB0294A1EB2E
:10D1B0000E01A142C846A64656D353D05DB1B3EB8B
:10D1C000080261EB0E0101FA07F722FA06F3F140BB
:10D1D0001F43C5E9007100263146BDE8F087C2F162
:10D1E0002003D8400CFA02FC21FA03F391400143DA
:10D1F0004FEA1C471FFA8CFEB3FBF7F007FB103613
:10D200000B0C43EA064300FB0EF69E4204FA02F4BE
:10D2100008D91CEB030300F1FF382FD29E422DD911
:10D22000023863449B1B89B2B3FBF7F607FB163346
:10D2300041EA034106FB0EF38B4208D91CEB0101C6
:10D2400006F1FF3816D28B4214D9023E6144C91A46
:10D2500046EA004638E72E46284605E70646E3E656
:10D260001846F8E64B45A9D2B9EB020864EB0C0E60
:10D270000138A3E74646EAE7204694E74046D1E76F
:10D28000D0467BE7023B614432E7304609E764441D
:10D29000023842E7704700BF02E000F000F8FEE706
:10D2A00072B6374880F30888364880F309883648D4
:10D2B0003649086040F20000CCF200004EF63471AE
:10D2C000CEF200010860BFF34F8FBFF36F8F40F2C3
:10D2D0000000C0F2F0004EF68851CEF20001086066
:10D2E000BFF34F8FBFF36F8F4FF00000E1EE100AD6
:10D2F0004EF63C71CEF200010860062080F31488DF
:10D30000BFF36F8F7FF0F4FB80F03EFB4FF05530A2
:10D310001F491B4A91423CBF41F8040BFAE71D49E3
:10D32000184A91423CBF41F8040BFAE71A491B4ADC
:10D330001B4B9A423EBF51F8040B42F8040BF8E72E
:10D3400000201849184A91423CBF41F8040BFAE703
:10D350007FF0D2FB80F06CFB144C154DAC4203DA2D
:10D3600054F8041B8847F9E701F012FA114C124DEA
:10D37000AC4203DA54F8041B8847F9E77FF0BABBE4
:10D38000000600200022002000C0000808ED00E098
:10D39000000000200006002030100B0800220020B2
:10D3A0008025002080250020802C0120E0C100087D
:10D3B00034C2000834C2000834C200082DE9F04F1E
:10D3C0002DED108AC1F80CD0C3689D46BDEC108AC3
:10D3D000BDE8F08F002383F311882846A047002082
:10D3E0007EF07AFBFEE77EF0E7F900DFFEE7000063
:10D3F00001F0FF01102A2BDB10F0070F08D010F806
:10D40000013B013A8B422DD010F0070F42B3F6D109
:10D41000F0B441EA012141EA014122F007047FF022
:10D4200000070023F0E80256083C85EA010586EA79
:10D43000010685FA47F5A3FA87F586FA47F6A5FAB5
:10D4400087F68EB9EED1F0BC01F0FF0102F00702C1
:10D4500032B110F8013B013A83EA010313B1F8D16C
:10D460000020704701387047002D06BF354603384D
:10D47000073815F0010F07D1013015F4807F02BF86
:10D48000013015F4C03F0130F0BC0138704700BFD7
:10D4900010F8012B11F8013B012A28BF9A42F7D05E
:10D4A000D01A7047034613F8012B002AFBD1181A33
:10D4B0000138704738B50022002304460D46FFF7B7
:10D4C000EDFA28B920462946BDE8384000F00AB8F0
:10D4D000204605F1004100F005F8404261EB4101B2
:10D4E00038BD00BFD0B50C4B002206460F46FFF7F3
:10D4F00063F8FFF739FB0446FEF7E4FF074B002211
:10D50000FFF75AF802460B4630463946FEF79CFEB6
:10D51000FFF72AFB2146D0BD0000F03D0000F0419E
:10D5200000207047704700007047000070470000FF
:10D53000002070470020704700207047012070478E
:10D54000002070477047000000207047002070479F
:10D5500070470000704700000020704700207047AF
:10D5600070B5154ED6F8A00503681B6898470428C7
:10D570001ADC01281DDC002814BF012441240F4BB4
:10D580001D68E86A0368DB69984701280AD0D6F865
:10D59000A0250B4B9A4205D0EB6A93F89C300BB157
:10D5A00044F08004204670BD0A2814BF01241924C9
:10D5B000E5E71924E3E700BF885500208425002013
:10D5C000305B0020044BD3F8A00503F5B562904210
:10D5D00014BF04200220704788550020014B93F8A7
:10D5E00050047047884500207047000038B5C57862
:10D5F0000B461C2D044628BF1C251C220021184662
:10D6000083F0F8F92A4604F10C01BDE8384083F0B4
:10D61000A7B9000038B5C5780B46102D044628BFC1
:10D62000102510220021184683F0E4F92A4604F15F
:10D630000C01BDE8384083F093B9000008B542F012
:10D6400061F930B9034A92F8343643F0040382F8A2
:10D65000343608BD8855002038B591ED000AF7EE44
:10D66000000A0D4619F084F820B10B4801F042FF82
:10D67000002038BDD5ED007A9FED087AF0EEE77A0C
:10D68000F4EEC77AF1EE10FA03D5034801F044FF37
:10D69000EEE70320EDE700BF8825002000000034FE
:10D6A00010B5044607F076FE204610BD13B58B8BEF
:10D6B000B72B0C4607D0B3F5967F21D002B0BDE85A
:10D6C000104045F099BF124912481E2201F04CFF4C
:10D6D000D4ED017A94ED007A0D48FCEEE77ABCEEC9
:10D6E000C77A17EE903A8DED017A9DF804109AB240
:10D6F00001F0D0FB002814BF0020042002B010BDB0
:10D7000004480549022201F02FFF0020F6E700BF80
:10D71000585B0020882500202C5B002000B5244B9E
:10D72000DFED246A007C03F5C56292ED007A03F216
:10D730002C62D2ED007AA3F580528BB092F972245C
:10D74000002A03F21C6218BFB0EE677A11680491D8
:10D7500003F21462D2ED007A8DED057AFDEEE77AE0
:10D7600003F5C36317EE902AD3ED007AF4EEE67A60
:10D77000F1EE10FA58BFF0EE667AFCEEE77A00237D
:10D7800003930693079317EE903A12B2ADF8202058
:10D79000ADF82220ADF82430B7221A23CDE90032AB
:10D7A0003E2103AA3FF0C0FA0BB05DF804FB00BFB6
:10D7B0008855002000FF7F4770B5164C94F83A2634
:10D7C0008AB022B90AB0BDE8704040F061BD057C66
:10D7D0005CF07AFDD4F89865D4F89C15D4F89435AB
:10D7E000A4F50054CDE90513B4F8E825ADF82620DA
:10D7F0000023CDE90733ADF8243068221C23CDE99E
:10D800000306CDE90032212103AA28463FF08CFA15
:10D810000AB070BD88550020F0B5454CB4F894347A
:10D82000DE078DB0054643D504F5A76304F5AB626A
:10D83000D3F800C01268CDF8252004F24C5304F24E
:10D84000345E1F68DEF800E0CDF80CE004F5A86354
:10D8500003AA1E68CDF810C004F244530696186857
:10D86000079004F5A96362201968089104F25453E3
:10D8700002211B68CDF829302123CDE900308DF835
:10D8800024101923C221287C05973FF04DFA287CEB
:10D890003FF0E0F90646287C40F0E0F800F1210373
:10D8A0009E4205D2287C0DB0BDE8F0403EF04EBC53
:10D8B000B4F89434990738D504F5C4631F68049705
:10D8C00004F234631E68059604F5C5631868069073
:10D8D00004F22C63287C1968079104F5C663C22101
:10D8E0001A680892032204F23C638DF82420114A3E
:10D8F0001B681268CDF8252004F21C64CDF829308D
:10D900006222212324680394CDE90032192303AA5B
:10D910003FF00AFA287C3FF09DF90446287C40F04D
:10D920009DF800F121039C42BCD30DB0F0BD00BFB7
:10D9300088450020C84B002005207047024BD3F8D3
:10D94000A00503681B6818478855002030B5CD78BE
:10D950008BB0272D28BF27250C462722002168469B
:10D9600083F048F82A4604F10C01684682F0F8FF7B
:10D970001C4BD3F8A01503F5B662914230D1DDED12
:10D98000057A9FED197AF0EEE77AF4EEC77AF1EEB8
:10D9900010FA25D59DF8262002F0410141291FD11A
:10D9A00011061DD402F01801182919D003F2B45140
:10D9B0000198086003F5B7610298086082F00402DC
:10D9C00003F2BC5103980860C2F3800283F8C425B7
:10D9D00003F5B86103F5B9630498079A08601A6003
:10D9E0000BB030BD885500200000003430B5194D13
:10D9F00095F8393685B00C464BBBCA788DF80C309B
:10DA0000092A28BF09220C3101A8CDE9013382F08F
:10DA1000A7FF9DF808305A1F012A18D903F0F70311
:10DA2000122B14D0A5F58053B3F9522412B9E27920
:10DA3000A3F85224227AE179074800F0B1F9227A5A
:10DA4000E179054800F0E4F9012385F8393605B09D
:10DA500030BD00BF885500207C530020F0B51B4B23
:10DA6000B3F9523489B005460E4614463BB1D77916
:10DA7000BB4204D009B0BDE8F04044F0B3B8A27A8C
:10DA8000637A43EA0223E27A43EA02431D2B13D06E
:10DA9000212B08D01BB921462846FFF7A7FF2246B5
:10DAA00031462846E6E701A92046FFF79FFD0848D2
:10DAB00001A902F005F8F2E701A92046FFF7AAFD47
:10DAC000034801A902F05AF8E9E700BF88450020A1
:10DAD0008825002013B5CA78072A4FF000030446B2
:10DAE00028BF07220C3168460093CDF8033082F03E
:10DAF00037FFBDF900304BB901231C21204684F8C3
:10DB00000F3302B0BDE8104045F02EBD02B010BD8D
:10DB100030B5CD7889B01E2D28BF1E250C461E229B
:10DB20000021684682F066FF2A4604F10C0168462F
:10DB300082F016FF0248694602F070F809B030BD65
:10DB40008825002000B589B0084601A9FFF74EFDE1
:10DB5000034801A901F0B4FF09B05DF804FB00BF60
:10DB6000882500201FB508466946FFF753FD034886
:10DB7000694602F003F805B05DF804FB8825002033
:10DB80002DE9F041CC7894B0262C28BF2624884675
:10DB90002622002107460AA882F02CFF02AD224669
:10DBA00008F10C010AA882F0DBFE284607F04EF9C6
:10DBB0009DF84A30022B06AC03D0032B44D0002B37
:10DBC00066D1DFED357ADDED106A9FED346A9DEDAB
:10DBD0000F7A66EEA76ADDED0E7A27EE067A67EE1B
:10DBE000867A0023FDEEE66ABDEEC77AFDEEE77A9F
:10DBF00017EE102A17EE901A0093204616EE903A70
:10DC000007F044F994E80F0085E80F0097F80F3308
:10DC100063BB012698F8083098F807208DF8193072
:10DC200000238DF818208DF81B3099220423CDE9AC
:10DC30000032387C8DF81A60032322462F213FF0F2
:10DC400073F814B0BDE8F081DFED137ADDED106AF2
:10DC50009FED126A9DED0F7A66EEA76ADDED0E7AF2
:10DC600027EE067A67EE867A0123BBE7BDF84460AB
:10DC700086B90B483246294601F014FC0028C8D06A
:10DC8000084A0621384641F0D1FA87F80F63C1E708
:10DC90000226BFE70026BDE70000C8428096184B69
:10DCA000882500208C4D090838B58A7A4B7A43EADA
:10DCB0000223CA7A43EA0243272B05460C460CD8B6
:10DCC0001C2B10D91D3B0A2B0DD8DFE803F01E0CCE
:10DCD0000C0C1B0C0C0C0C121500452B0FD0522BEE
:10DCE00001D1FFF733FE21462846BDE8384044F015
:10DCF0005DBEFFF7EFFEF6E7FFF742FFF3E7FFF742
:10DD000007FFF0E7FFF71EFFEDE7FFF72BFFEAE75E
:10DD100000207047C82070470120704700207047DE
:10DD2000002070470120704790F89C308B4286BFDE
:10DD3000283150F8210000207047000090F89C30F6
:10DD40008B4286BF283150F8210000207047000028
:10DD5000014B93F84E04704788450020C36A43F492
:10DD6000E053C362036B43F4E0530363436B43F438
:10DD7000E05343637047000013B54FF44470CDE99E
:10DD8000002107F0FFFA044628B1DDE9002145F043
:10DD90002FF8024B2360204602B010BD284F09081F
:10DDA0002DE9F04FDFF8649085B006460F469046A7
:10DDB00000254FF4837A96F89C30ECB2A34222D926
:10DDC00020463EF047FF834620463FF047FE031DB6
:10DDD0009B4514D399F97334ADF808309422062387
:10DDE000CDE90032422102AA20468DF80A708DF852
:10DDF0000B80ADF80CA03EF097FF0135DBE7204625
:10DE00003EF0A4F9F9E705B0BDE8F08F88450020A1
:10DE10002DE9F04FDFF8649085B006460F46904636
:10DE2000002540F2011A96F89C30ECB2A34222D9A8
:10DE300020463EF00FFF834620463FF00FFE031DB5
:10DE40009B4514D399F97334ADF808309422062316
:10DE5000CDE90032422102AA20468DF80A708DF8E1
:10DE60000B80ADF80CA03EF05FFF0135DBE72046EC
:10DE70003EF06CF9F9E705B0BDE8F08F8845002069
:10DE8000704700001FB500F5405303F21C6203F217
:10DE90001463002100F59F5012681B68019108303F
:10DEA00001A90292039302F027F803F025FC03F086
:10DEB000CFF905B05DF804FB70B586B006461322B5
:10DEC000002101A810EE105A10EE904A82F092FD47
:10DED000A3238DF8043095238DF805305CF0FCF910
:10DEE0001322CDF80700CDF80B1006F58F5001A9CD
:10DEF000CDF80F50CDF813403BF0B4F806B070BD2C
:10DF00002DE9F0418AB004468846174600212322B5
:10DF100001A8109D1E4682F06DFDA3238DF80430EC
:10DF200095238DF8053001238DF806305CF0D4F987
:10DF30002B68CDF81B306B68CDF80700CDF80B10BF
:10DF4000CDF81F302322AB68CDF80F8001A904F56E
:10DF50008F50CDF81370CDF81760CDF823303BF01B
:10DF600081F80AB0BDE8F0819720704710B500F540
:10DF700040530446D3F8A00503681B6898471A224B
:10DF8000C1B204F58F503BF02DFA04F59070BDE856
:10DF900010400FF04DBD000037B500F5115104469B
:10DFA00001220C3139F002FE012504F50A51104A14
:10DFB000009500230831DA2037F02EF90D4A00953C
:10DFC000002304F58F51FD2037F026F90A4B1A681B
:10DFD000D20705D4094A1D6004F598540C34146026
:10DFE0000648012103B0BDE8304037F067B900BFF3
:10DFF000C4C70A08540C0A0880250020002200200B
:10E0000000207047002070470069C0F3401070473F
:10E010000F299DBF302303FB0100503000207047C3
:10E0200000207047012070477047000000207047B3
:10E030000020704700207047002070470020704784
:10E040000020704700207047002070470020704774
:10E050000020704770470000036800221B681847C3
:10E060001020704700207047704700000320704761
:10E070000120704770470000012070470020704762
:10E080007047000000F512501C3070470048704780
:10E090006473090808B500F54050D0F8A00503687E
:10E0A0001B689847C0B208BD034808600F21117073
:10E0B0004FF0FF321A607047F48A09080020704759
:10E0C000002070477047000016F01AB93BF030B9D5
:10E0D00045F0B0BD43F0E6BE05F0CABC06F0A6BCF4
:10E0E00000F006BF00F000BF00F01EBF01F084BCCE
:10E0F00000F0ECBE00F0F2BE00F05CBF70B5224B49
:10E10000036000F500550446D5F8B00F1F4BC5F865
:10E11000F43D08B107F042F91D4B236095F8C43077
:10E1200043B9D5F8C0502DB1284614F06DFF2846EC
:10E1300007F030F904F59750103059F091FA04F5D2
:10E140009550143047F0DCFE04F6E46504F684666E
:10E15000B54204D0183D284614F0C6FBF8E70D4B35
:10E16000C4F8C83804F628203CF03AFF04F6FC1046
:10E170003CF036FF04F65C103CF032FF04F513600F
:10E180003CF02EFF204670BD288C090884240A0824
:10E19000B8050A0804D9090838B54D4B044640F8BB
:10E1A000043B48F0ABFF04F1100006F065FD04F1FC
:10E1B000680038F06DFF04F590700EF0F3FF04F581
:10E1C0008C6005F0C5FA04F2845007F0E9F804F613
:10E1D000C80015F0DBFE04F5666048F017FF04F593
:10E1E000736038F077FC04F58F503AF083FE04F545
:10E1F000945018304EF0FEFA04F59550143047F064
:10E2000067FE04F59750103059F016FA04F598504F
:10E210000C3039F049FA04F59B504AF019F904F52D
:10E22000805300252B4A83F8845304F59C5004F551
:10E230009C5304331430136034F0AAFB04F59F5050
:10E240002946083001F04EFF04F5D250103053F04B
:10E2500005FB04F5FA50143056F026FA04F5015087
:10E260002C3058F043FB04F50350103058F078FF81
:10E2700004F50450283001F095FD04F50A500830EB
:10E2800053F0E0FF04F50B501349203037F01CFD2C
:10E2900004F50B5038304EF051FD04F50E5034307B
:10E2A00059F0E2FC04F5005304F5105083F80C54C7
:10E2B0000A4D243059F0FAFD2B6813B108485BF081
:10E2C000D1FF2046074937F0FFFC2C60204638BDBF
:10E2D000B8050A08106700201CC20A08605E00200A
:10E2E000F4880908D0040A0810B59FED225A9FED62
:10E2F000224A9FED222ADFED221A9FED221A9FED7E
:10E30000220A86B00446F0EE453AB0EE453AF0EE09
:10E31000452AF0EE450AF7EE004A54308DED054AE5
:10E320008DED042ACDED031A8DED021A8DED015A03
:10E330008DED000A53F032F89DED015A9DED054A2E
:10E340009DED042ADDED031A9DED021A9DED000AF4
:10E35000F7EE004AF0EE453AB0EE453AF0EE452AC7
:10E36000F0EE450A04F59E7053F018F8204606B00A
:10E3700010BD00BF00000000CDCCCC3D00007A45B0
:10E380000AD7A33CCDCC4C3DCDCC4C3EF0B500F5EE
:10E390000055234BB5F84E241A7087B0044647F059
:10E3A000F5FB47F073F9204601F06CFC04F580534F
:10E3B00093F8642612F0010210D102A8019206F02F
:10E3C00045FD04F59F5002A9083002F057FF28B11F
:10E3D0002368019ADB6C02A920469847114E3368E6
:10E3E000DB6A93F89C7037B195F80E341BB95BF07B
:10E3F0006BFFC5F81004336885F80E74DB6A93F878
:10E400009C20094B5A7139F0B5F838F007FE04F535
:10E410001650083007B0BDE8F04053F00FB800BF09
:10E42000C5220020842500208D5D0020FFF7AEBFAF
:10E4300010B50821044601F0DFF918B117F04EFDC0
:10E4400015F06EFC0121204601F0D6F910B12046EE
:10E45000FFF718FD0421204601F0CEF918B104F5AC
:10E460008F503AF0BDF91021204601F0C5F928B1CE
:10E4700004F58F50BDE810403AF04CBA10BD0000D2
:10E48000FFF7D6BF102926D8DFE801F0090D1119D2
:10E490001525252525251D2525252525210000F5C2
:10E4A00056502C30704700F557501430704700F527
:10E4B00057500C30704700F556503030704700F51B
:10E4C00057501030704700F556502430704700F513
:10E4D00056502830704700207047000008B553F0B0
:10E4E000B5FF044B1B68DB6A93F89C10BDE808403D
:10E4F00053F088BF84250020FFF7F0BF2DE9FF41CE
:10E500000446FFF749FE884B236004F5115004F5DB
:10E5100000560C30FFF7E8FE002304F51950C6F84A
:10E520007036343045F09CFDDFF860827F4BC6F8D2
:10E53000743642F2C46542F6C417601945F01EFFF6
:10E5400044F805803035BD42F7D1601947F0F6F93F
:10E5500004F5375018303CF085FF04F5375024306F
:10E560003CF080FF04F537570023A6F8F03D343720
:10E570006F4BC6F8F43D07F114005BF001F804F5A9
:10E58000385504F53A582C3508F11008284614354A
:10E5900041F050FD4545F9D10723C6F8B43F0023AB
:10E5A000A6F8B83F4FF4CB7006F0F2FEC6F8B00FF5
:10E5B00004F53E503C3004F540555AF0E1FF284642
:10E5C0005AF0DEFF5B4B1A6802B91F605A4BC6F85F
:10E5D000F43D5A4B039300260294009604AB04F5D5
:10E5E000405013E90C0040211C3005F05BFE04F59F
:10E5F0005650103006F02AFC04F556532833C5F85F
:10E60000A0354F4BC5F8A4354E4BC5F8A8354E4B39
:10E61000C5F8AC354D4BC5F8B03505F2B4530027FD
:10E620004FF07E521A60DF609F605F60484BC5F814
:10E63000CC3504F55758474BC5F8D03508F11808C4
:10E64000454BC5F8D43508F1040006F0FFFB08F18E
:10E65000140006F0FBFB05F2046340481F605F6096
:10E660009F603F4B04F558521860383233464FF6DE
:10E67000FF774FF0140C9EB20CFB06010133097CAE
:10E680000029F8D1374B38491E800B6813B1374841
:10E690005BF0E8FD85F8393604F55850012385F81C
:10E6A0003A363C300A6059F0AFFC314BC5F83C3685
:10E6B000304BC5F89436304BC5F89C3604F55A50AB
:10E6C0002E4BC5F8A436C5F89046C5F89846C5F84F
:10E6D000A046383006F0BAFB04F55B50143006F063
:10E6E000B5FB04F55B50303006F0B0FB04F559562D
:10E6F000234BC5F80437A5F8087706F1CC0006F0DF
:10E70000A5FB4FF0FF333436C5F868371D4B1E4963
:10E710001E60304637F0D8FA2046A5F8B076A5F846
:10E72000CC7604B0BDE8F081288C0908D8880908A7
:10E7300084240A08A461002004500908F9E00008B4
:10E740009C8C090880890908E48C0908D08C090888
:10E75000F88C090894890908A88909081083090810
:10E76000285E0020265E0020E45D0020088909085C
:10E7700040890908BDE00008C1E00008C5E00008C4
:10E780000000FFFF605D00204CE309082C890908A8
:10E7900038B5054B1C6823680A461D68034B0146C3
:10E7A0002046A847002038BD842500208825002069
:10E7B00010B55BF0ABF9064C064B18602046FFF72E
:10E7C0009DFE2046044A0549BDE810407FF0E4BBA9
:10E7D00088250020842500201CC00020FDE00008C2
:10E7E00038B52DED028B0D46F0EE608AB0EE408A12
:10E7F000144602F081FF90ED937AD0ED957A67EEA2
:10E80000877A90ED927A67EEA87AE7EE087AC5EDFE
:10E81000007AD0ED920AD0ED937A90ED957A67EE7A
:10E82000A07A67EEA80AE7EE480ABDEC028BC4EDB9
:10E83000000A38BD30B52DED068B83B0F0EE409A5E
:10E84000B0EE60AA0D46044602F056FFD0ED7F7A86
:10E85000D0F80002B8EEE79A18F056F807EE900AE2
:10E86000F8EEE78A79EEC9AA3AEE688AFDEEEAAADE
:10E87000B0EE480A18F02AF8BDEEC00A5DB110EEFD
:10E88000103ADFED1D0A002BCCBF38EE608A38EE5F
:10E89000208ABDEEC80AF8EEC00A01AA6946B8EEA1
:10E8A000EA0A2046FFF79CFF144BDFED157A00992A
:10E8B00003F5C46269EEA79A116003F2246201991C
:10E8C000116029EE279AA3F6CC22C2ED009A2AEE17
:10E8D00027AAA3F6C82268EEA78A82ED009AA3F6BB
:10E8E000E412A3F51E6382ED00AAC3ED008A03B013
:10E8F000BDEC068B30BD00BF00A00C478855002042
:10E900000AD7233C38B52DED028B0D46B0EE408A78
:10E91000F0EE608A144602F0EFFED0ED937A9FEDA0
:10E92000147AF0EEE77AF4EEC77AF1EE10FA1DD41D
:10E93000D0ED957A90ED927A67EEE87AE8EE077A74
:10E94000C5ED007A90ED937AD0ED957A90ED926ACC
:10E95000C7EE876A0120C6EE077A67EEA80AE6EEE0
:10E96000880AC4ED000ABDEC028B38BD0020FAE72E
:10E970000000003430B52DED068B5F4CDFED5F8A73
:10E98000B4F98C345B4285B008EE103A054604F6C3
:10E99000D8503CF06BFDB8EEC88AB4F98C3490EDD9
:10E9A00000AA28EE288AF6EE009A98EE29AA04F624
:10E9B000D85008EE103A3CF059FDB8EEC88AB4F9C8
:10E9C000903490ED009A28EE288A04F6E45098EEF0
:10E9D000299A08EE103A3CF049FDB4F99234D0ED92
:10E9E000009A04F6E4500AEE903A3CF03FFDB8EE8F
:10E9F000C88AF8EEEAAAD8EE289A6A4602A990EDEB
:10EA0000008A8DED00AA9AEEA88A2846F0EE4A0AFE
:10EA1000B0EE690A8DED038A8DED019ACDED029A73
:10EA2000FFF770FF01AA03A9F0EE490AB0EE480A09
:10EA30002846FFF767FF02F05FFED0F8000217F0EC
:10EA400063FF04F5B05304F28444D4ED007A93EDEF
:10EA5000050A30EE270A08EE100A20EE280A17F001
:10EA600035FFB8EEC88A30EE480A17F02FFFDFED09
:10EA7000247A9DED007AB5EEC00AF1EE10FAACBF33
:10EA800070EE676AF0EE406AB4EEE67AB4BF70EEFC
:10EA9000277AF0EE407AF1EE10FA2ADD9DED016A58
:10EAA000B4EEE76AF1EE10FA23D5B5EEC00AF1EE46
:10EAB00010FA08DD77EE665A37EEC65AF4EEC55AFC
:10EAC000F1EE10FA13D4B5EEC00AF1EE10FA10D53B
:10EAD00037EE667A77EEC67AB4EEE77AF1EE10FAA0
:10EAE000CCBF0120002005B0BDEC068B30BD01205D
:10EAF000F9E70020F7E700BF884500200000C84282
:10EB000000A00C4770B5364C2DED028B04F2146258
:10EB1000A4F67C33D3ED007A92ED000ADFED318A62
:10EB200030EE270AA4F5805684B020EE280A054668
:10EB300017F0CCFEB6F9923401EE103AB6F99034E3
:10EB400004F21C6200EE903AA4F67833D3ED007A1A
:10EB5000B0EE408A92ED000AB8EEC11A30EE270AF4
:10EB6000F8EEE00A0C2017F005FF20EE280A2846F0
:10EB70008DED010AFFF7FEFE9DED010A0146F0EE64
:10EB8000480A2846FFF756FE9DED010A03AA02A98E
:10EB9000F0EE480A2846FFF723FEB6F98E34002B24
:10EBA0000FDD07EE903A04F5C362F8EEE77A92EDD6
:10EBB000007AB4EEE77AF1EE10FA02DA94F8D8357A
:10EBC0004BB99DED020A084800F018FB9DED030AC1
:10EBD000054800F0F5FB04B0BDEC028B70BD00BF32
:10EBE000885500200000C8428825002038B54C4CCC
:10EBF00094F83436054613F0010047D1A4F580524D
:10EC00009FED487AB2F9602407EE902AF8EEE77A91
:10EC100004F2146167EE877A91ED000A13F0100F89
:10EC2000BFEE007AF7EE006A08BFB0EE667AA7EE94
:10EC3000270AC3F30012DFED3C7A81ED000AB5EE3E
:10EC4000C00AF1EE10FA0AD51AB160F3041384F881
:10EC50003436B4EEE70AF1EE10FA06DC0BE0B4EE5F
:10EC6000E70AF1EE10FA06DD2AB994F8343643F0DB
:10EC7000100384F834369FED2C1ADFED2C0A2C207B
:10EC800017F078FE04F2146383ED000A94F834362A
:10EC90009A07C3F3400032D425499FED227AB1F997
:10ECA000622407EE902AB1F99024B1F9921400EE93
:10ECB000902A01EE101AF8EEE77A04F21C621907A6
:10ECC00067EE877AF8EEE00A92ED007AB8EEC11AA4
:10ECD0001AD577EE677AF4EEE07AF1EE10FAC2ED2B
:10ECE000007A03D560F3C30384F8343604F21C645D
:10ECF00094ED000A3C2017F03DFE84ED000A284602
:10ED0000BDE83840FFF7FEBE77EE877AF4EEC17AB1
:10ED1000F1EE10FAC2ED007AE8DD43F00803E3E714
:10ED2000885500200AD7A33C0000B443000000002F
:10ED3000884500200A20704701207047094B93F84E
:10ED4000D815024609B1FFF7DDBE93F8391629B987
:10ED5000A3F5805393F89834DB0702D51046FFF7EC
:10ED600045BF704788550020042070470120704738
:10ED700030B52DED028B8BB004465BF0A5FA07ABE6
:10ED8000054606AA05A9201D19F068FB274A9FED34
:10ED9000288A136841F28831EB1A8B421CD915601E
:10EDA00043F0E4FDDDED067A67EE887A054617EE5E
:10EDB000900AFDF7A9FBDDED077A67EE887ACDE9C9
:10EDC000020117EE900AFDF79FFB1A4ACDE90001F8
:10EDD000062128463CF09AFFDDED067ADDED070AB4
:10EDE0009FED150A60EE880A27EE888A60EE800A99
:10EDF000204628EE000A0021FFF71CFDDDED070A82
:10EE00009DED060A09AA08A92046FFF7E9FC9DED39
:10EE1000080A0A4800F0F2F99DED090A074800F0D7
:10EE2000CFFA0BB0BDEC028B30BD00BFF85C002008
:10EE3000E02E6542A88C09080000C8428825002001
:10EE40000020704701207047024B01461868026895
:10EE500012681047AC61002008B50020FFF7F4FFEE
:10EE6000C188472046F0F6FC472046F08FFB012082
:10EE7000FFF7EAFFC188482046F0ECFCBDE80840F7
:10EE8000482046F083BB00000220704701207047F5
:10EE9000FFF7ACBE08B50B46013BDBB2012B1146B8
:10EEA00011D85BB9472046F0D5FC472046F06EFBF1
:10EEB00046F098FD46F04AFA012008BD482046F089
:10EEC000C9FC4820F2E70020F7E7000008B545F04C
:10EED00021FABDE8084045F0FDB8000000F59F505C
:10EEE0000021083002F08EBB00F2845006F0E2BE32
:10EEF00010B5044606F0CEFF90F921308BB190F8A2
:10EF0000403373B194F9A8355BB1064B1B68DB6ADB
:10EF100093F89C302BB904F28450BDE8104006F001
:10EF2000E1BC10BD8425002070B5044600F590704A
:10EF30000FF0D6FC94F814341C4904EB0312D2F8F9
:10EF4000C4010A68824210D0B02202FB034294F846
:10EF5000585492F8F12145B9022A06D9144E086096
:10EF60003278012A02D9013A327070BDFDD104F520
:10EF70004055D5F898252AB9D5F89C2512B905230E
:10EF80003370F2E7B02202FB034303F5FE730FCBAD
:10EF900005F5B26585E80F00236804F55651DB6C72
:10EFA00000221031204698470023E9E7FC5C00204E
:10EFB0000C2200207047000037B5044646F0E6FDFD
:10EFC00046F064FB04F500554721002046F090FC14
:10EFD0004821012046F08CFCB5F88C1401EB81012E
:10EFE00001EB8101490089B2472046F0B9FAB5F931
:10EFF0009034B5F992140F4DC91A01EB810101EB60
:10F000008101490089B2482046F0AAFA46F0EAFC9C
:10F0100046F09CF904F5375001A9183001953CF0F1
:10F02000B7FA04F5375001A9243001953CF0B0FA45
:10F0300003B030BDCDCCCC3DF0B52DED028B00F54D
:10F04000005785B0B7F89024B7F892340446642589
:10F05000482012FB05F613FB05F546F071FA04F59E
:10F06000585304F512502030B0EE408ADFED230AE9
:10F0700093ED080A0190002152F04AFB07EE906AD6
:10F0800038EE000AF8EEE77A0198B4EEE70AF1EEFE
:10F0900010FA25D98DED020A07EE905A9DED027AFD
:10F0A000F8EEE77AF4EEC77AF1EE10FA03D8CDED78
:10F0B000027A52F021FA48209DED020A46F02CFA1D
:10F0C00097F8F13D04F53750243083B10C4B03938E
:10F0D00003AA02A93CF060FA05B0BDEC028BF0BDBA
:10F0E0000190CDED027A52F007FA0198D4E702A917
:10F0F0003CF0BEF9012387F8F13DEDE70AD7A33CC8
:10F100000AD7A33C00F5585300F5005293ED087A56
:10F1100000F5125002F58F63D3ED007A90ED006A8E
:10F1200067EE867AF0EEC76AF4EEE76AF1EE10FA5F
:10F1300004D59FED180A482046F0EEB9DFED167AA7
:10F14000B5EEC07AF1EE10FA20EE270A10DDB2F823
:10F150009034642113FB01F307EE903AF8EEE77A5E
:10F16000F4EEC07AF1EE10FA02D59FED0C0AE2E758
:10F17000B2F89234642213FB02F307EE903AF8EEF1
:10F18000E77AF4EEC07AF1EE10FA02DD9FED040AA0
:10F19000D1E77047000000000000C84200A00CC684
:10F1A00000A00C4610B5044600F5585304F5005471
:10F1B00000F51250DFED100A93ED080A002120300F
:10F1C00052F0A6FAB4F99204B4F990343221C21A7A
:10F1D0001B1A4A434B4301EE102A00EE903A80205E
:10F1E000B8EEC11AF8EEE00A17F0C4FBBDE8104013
:10F1F000482046F091B900BF0AD7A33C00F5005360
:10F2000093F97034012B03D0022B03D0FFF714BF06
:10F21000FFF778BFFFF7C6BFF0B52DED028B00F505
:10F2200000573223B7F88C54DFED310A00F516563B
:10F2300015FB03F5083600F5585393ED090A83B022
:10F2400000210446304652F063FA9FED2A1ADFEDA2
:10F250002A0ABF2017F08EFB4720B0EE408A46F006
:10F260006FF99FED241ADFED240A30EE080AC02062
:10F2700017F080FB6B4207EE903AF8EEE77AB4EEB7
:10F28000E70AF1EE10FA26D98DED000A07EE905A42
:10F290009DED007AF8EEE77AF4EEC77AF1EE10FA17
:10F2A00004D83046CDED007A52F026F947209DED86
:10F2B000000A46F031F997F8F03D04F53750183060
:10F2C0007BB10E4B019301AA69463CF065F903B08E
:10F2D000BDEC028BF0BD3046CDED007A52F00CF95A
:10F2E000D4E769463CF0C4F8012387F8F03DEEE727
:10F2F0000AD7A33C00A08C4600A08CC60AD7A33C2A
:10F3000000F55853D3ED097A9FED127A00F50050BD
:10F3100000F2744300F27C4067EE877A90ED006A59
:10F3200093ED007A27EE067AF0EEE76AF4EEC76A0C
:10F33000F1EE10FA04D59FED080A472046F0ECB82C
:10F34000F5EEC07AF1EE10FACCBF9FED040A9FED06
:10F35000040AF2E70AD7233C0000000000A08C4614
:10F3600000A08CC610B5044600F5585304F50054AF
:10F3700000F51650DFED110A93ED090A002108305F
:10F3800052F0C6F9B4F98C344FF6CE71322213FB29
:10F3900002F213FB01F301EE102A00EE903AF12085
:10F3A000B8EEC11AF8EEE00AB1EE400A17F0E2FA40
:10F3B000BDE81040472046F0AFB800BF0AD7A33CD5
:10F3C00000F5005393F97134012B03D0022B03D0C5
:10F3D000FFF722BFFFF794BFFFF7C4BFFEF7C6BD1C
:10F3E00070B500F5005088B090F999040C46D8B17A
:10F3F00005210E4846F088FC092106460B4846F0D8
:10F4000083FC01210390094846F07EFC04AD0021F5
:10F410000346039A00912846314605F037FD95E8EA
:10F420000F0084E80F00012008B070BD005D0020CF
:10F4300037B50C460022054611460F4846F07CFCC5
:10F4400062680D48012146F08FFCA2680A48052138
:10F4500046F08AFCE2680848092146F085FC05F57B
:10F46000125001240DF1070119308DF8074037F0D3
:10F470002BFA204603B030BD005D002037B503688D
:10F480000191DD6C04460FF069FA90F8F412019ACC
:10F49000B02303FB0101DC3120462B4603B0BDE85D
:10F4A000304018477FB5044604F59F566846083635
:10F4B0000D4605F0CBFC6946304601F023FF48B904
:10F4C00029462046FFF7B4FF064650B900263046CD
:10F4D00004B070BD2946304601F0BEFD0028EFD1D2
:10F4E000F4E795E80F0004F55654103484E80F0053
:10F4F000EDE7000010B5074B1B680446D86A0368A7
:10F5000001211B68984704F58F500121BDE8104088
:10F5100039F090BD8425002010B5074B1B680446C8
:10F52000D86A036800211B68984704F58F500021B2
:10F53000BDE8104039F07EBD8425002010B504469A
:10F540005AF0C2FE04F500540021C4F870064720AA
:10F5500046F09EF90021482046F09AF946F042FA1A
:10F56000BDE8104045F0F2BE70B5044604F5005306
:10F5700004F5405583F80C24D5F8A0358B42084695
:10F58000164629D0C5F8A0150B685B68984720B3CC
:10F590002046FFF7AFFFD5F8A00503681B68984722
:10F5A0003246C1B204F58F5039F01CFF04F53750D4
:10F5B0000021343004F5805443F0F6FF04F5BD63B8
:10F5C000D3ED007A9FED077AF8EEE77A05F214653D
:10F5D00067EE877AC5ED007A70BD2046FFF79CFF85
:10F5E000D9E700BF0AD7233CF7B5044600F59C5085
:10F5F000143033F057FB644B04F5405001221C30AB
:10F600009A71DA7104F58C6704F0F8FE04F5375648
:10F610000823C4F874343846343604F05FFD3046AD
:10F6200040F04EFD304644F005FB06F033FC20234D
:10F63000036306F02FFC07F0F3FC04F59F5502234B
:10F64000C4F8A43104F5907008350DF03FFE28464B
:10F6500000F0C0FE04F58053002283F8F126B4F9CF
:10F66000A43004F6C8001BB9B4F8A230A4F8A43042
:10F67000B4F8A41016F0DCFC284600F0A5FF3846CC
:10F68000012104F005FB414B0093414B019302AB78
:10F6900013E9060004F58F5039F0C0FC44F03AFE3F
:10F6A0009922292145F092FD44F034FE44F0DAFD20
:10F6B00004F500552046FFF77FFC05F2644393ED07
:10F6C000007ADFED347AF0EEC76AF4EEE76AF1EE25
:10F6D00010FA04F540574FD805F58D63D3ED007A45
:10F6E000DFED2D6AB0EEE76AB4EEE66AF1EE10FAED
:10F6F00042D8DFED2A6A27EE267A67EEA67ABDEEBB
:10F70000C77AFDEEE77A17EE103AC7F8983517EE8C
:10F71000903AC7F89C35D7F8983543B9D7F89C3557
:10F720002BB904F5565110312046FFF759FE1C4BFA
:10F730001B68986A03684FF47A715B68984795F97B
:10F7400096142046FEF79EFE014610B904F5565168
:10F750002C311F22204605F26C45FFF705FFD5ED41
:10F76000007AF5EEC07AF1EE10FA0BDD204603B018
:10F77000BDE8F040FFF7E2BE0A4A052130463CF002
:10F78000C5FAC8E703B0F0BD8D5D002088250020D4
:10F79000DDF300080000B442000034438096184BAB
:10F7A00084250020048D090808B50A2922D8DFE83D
:10F7B00001F00D1911151D2121212121060000F54F
:10F7C00056512431FFF7D0FE012008BD00F55651F7
:10F7D0002C31F7E700F557510C31F3E700F557519D
:10F7E0001031EFE700F557511431EBE700F55651B2
:10F7F0003031E7E70020E8E700F58F503AF0AABA89
:10F8000000207047002070470148032146F0DEB910
:10F81000005D002070B505462DED028B05F54054C6
:10F820005AF046FDD4F8FC35DFED227AC31A08EE13
:10F83000103AB8EE488A28EE278AF1EE047AB4EE40
:10F84000E78AF1EE10FA33D504F2DC530FCB04F261
:10F85000EC5686E80F0004F5C163D3ED000A04F20C
:10F86000046393ED000A05F5575068EE200A28EE70
:10F87000000A2C3005F07AFD04F20C6393ED007A57
:10F88000DFED0D7AD4F8F03527EE277A07EE903ABF
:10F89000F8EEE77AE7EE087AFDEEE77A17EE903AAF
:10F8A000C4F8F035012384F8D835BDEC028B70BD67
:10F8B0000023F8E7BD3786350000C84230B585B073
:10F8C0006D460446284605F0C1FA04F59F502946C6
:10F8D000083001F0D3FC50B104F54054002384F803
:10F8E0003A3695E80F0004F5B26484E80F0005B0DD
:10F8F00030BD0000F8B52DED028B00F540540546F3
:10F9000094F8D835002B69D0D4F8A02500F55753CA
:10F910000C3300F5565600F557579A4206F110067B
:10F9200007F12C0719D094F83436DA0715D4394684
:10F93000304605F009FC9FED2C7AF6EE007AE0EEF9
:10F94000077A04F214639FED297AFDEEE77AF8EE68
:10F95000E77A67EE877AC3ED007A3046394605F0DC
:10F9600095FC05F5005504F5C36383ED000A95F990
:10F970007234DFED1F6A012B05BFD4F8F035D4F8DF
:10F980009425D4F810369B1A07EE903AF8EEE77AF1
:10F9900004F22C6687EEA67A86ED007AD4F8A005EC
:10F9A00003681B689847022818D094F834369B07E0
:10F9B00014D404F5C363D3ED000A95F972349FEDB6
:10F9C0000D8A04F21C6563B904F5C56494ED000A60
:10F9D0007EF02AFE20EE080A85ED000ABDEC028BBF
:10F9E000F8BD96ED000AF3E7A00CB3450AD7233C17
:10F9F0000000C842E02E654273B5044604F5005588
:10FA0000FFF708FF2046FFF759FF05F26C46204636
:10FA1000FFF770FFD6ED007AF5EEC07AF1EE10FA3E
:10FA200009DC244B1E68F06A0368DB6998470128EB
:10FA300016D102B070BD5AF047FCD5F8703696ED7D
:10FA4000007ADFED1D6AC01A07EE900A27EE267ACB
:10FA5000F8EE677AF4EEC77AF1EE10FAE1D5E8E74E
:10FA6000F36A93F89C10E9B995F99734012B10D1FA
:10FA70009FED120A472045F04FFD9FED100A4820E8
:10FA800045F04AFD45F0AEFF02B0BDE8704045F0DC
:10FA90005DBC4720019145F0DDFE0199482045F00D
:10FAA000D9FEEFE704F54054D4F8A00503689B683D
:10FAB0009847E7E78425002000007A440000000012
:10FAC00037B54B68054613B98A68002A51D005F549
:10FAD00040540A20C4F8E4358B68C4F8E835CA6895
:10FAE00092FBF0F2C4F8E0250B6993FBF0F3C4F845
:10FAF0001036B1F91630DFED207AB1F9142007EE97
:10FB0000103AB1F91830B8EEC77A87EE276A07EED7
:10FB1000103AB8EEC77A04F20463C7EE276A07EE1C
:10FB2000102AB8EEC77AC7EE275AC3ED005A04F57B
:10FB3000C16383ED006A04F20C63C3ED006A5AF0FE
:10FB4000B7FBC4F8FC055AF0BFFB0221C4F800065D
:10FB50002846FFF751FE60B105F558530433009372
:10FB6000D4F8E035D4F8E825D4F8E4152846FEF7B3
:10FB7000C7F903B030BD00BF0000C84210B52DED7D
:10FB8000028B044691ED018ADFED227A94F87134FC
:10FB900028EE278A00F58C60242202FB0303F0EE96
:10FBA000480A93ED090A03F01BFDB4EE400AF1EE9A
:10FBB00010FAF0EE400A24D69FED177AF0EEC07AE4
:10FBC000F4EE477AF1EE10FA1BDC04F5405303F52E
:10FBD000C661D1ED007A77EE807A03F5C562C2ED99
:10FBE000007A93F8340640070BD5F1EE407AC1ED68
:10FBF000007A0021116093F834266FF3820283F8B3
:10FC00003426B0EE480ABDEC028B2046BDE8104019
:10FC1000FEF752B90000C842FFFF7F7FB1F9002014
:10FC200007EE902A00F54050F8EEE77A00F21463F0
:10FC300010B5C3ED007AB1F9022007EE902AF8EE74
:10FC4000E77A00F21C63C3ED007A00F5C36300227B
:10FC50001A60B1F9002090F8343647F6FF74121B91
:10FC600018BF012262F3000380F83436B1F9023084
:10FC700090F834261B1B18BF012363F3410280F860
:10FC8000342610BD10B500F54054D4F8000650B12C
:10FC90005AF01AFBD4F80036C01A41F28733984262
:10FCA0008CBF00200120014B187110BD8D5D00201C
:10FCB00070B52DED028B00F5005400F5405316464B
:10FCC00003F21462D2ED008AB4F9922401EE102AF4
:10FCD000B4F9902403F21C6300EE902A04F59162BB
:10FCE000D3ED007A92ED000ADA20B8EEC11AF8EEF0
:10FCF000E00A30EE270A0D4616F03CFEB4F99024D7
:10FD0000B4F9923407EE902AF8EEE77A9B1A30EEB7
:10FD1000670A07EE903A30EE000AF8EEE77AB7EE9F
:10FD2000008A80EE277A04F2844337EE487A86ED23
:10FD3000007A93ED000A38EE800A16F087FDB4F9D8
:10FD40008C3407EE103A30EE000AB8EEC77A012084
:10FD5000C0EE077A77EEC87ABDEC028BC5ED007A6B
:10FD600070BD000070470000002070477047000021
:10FD70000020704700207047002070470020704727
:10FD80009FED010A704700BF000000009FED010ACF
:10FD9000704700BF0000000070470000002070475F
:10FDA0007047000010B50446143000F019F804F153
:10FDB0002C0000F015F804F174005AF091FA04F1E7
:10FDC000F4005AF08DFA4FF0FF33C4F8503120465A
:10FDD00010BD0000014B1868704700BF045D002093
:10FDE00070470000F0B52DED048B91B004466D46D0
:10FDF000284605F02BF894F8BC33002B72D004F59C
:10FE00007A730FCB85E80F0094F8F833D4EDEC8AC1
:10FE100094EDED8A94EDEE9A002B63D094F8D033F4
:10FE2000002B5FD02D22002104A8D4F8C073D4F891
:10FE3000C463D4F8C853D4F8CC4380F0DBFDA323CB
:10FE40008DF8103095238DF8113046238DF812303F
:10FE50005AF042FA9FED250A9FED257ACDF817104A
:10FE600068EE807ACDF8130067EE877AFDEEE77AC8
:10FE700017EE903A68EE007A29EE000A67EE877A6C
:10FE8000ADF81B30FDEEE77A20EE070A17EE903A48
:10FE9000ADF81D3016F004FDDDED017A9FED157A09
:10FEA000CDF82D70BCEEC00AF8EEE77A10EE103AED
:10FEB00067EE877AADF81F3017EE903ACDF8213013
:10FEC000029BCDF82530039BCDF82930CDF8316069
:10FED000CDF83550CDF8394039F072FF2D2204A904
:10FEE00039F0C0F811B0BDEC048BF0BDE02E6542D6
:10FEF0000000C8420AD7233C30B52DED028B8BB0F1
:10FF0000044624220D4601A8002180F073FDA3239E
:10FF10008DF8043095238DF8053048239FED1F8A16
:10FF20008DF806305AF0D8F9D4ED817A2B68CDF8E7
:10FF30000F3067EE887A95ED020ACDF80B1017EEB8
:10FF4000903AD4ED827ACDF8133067EE887A6B68F8
:10FF5000CDF8173017EE903ACDF80700CDF81B30EA
:10FF600016F074FC10EE103A94ED830ACDF81F30B1
:10FF700020EE080A16F06AFC10EE103ACDF8233095
:10FF800094F80C338DF8273039F01AFF242201A998
:10FF900039F068F80BB0BDEC028B30BDE02E654245
:10FFA00030B587B014460D4618220021684680F00F
:10FFB00021FDA3238DF8003095238DF801304923CE
:10FFC0008DF802305AF088F9A3680393E36804932C
:10FFD0006368CDF807100593CDF803008DF80B503A
:10FFE00039F0EEFE1822694639F03CF807B030BD12
:10FFF00010B58EB0044602A804F028FF02A92046DE
:020000040801F1
:1000000001F03CF9002845D001F076FB694600F08C
:10001000CDFF1F22002106A880F0ECFCA3238DF861
:10002000183095238DF819304A238DF81A305AF07C
:1000300053F9DDED037A9FED1B7A049BCDF8233055
:10004000F8EEE77A059BCDF8273067EE877ACDF892
:100050001B0017EE903ADDED007ACDF82B30F1EE73
:10006000677A17EE903ACDF81F10204601A9CDF817
:100070002F3000F00FFC78B1DDED017AF1EE677AF8
:1000800017EE903ACDF8333039F09AFE1F2206A9C8
:1000900038F0E8FF0EB010BD39F092FEDFED027AC5
:1000A000EEE700BF0AD7233C5241C07F0023036024
:1000B00043608360C360036143618361C361036222
:1000C0007047000090F8F432B02202FB030390F86E
:1000D000382393F8D13012B1012B28BF01231846E1
:1000E000704700002DE9F04F04468BB04FF0000A36
:1000F0000D461CF0D3FC84F814A204F506704FF0F2
:100100007E5759F03DFA4FF47A73A4F8623284F8BE
:100110006852C4F84872C4F84C72C4F8507204F5BE
:100120001B70002504F092FE04F52B790323C4F81C
:10013000803204F53476C4F89452C4F89852C4F866
:100140009C52C4F8A052C4F8A452C4F8A85248461D
:10015000FFF7ACFF04F5487B3046FFF7A7FFC4F874
:100160001453C4F81853C4F81C535846FFF79EFFA5
:10017000C4F84453C4F84853C4F84C53C4F850531B
:10018000C4F85453C4F85853C4F85C53C4F86053CB
:10019000C4F86453C4F86853C4F86C53C4F870537B
:1001A000C4F88C53C4F89053C4F89453C4F8A853BB
:1001B000C4F8A453C4F8A053C4F8B053C4F8B4535B
:1001C000C4F8B853C4F8CC53C4F8C853C4F8C453E3
:1001D000C4F89C73C4F8C07304F5757004F036FE5F
:1001E00004F57A7004F032FE04F58063C4F8FC5321
:1001F0001D6004F5816304F583601D605D609D6092
:1002000004F024FE04F22C4304F264481D605D6097
:100210009D606D4BC4F83C3404F50D73C4F8403454
:1002200004F50E73C4F8443404F50F73C4F848346D
:1002300004F51073C4F84C3404F24523C4F8503468
:1002400004F51173C4F8543404F58B6340461D6003
:100250005D609D60FFF72AFF04F59160FFF726FFC0
:1002600004F5976304F23C421D605D609D6004F2FA
:10027000C44304F2BC501D605D609D6004F59A6348
:100280001D605D609D6004F2DC431D605D609D60EB
:1002900004F2EC431D605D609D6004F2FC431D6050
:1002A0005D609D6004F5A1631D605D609D6004F26A
:1002B0002C53C2F8E070C2F8E4701D605D609D6070
:1002C00004F5A7631D605D609D6004F244531D60EA
:1002D0005D609D6004F5AC631F605D6004F2845353
:1002E0001D605D609D6004F5B2631D605D609D6092
:1002F00004F5B5631D605D609D6004F0A7FD04F228
:10030000CC5324221D605D6004F2D45351461D601D
:100310005D6004F2DC5340461D605D6080F06AFB66
:1003200004F2FC50C8F82070C8F81070C8F80070CB
:10033000FFF7BCFE04F5C46304F5CA601D605D6090
:100340009D6004F22C631D605D609D6004F5C763D1
:100350001D605D609D6004F244631D605D609D6092
:1003600004F074FD194B1A491C60204635F0ACFCB2
:1003700051462422584680F03DFBC4F84073C4F82F
:100380003073C4F8207304F5257207CA04F5287386
:1003900083E80700484694EDAA1AD4EDA90A94ED23
:1003A000A80A16F0DFFE3546494668466E4616F046
:1003B000FBFD0FCE0FC50FCE0FC533682B60204657
:1003C0000BB0BDE8F08F00BF448F0908085D002026
:1003D000F48D090810B5044688B001F017FA94F9B5
:1003E0003232012B02D1274804F014FD022B0AD12E
:1003F000032384F8323204A9012304F111008DF89B
:10040000103036F023FA94F8323284F8903204F245
:100410003C4001F0B1F994F93132642B30D16523BD
:1004200004A904F231208DF8103036F04DFA04A9F9
:10043000204634F091FC18B304238DF818300023C3
:10044000CDE9013303930F230593694604A834F0E3
:1004500003FE059B28B108AA02EB8302009942F82B
:10046000581C0133112B0593EFD957F0B1FD9DEDC9
:10047000031ADDED020A9DED010A652157F066FDC4
:1004800008B010BD548D090870B500F5257600F54B
:1004900028758CB004463146284618F091FAE0B928
:1004A00096E8070085E8070004F52B7194EDAA1A79
:1004B000D4EDA90A94EDA80A0191084616F052FE5F
:1004C00002AD019902A816F06FFD0FCD04F534744A
:1004D0000FC40FCD0FC42B6823600CB070BD00009B
:1004E00013B540F2411200F50671044601A812F05E
:1004F00047FB04F23C4001F027FB20461CF0ACFC1B
:1005000001A812F05FFB02B010BD0000F8B50B6847
:10051000C0F804324B68C0F808328B68C0F80C325F
:1005200001F10C0607460C4600F548750FCE0FC5C5
:100530000FCE0FC533682B6004F1300207CA07F5F0
:10054000457383E8070004F13C0207CA07F55173BD
:1005500083E8070004F1480207CA07F5547383E8EB
:100560000700543494E8070007F5577383E8070041
:10057000384601F05FFA3846BDE8F84001F042BA6B
:1005800013B5044600F23C40019002F021FF04F54F
:10059000BE610198009102F02FFA0099204602B046
:1005A000BDE81040FFF7B2BF4A78064BC2F34012D5
:1005B0001A754A78C2F380125A750A78C2F300128B
:1005C0009A7570478D5D002013B540F2F522044600
:1005D00000F5067101A812F0D3FA002104F23C40A4
:1005E00001F026FD94F8603223B120461CF0ECFDAA
:1005F00084F8600201A812F0E5FA02B010BD000014
:1006000038B590F80C3305460C462BB1032B0BD0B4
:1006100095F86832DB070CD405F5CA630FCB84E884
:100620000F0095F8600603E01CF06CFC0028EFD08A
:1006300038BD0020FCE7000000F23C4090ED380A95
:100640007047000000F23C4090ED390A704700000E
:1006500010B490F80C230C462AB1032A0AD00020CB
:100660005DF8044B704700F5B56007C884E80700E3
:100670000120F5E75DF8044B1CF02CBC90F88403D6
:10068000431E58425841704738B590F80C330D4618
:100690008BB900F23C4001F0C9FA044610B90024BD
:1006A000204638BD01F016FAD5ED007A27EE800A13
:1006B00085ED000AF4E7D0EDE07AC1ED007A90F81C
:1006C0007C43002CEBD090EDDE7ADFED086AB4EECF
:1006D000E67AF1EE10FAF7EE006AB8BFB0EE667A8D
:1006E00067EE877AC1ED007ADAE700BF00000034D8
:1006F00090F80C33032B01D11CF06CBB0020704729
:1007000090F80C23032A01D11CF092BC00F23C406B
:1007100001F0F0BE30B590F80C3385B004460D46BC
:100720008BB1032B18D004F5257018F083F92846F7
:1007300001A98DED010ACDED020A8DED031A17F026
:10074000B3FF012006E000F23C4001F019FA002856
:10075000E9D1002005B030BD90F86032002BF8D010
:100760001CF04EFCDFE700007FB590F80C2332B19F
:10077000032A4FF0000309D0039304930CE000F226
:100780003C4007B05DF804EB01F0D6BA03A903932F
:10079000049305931CF014FB9DED030ADDED040AA0
:1007A00007B05DF804FB000007B590F80C3333B1D7
:1007B00000F57F7003B05DF804EB18F091B800F21B
:1007C0003C4001F0B9FA68468DED000ACDED010A12
:1007D00018F086F803B05DF804FB000090F80C03F5
:1007E000003818BF0120704708B590F80C23032A81
:1007F00005D0BDE8084000F23C4001F085BA1CF08D
:10080000DFFA012008BD000010B590F80C230C465B
:100810001AB1032A07D0002010BDBDE8104000F235
:100820003C4001F015BA1CF0E1FA012084ED000A09
:10083000F2E7000090F80C33032B01D11CF0C0BB91
:100840000020704730B590F80C3385B005460C4653
:1008500023B1032B09D0002005B030BD00F23C408D
:1008600005B0BDE8304002F0F7B8002302A90293BA
:1008700003931CF08DFA0028EDD001A928461CF046
:1008800093FA0028E7D0029B2360039B6360019BDF
:10089000A360E1E790F80C231AB1032A05D00020E9
:1008A000704700F23C4002F0FDB81CF07DBA000039
:1008B00090F932323BB990F8683213F0010F14BF4F
:1008C000032000207047032070470000F7B504465E
:1008D000FFF7EEFF0546002862D0032839D194F8CF
:1008E00060326BB394F86832D8072BD501A9204643
:1008F0001CF09CFDBDF80430002B18BF002594F8B7
:10090000146206F0FD06012E4AD10023032D019347
:1009100007D101A920461CF095FD20461CF094FB50
:10092000064604F23C4002F049F908B994F809037C
:100930009DF80430D90703D55A0701D59F0632D454
:1009400000252DE020461CF0FDF9002808BF0025F9
:10095000D5E70025D3E713F0020F2EE094F94432D7
:1009600023B99DF80430DB092FD0E9E7002EF8D039
:100970000DF0F4FFFFF7A6FB022807D99DF805301C
:100980009806DDD59DF80430D906D9D5FB6A93F8D1
:100990009C30002BE5D118E0DA0601D41B0718D5EE
:1009A000284603B0F0BD0028FAD094F80923B4F922
:1009B0006436002ACFD013F0010FF1D1154B1F6818
:1009C000FB6A93F89C30002BC8D19DF804309C073B
:1009D000E2D405F05FFA05F05BF90028B0D10DF024
:1009E000BDFFFFF76FFB0228AAD90DF0B7FF90F803
:1009F000F432B02202FB030090ED3B7AF0EE007A75
:100A0000B4EEE77AF1EE10FA9AD59DF80530DB09DD
:100A1000C6D195E7842500202DE9F04790F8603293
:100A200092B00446002B00F0948020461CF00AFE91
:100A30002046FFF74BFF03287BD104F548780027B9
:100A4000414620460097019702971CF0CFFA69466D
:100A500020461CF0C1FA009BC4F80432019BC4F884
:100A60000832029BC4F80C32204600F0E3FF204617
:100A700000F0C8FF15F032FA054620461CF07AF95E
:100A80000028A8BFC6B203AA4FF0FF312046BCBF62
:100A900095F8EB9495F8EC640397A8BFB1460497DA
:100AA00005971CF0B1F903A817F0C4FF4FF00C0A2A
:100AB0000AFB095084EDD10AC4EDD20A84EDD31AA1
:100AC00004F5517100F55C7017F0C4FF04F5577719
:100AD0000AFB065584EDC50AC4EDC60A84EDC71AA3
:100AE0003A464FF0FF31204605F500751CF0A0F99D
:100AF00095E8070006AE86E807003946304618F04C
:100B00000FF804F52B72414609A816F0DDF93146BD
:100B100009A816F05BF909A9204684EDD40AC4EDB2
:100B2000D50A84EDD61A1CF08DFC09A92046FFF7E2
:100B30003BFD94F86636002B3AD109A804F086F9FB
:100B400009A920461CF0EAF990B3012384F866361F
:100B50002EE0D0F864321BB959F0B6FBC4F8640239
:100B6000154B1B68D86A03685B68984788B159F0D1
:100B7000ABFBD4F86432C01AB4F86232984204D99C
:100B800020461CF021FB84F8600294F860327BB1AF
:100B90004BE759F099FBD4F86432C01A41F287331D
:100BA0009842E4D839F00CF939F0F0F80028DED199
:100BB00012B0BDE8F08700BF8425002090F80C3308
:100BC00023B1032B4FF0000007D0704790F9322279
:100BD000032A04D10A70012070470870FBE7184609
:100BE0007047000073B50D460DF107010446FFF78D
:100BF000E5FF064628B19DF807302BB1032B09D03D
:100C00000026304602B070BD04F5CA630FCB85E8FC
:100C10000F00F6E7294620461CF074F994F860624C
:100C2000EFE700007FB50E460DF103010446FFF724
:100C3000C5FF054618B90025284604B070BD9DF8CB
:100C4000033083B1032B16D004F5257017F0F2FEA4
:100C500001A930468DED010ACDED020A8DED031A92
:100C600017F022FDE8E7314604F23C4000F088FF2F
:100C70000028E9D1DFE794F86032002BDBD0314661
:100C800020461CF0BDF9DFE737B50D460DF1070131
:100C90000446FFF793FF28B19DF8073023B1032BDB
:100CA0000FD0002003B030BD04F5BE631B682B607D
:100CB00004F2F45304F5BF641B686B602368AB60F7
:100CC000F0E7204629461CF087F994F86002E9E72E
:100CD00010B50446FFF7ECFD18B1032807D000203B
:100CE00010BD04F23C40BDE8104000F073BF94F822
:100CF0006032002BF3D020461CF024F80028EED000
:100D000094F8143203F0FD03012BE9D194F80C039D
:100D1000C31E58425841E3E710B50446FFF7C8FD2B
:100D200080B1032810D194F8600250B159F0CCFA88
:100D3000D4F86432C01A44F62063984294BF00206D
:100D4000012010BD0120FCE70020FAE708B50246AB
:100D5000FFF7AEFD032804D110461CF073FB012001
:100D600008BD0020FCE7000030B585B004460191C5
:100D7000FFF730F80199054610B9002005B030BDE5
:100D80000191FEF7F7FF01990028F6D02846FEF7FB
:100D9000F5FF0028F1D0B4F864365907EED494F882
:100DA0000933002BEAD00B4A1268D26A92F89C50A1
:100DB0006DB103A92046FFF7C9FF30B19DF80E3091
:100DC0009A07DBD5C3F38000D8E72846D6E7184654
:100DD000D4E700BF842500202DE9F04190F80C33C2
:100DE0008CB00027032B06460C461546009701974A
:100DF000029719D11BF0BEFF6A4680464FF0FF31C3
:100E000030461CF015F8B8F1FF3FA7606760276017
:100E10000DD115F063F82B4690F8EC14224613F030
:100E20008DFF0CB0BDE8F0814FF0FF38EBE715F017
:100E300055F82B4622465FFA88F113F07FFF95EDB7
:100E4000000A684617F032FE03A920468DED051A08
:100E50008DED030ACDED040A17F062FE06F52B7244
:100E600006F5487103A816F02FF8214603A815F0DF
:100E7000ADFF84ED021A84ED000AC4ED010A95ED80
:100E8000007ADFED037AA7EE271A84ED021AC8E78D
:100E90000AE81C4137B5054600F5067140F60332F5
:100EA00001A811F06DFE2846FFF702FD044640B18F
:100EB00003280AD0002401A811F084FE204603B0C4
:100EC00030BD28461BF0E2FFF5E728461BF0DEFFA9
:100ED0000446F0E708B50246FFF7EAFC10B1032824
:100EE00006D008BDBDE8084002F23C4000F03CBE20
:100EF000BDE8084010461CF0B1BA00000B4610B423
:100F000011462BB1032B09D000205DF8044B70472C
:100F10005DF8044B00F23C4000F03CBE5DF8044B31
:100F20001BF0FCBF13B50446FFF7C2FC0A4601469E
:100F300020460192FFF7E2FF70B9084B019A1B6847
:100F4000DB6A93F89C0038B194F80C13204602B089
:100F5000BDE81040FFF7D2BF02B010BD84250020CD
:100F600037B504460D4640F2B25200F5067101A8AD
:100F700011F006FE294620461BF0EEFF94F80C33D4
:100F8000032B054610D148B104F583612046FFF7D5
:100F9000C9FF84F82804204600F07CFD01A811F068
:100FA00011FE284603B030BD0025F7E770B590F874
:100FB0007C32DB0786B004460D460CD402F0BEFF3F
:100FC000437C242202FB0300D0ED0B7AF1EE677A1A
:100FD000C5ED007A3BE002A803F038FF01A92046E6
:100FE000FFF758FCE8B90DF0B9FC94F94432022B34
:100FF0000646E3D1FFF766F80228DFD996F8F40237
:101000009FED147AB02303FB0066D4F87032D6F853
:10101000E0209B1A07EE903AF8EEE77A67EE877ABF
:10102000D6E702A92046FFF77DFF0028DBD0D4F8E1
:101030007022039BDFED076A9DED017A9B1A07EE94
:10104000903AF8EEE77AA7EEE67A85ED007A06B0F8
:1010500070BD00BF0AD7233CF0B50C4687B000F541
:101060000671064640F6863201A811F089FDA36894
:1010700053B9E36843B9636833B9002701A811F095
:10108000A1FD384607B0F0BD204603F0B5FF0028AB
:10109000F3D094E80F0002AD85E80F000021284648
:1010A00003F06CFF07460028E7D096F87C32DB0798
:1010B00004D438F085FE192138F0BEFD95E80F0004
:1010C00006F51B7C8CE80F0096F87C3243F0010398
:1010D00086F87C32304600F0DDFC41F047FC4621CA
:1010E00042F062FA41F042FC452142F05DFA054BC4
:1010F000A2681B68DB6A1A61E2685A6162689A61D9
:10110000BCE700BF8425002038B5144B1B68DD6A9E
:101110002B6804465B6828469847F0B12B690BB9E9
:101120006A69D2B1C4F874326B69C4F87832A969BB
:10113000002204F51B7003F08FFE94F87C3223F03C
:10114000030343F0030384F87C3241F00FFCBDE855
:101150003840034A06213AF0D9BD38BD8425002025
:101160007C8D090810B588B004460593FFF7A0FBF5
:101170000328059B4FF000000AD10690079006A8AF
:1011800002900B9801900A98009020461BF042FFB5
:1011900008B010BD38B50446FEF71CFE0546D0B1B8
:1011A00094F80C33032B03D095F84E41204638BDFC
:1011B00020461BF09BFEFF280446F5D0014628463A
:1011C000FEF7DCFD0028EFD021462846FEF7D2FDD1
:1011D0000028E9D0EAE70446E8E7000008B590F8FF
:1011E0000C33032B05D014F079FE90F9EB04C0B258
:1011F00008BD1BF0BFFD431CF9D1F4E708B590F81A
:101200000C3383B1032B03D1BDE808401BF0AABD0A
:1012100037F09AF940F6ED424FF4801137F04CF96F
:101220004FF0FF3008BD1846FCE7000090F80C3383
:10123000032B01D11CF052BB7047000090F80C3317
:10124000032B01D11BF0DCBC704700001BF062BD1A
:1012500010B504461EF0D0FB2046FEF7C3FD204625
:10126000BDE81040FEF7C4BE90F80C330BB1032B61
:1012700001D11CF0AFBB00207047000030B500F575
:10128000757304460D460FCB85E80F0094F8E40310
:1012900030BD00007FB5054668460E4603F0D6FD1A
:1012A00095F87C32DB0703D40024204604B070BDDF
:1012B00069462846FFF7E2FF04460028F4D0694655
:1012C00005F51B7003F07CFF86ED000AC6ED010AF0
:1012D000EBE70000D0F880330B6090F87C03704798
:1012E000D0F888330B6090F88503704730B500F56F
:1012F000677304460D460FCB85E80F0094F8AC03E6
:1013000030BD000030B500F5836304460D460FCBB9
:1013100085E80F0094F8280430BD000010B500F2F5
:101320002C4203460C4607CA84E8070093F83804A9
:1013300010BD00002DE9F0432DED028B8BB005466A
:101340000E461746FFF726FF014680462846FFF760
:101350000BFD0446002848D0FEF73CFD4146FEF751
:101360000FFD86ED000A95F93032002B3ADD0DF0C5
:10137000F5FAFEF7A7FE012834D90DF0EFFA90F840
:10138000F432D5EDDE7ADFED5D8A96ED000AB0220B
:1013900002FB030095F93032D0ED3B0A07EE103A1C
:1013A000F4EEE87AB8EEC77AF1EE10FAB7EE008AFA
:1013B000B8BFF0EE487A37EE201A20EE270A70EE1A
:1013C000C70A40F2B63015F0D5FAD5EDDE7AF4EE64
:1013D000E87AF1EE10FAB8BFF0EE487A80EE277A9C
:1013E00086ED007A01233B7003E095F8083333B9AA
:1013F000387020460BB0BDEC028BBDE8F08395F849
:101400000C334FF00009CDF80490CDF80890CDF8DA
:101410000C9043B1032B10D0CDF81090CDF8149060
:10142000CDF818907CB902233B703246414605F254
:101430003C4001F087FB0446DBE701A928461BF08E
:1014400049FD0446E8E795F80C33002BEBD004A9DE
:101450002846FFF763FF04460028E4D001A904A84A
:1014600017F00EFB07A8CDED080A8DED091A8DEDDA
:10147000070A17F019FF04A8B0EE408A17F014FF0E
:1014800095F93032002B30DD07EE903AF8EEE77A2E
:101490004FF47F7070EE670A37EE801AF5EEC00ADF
:1014A000F1EE10FA48BFDFED160AF4EE410AF1EE54
:1014B00010FAB0EE480AC8BFB0EE601A15F05AFA3A
:1014C000B0EE408AD5EDDE7A9FED0C7AF4EEC77A65
:1014D000F1EE10FAB7EE007AB8BFF0EE477A88EE78
:1014E000277A032386ED007A7DE7B5EEC08AF1EE18
:1014F00010FA48BF9FED028AE4E700BF0000003405
:101500000000000010B50446FFF768FE84F80D03E4
:101510002046FFF763FE84F80E032046FFF75EFEC9
:1015200084F80F032046FFF769FE04F55A7184F82A
:1015300010032046FFF78CF884F8740300F0CAFA11
:1015400004F5617284EDDE0A04F560712046FFF750
:10155000F1FE04F5627184F87C032046FFF794F8ED
:1015600004F5637184F885032046FFF7C1F804F59C
:10157000677184F898032046FFF7CCF804F56C7186
:1015800084F8AC032046FFF77FFB04F5707184F804
:10159000BC032046FFF746FB04F5757184F8D003C1
:1015A0002046FFF72DF804F57A7184F8E40320460D
:1015B000FFF718FB84F8F8032046FFF7D5F804F589
:1015C000806384EDFF0A2046C3ED000AFFF7ECF8C4
:1015D00004F2044383ED000A04F2144204F581612D
:1015E0002046FFF7F9FB04F583612046FFF79AFCDC
:1015F00004F22C4184F828042046FFF7F5F884F81B
:10160000380410BD37B50D46044600F0FFF81DB98B
:1016100014F064FC13F066FA4FF4BE7204F5067120
:1016200001A811F0ADFA94F869322BB92046FFF702
:101630006BFD012384F86932224B1D68A86A036898
:101640009B6998472046FEF71FFF2046FEF798FF4C
:10165000204600F051FA2046FFF7DEF9286B30B142
:101660000368D4EDD20ADB6894EDD10A9847D4F828
:10167000100208B159F096FD204600F07DF8204692
:10168000FFF724F994F8903284F80C0383420ED0CB
:1016900084F8900298B10C4D0C4B032808BF1D46EE
:1016A00041F064F90A4A2B4606213AF02FFB204606
:1016B000FFF728FF01A811F085FA03B030BD054DF2
:1016C000EEE700BF84250020BF600908738D09087C
:1016D000948D0908788D0908D0EDDE7A9FED057AA2
:1016E000F4EEC77AF1EE10FAB7EE000AA8BFB0EE3A
:1016F000670A704700000034014B1868704700BF4C
:10170000085D00204FF0FF30704700000120704757
:1017100070470000002070470020704770470000AD
:10172000704700000020704700207047002070477D
:10173000002070470020704700207047002070474D
:10174000012070470368D3F8943018470020704791
:10175000002070470020704700207047002070472D
:10176000002070470020704700207047002070471D
:1017700000207047704700007047000008B514F063
:10178000ADFB90F8EC0408BD08B514F0A7FB90F889
:10179000EB0408BD30B52DED028B9FED1A1ADFED7D
:1017A0001A0A91ED000A87B005462D200C468DEDF2
:1017B000011ACDED000A15F0DDF89DED011ADDED01
:1017C000000AF0EE408A2E2094ED010A15F0D2F8BE
:1017D0009DED011ADDED000AB0EE408A2F2094ED58
:1017E000020A15F0C7F803A905F52570CDED038AA7
:1017F0008DED048A8DED050A35F04AF907B0BDEC90
:10180000028B30BDC2B8323EC2B832BE10B50446FB
:1018100058F05AFDD4F8F4321BB1C21AB2F57A7FEF
:1018200012D30A4A1268D26A92F89C2002B15BB9BC
:10183000C4F8F40294F8314214F050FB80F8E2440A
:1018400004F028FB80F8254010BD00BF842500204F
:101850002DE9F0432DED028B91ED007AD1ED037A65
:1018600087B08DED047AB0EEC77AB5EEC07AF1EEAE
:1018700010FADDE91087DDF84C90CDED057A0C46C5
:1018800015461E4606DCF0EEE77AF5EEC07AF1EE7C
:1018900010FA02DD04A817F075F86B20B7EE001AF5
:1018A000FFEE000A9DED050A15F064F86C2089ED45
:1018B000000AB7EE001AFFEE000A9DED040A15F0CB
:1018C00059F804A888ED000A16F0E4FFB7EE008A84
:1018D000002852D00023C9F8003088ED008AD4EDEA
:1018E000067A67EEA77AF4EEC87AF1EE10FA4ADBD0
:1018F0000023336085ED008ADFED3F0A96ED000A94
:101900007C20B7EE001A15F035F886ED000A95ED4B
:10191000000A7D20B7EE001AFFEE000A15F02AF843
:1019200085ED000AD4ED067A129BDFED346AF1EE04
:10193000677AC3ED007A96ED007AF0EEC77AF4EE9E
:10194000E67AF1EE10FA2BD503AB02AA01A92046E4
:1019500015F068FC9DED018AB0EE480A7CF042FC6F
:1019600085ED000AB0EE480A7CF092FD87ED000A92
:1019700007B0BDEC028BBDE8F08304A816F076FF3B
:101980000028A7D1ABE738EE670A14F025FF86EDF3
:10199000000A94ED087AC7EE007AC5ED007AABE74D
:1019A00094ED076AC6EE077AC7ED007A96ED007AE5
:1019B000B0EEC77AB4EEE67AF1EE10FAC4D495ED43
:1019C000007ADFED0F6AB0EEC76AB4EE666AF1EE38
:1019D00010FAB9DCB4EE477AF1EE10FAB4D6B0EEF4
:1019E000E77AB4EE667AF1EE10FAADDCF4EE677ADF
:1019F000F1EE10FABCD7A7E70000000000000034A9
:101A0000FFFF7F7F1FB500F51773039300F5167373
:101A1000029300F51573019300F51473009300F51C
:101A2000127200F5137300F54871FFF711FF05B04E
:101A30005DF804FB9FED156A90ED817ADFED146A85
:101A4000D0ED837A27EE067A67EE867A27EE267A3D
:101A500067EEA67ABDEEC77AFDEEE77A80ED7E7A74
:101A600090ED827A27EE067A17EE903A27EE267AE4
:101A7000002BB8BF03F50C43BDEEC77AB8BFA03347
:101A800080ED7F7AC0F80032704700BFE02E6542DB
:101A90000000C8421FB50E4B1B680446B3B1684630
:101AA00003F0D4F969462046FFF72CFC20B16A46C2
:101AB00000212046FEF774FA94F87C32DB0705D546
:101AC00004F51B7201212046FEF76AFA04B010BD2E
:101AD000D45F002008B502F031FABDE8084001F0FB
:101AE000BFBD000010B580F8F812044658F0ECFBBA
:101AF000C4F8FC0210BD000010B590F8F83204469E
:101B000053B158F0E1FBD4F8FC32C01AB0F57A7F3B
:101B100084BF002384F8F83294F8003353B158F0AE
:101B2000D3FBD4F80433C01AB0F57A7F84BF002306
:101B300084F8003310BD000000F5B6700B4607C8EE
:101B400083E80700012070470023C0F89C30C0F8EC
:101B50009830C0F89430C0F8A830C0F8A430C0F86D
:101B6000A030C0F8AC30704770470000024B0B60EB
:101B70004FF07C53136070470000484270470000EC
:101B800008B50B4600F12801184616F0D7F90120D8
:101B900008BD000010B500F5C0700C460FC884E801
:101BA0000F00204603F042F930B1FFF7A5FD00F524
:101BB0001B700FC884E80F00204603F037F980F04F
:101BC0000100C0B210BD000010B5044603F0E2FBF6
:101BD000204610BD10B5D0F8783104465BB158F0FE
:101BE00073FBD4F87831C01A41F28833984294BF1D
:101BF0000020012010BD0120FCE7000013B5009378
:101C000003680192D3F890309847DDE9002104463B
:101C100028B90448044B0068C06A11F08FF92046C7
:101C200002B010BD84250020B48E090813B5044607
:101C30000191FEF7CFF82368019A1B6D014608B1A8
:101C400090F84E11204602B0BDE810401847000041
:101C500030B585B0002301930293039303680D46CA
:101C6000DB6D01A99847044620B1039B2B602046F9
:101C700005B030BD02F062F9417C01F02DFE044652
:101C80000028F4D002F05AF901F08CFDB1EE400AC0
:101C900085ED000AEBE7000090ED007ADFED0F7AAA
:101CA000B0EEC77AB4EEE77AF1EE10FA14D590ED03
:101CB000017AB0EEC77AB4EEE77AF1EE10FA0BD5FE
:101CC00090ED027AB0EEC77AB4EEE77AF1EE10FA50
:101CD0004CBF0120002070470020704700000034F6
:101CE00010B5FEF777F8044658B190F84E11FEF79C
:101CF00041F830B194F84E112046BDE81040FEF78F
:101D00003DB8002010BD000038B50D460CF026FE91
:101D10000446FEF7D7F9022881BF94F8F402B023F5
:101D200003FB004000F5827089BF07C8002085E8EA
:101D30000700012038BD00002DE9F0432DED028B96
:101D40008FB003680025DB6C039504950595069517
:101D5000029502A904469847064638B1FFF7BAFE35
:101D6000DDED027A27EE800A8DED020A0CF0F6FD19
:101D7000FEF7A8F90746002E50D0DDED027AD4ED2B
:101D80006A6A94ED6B7A23680B9527EE877A67EE83
:101D9000A67A8DED097ACDED0A7A0C950D959B6C9E
:101DA0000BA9204609AD98470BA9284616F0D8FC88
:101DB000012F8DED030ACDED040A40F2B3800CF043
:101DC000CDFD90F8F432DFED5B7AB02505FB030022
:101DD00090ED3C8A28EE278AB0EE480A7CF002FAA1
:101DE000F0EE408AB0EE480A7CF052FBCDED0B8A53
:101DF0008DED0C0A0CF0B2FD90F8F43205FB0300F7
:101E000090ED3B0A0BA816F0CBFC09AD8DED050A51
:101E1000CDED060A05A896BB03C885E00128CED8FB
:101E20009DED020AB5EEC00AF1EE10FA7FDD07AEB5
:101E3000D4F8AC21D4F8A83107923046089316F0B4
:101E4000CDFC23680B950C950D959B6C0BA920463A
:101E50009847DDED077A9DED0B7A77EE877A9DED59
:101E60000C7ACDED077ADDED087A77EE877A09AB4B
:101E7000CDED087A96E8030083E8030049E0236982
:101E800093ED000AB7EE008A38EE408A16F088FC1F
:101E900004F5C8798DED090A4846B0EE480ACDED43
:101EA0000A0A16F07DFC0BA92846CDED0C0A8DED33
:101EB0000B0A16F055FC04F5D07603AFC4ED650AA5
:101EC000314684ED640A384616F05AFC04F5CC78A5
:101ED0008DED090A4046B0EE480ACDED0A0A16F02B
:101EE0005FFC0BA928468DED0B0ACDED0C0A16F010
:101EF00037FC97E8030084ED660AC4ED670A86E8BC
:101F000003004946404616F02BFC8DED090ACDED45
:101F10000A0A9DED090ADDED0A0A0FB0BDEC028B3D
:101F2000BDE8F083DDE9030185E80300F1E70995E9
:101F30000A95EEE735FA8E3C10B590F84213044648
:101F400003F0C2FB7C23C0B203FB0044D4F8A00022
:101F500010BD0000044B026F1B68DB6A5A60426FC1
:101F60009A60826FDA60704784250020F0B58FB0E8
:101F7000044613F0B3FF002302930393049390F8F5
:101F8000EB1401AB02AA054612F07AFE04F19407A5
:101F9000D8B39DED010AB5EEC00AF1EE10FA34DDBA
:101FA00002A816F093FD04F1B00684ED2C0AC4EDEE
:101FB0002D0A84ED2E1A3946304616F097FD04F1AD
:101FC0007C01304616F046FD04F1880105A88DED30
:101FD000050ACDED060A8DED071A16F03BFD08A89F
:101FE0008DED080A9DED010ACDED090A8DED0A1A65
:101FF00016F05CFD0BA904F128008DED0B0ACDED68
:102000000C0A8DED0D1A15F0B9F995F8EB040C23B7
:1020100003FB0050394600F55C7016F01BFD84EDA3
:102020002C0AC4ED2D0A84ED2E1A0FB0F0BD00006D
:102030002DE9F047824B00251F682DED028BC0F87B
:102040009C50C0F89850C0F89450C0F88450C0F824
:102050008050C567C0F89050C0F88C50C0F88850C8
:10206000C0F8B850C0F8B450C0F8B0500446F86A90
:1020700003688AB05B680E46984704F12809002877
:1020800054D058F021F942F20F7398424ED8FB6AAF
:102090009FED6C8A93ED010A84ED1C0AD3ED020AD0
:1020A000C4ED1D0A93ED031A484684ED1E1A15F07F
:1020B00059F840F05BFCD4ED1E7A67EE887A05464D
:1020C00017EE900AFAF720FAD4ED1D7A67EE887AB7
:1020D000CDE9040117EE900AFAF716FAD4ED1C7A4E
:1020E00067EE887ACDE9020117EE900AFAF70CFA4A
:1020F000554ACDE900010621284639F007FE94ED46
:102100001E8AB0EE480A7CF06DF884ED6B0AB0EEE2
:10211000480A7CF0BDF984ED6A0A58F0D5F8C4F895
:102120007C010AB0BDEC028BBDE8F087A6B194ED4E
:102130001C0AB4EE400AF1EE10FA0DD6D4ED1D0AD9
:10214000F4EE600AF1EE10FA06D694ED1E1AB4EE23
:10215000411AF1EE10FA52D713F0C0FE90F8EC34A9
:102160004FF00C0A0AFB030303F50073074693E8DC
:10217000070007AE86E807004FF01508B2EE028AA6
:10218000F2EE068A304617F08FF8B4EEC80AF1EE88
:1021900010FA38D508F1FF3818F0FF083CD1304666
:1021A00017F082F8F1EE047AB4EEE70AF1EE10FAD5
:1021B00043DD9DED090ADDED087A9DED078A20EEED
:1021C000000AA7EEA70A7CF079FBF0EE400AB0EE19
:1021D000480A7CF029FADDED090A84ED1D0A9DED1F
:1021E000080AF1EE600AB1EE400A7CF01DFA84EDB7
:1021F0001C0A9FED161AD4ED1D0A94ED1C0A4846E0
:1022000014F0B0FF7BE7304617F04EF8B4EEE80A62
:10221000F1EE10FABEDCC2E7384612F081FB384618
:1022200012F060FC97F8EC340AFB037303F50073BB
:1022300093E8070086E80700A4E725676567D8E705
:1022400084250020E02E6542C08E090800000000B1
:102250000021FFF7EDBE000037B5044608461546DD
:10226000019117F021F8B7EE007AC7EE007AB4F8C2
:10227000DC3001980133A4F8DC3094ED367A37EE87
:10228000277A84ED367AB0EE007AF4EEC77AF1EE72
:1022900010FA06D5B6EE007AF4EEC77AF1EE10FA2F
:1022A0000DDC9FED0E7AF4EEC77AF1EE10FA13D53D
:1022B0009FED0B7AF4EEC77AF1EE10FA0CDDB0EE7A
:1022C000670A16F0F3FB012085ED000AC5ED010A4F
:1022D00085ED021A03B030BD0020FBE700247449ED
:1022E000BD37863570B52DED028B00F1280600F163
:1022F00034058AB029460446304616F053FCB6EE43
:10230000008A20EE088A2846B0EE480A16F0CEFB76
:1023100007A93046CDED080A8DED091A8DED070AA3
:1023200016F0AEFB30468DED010AB0EE480ACDED59
:10233000020A8DED031A16F0B9FB07A928468DEDA8
:10234000070ACDED080A8DED091A16F099FB04A9CC
:1023500001A88DED040ACDED050A8DED061A16F0E3
:1023600035FC324601A920468DED070ACDED080A5D
:102370008DED091AFFF770FF58B957F0A5FF01213D
:10238000C4F878012046FFF753FE0AB0BDEC028B7B
:1023900070BD2A4604A92046FFF75EFF0028ECD056
:1023A00004F1400207A92046FFF756FF0028E4D0B9
:1023B000EBE7000030B52DED028B0D4683B091F8B0
:1023C00042130446284603F07FF9C1B27C2000FB8B
:1023D0000151903104F1280014F054FD68468DED50
:1023E000000ACDED010A16F07BFADFED1C7AB4EE9F
:1023F000E70AF1EE10FA05D59FED190A03B0BDEC1E
:10240000028B30BD684616F0BDFA684616F042FAF7
:102410000028F1D1284694ED488A03F0C9FAF0EE7D
:10242000400AB0EE480A14F0A3F980B9284603F038
:10243000BFFA84ED480AB0EE408A7BF0D3FE84ED0B
:10244000490AB0EE480A7CF023F884ED4A0A04F504
:102450009271684616F0ECF9D0E700BF0000003436
:10246000000000009FED0C7AB4EEC70AF1EE10FAFE
:102470000BD4DFED0A7AB4EEE70AF1EE10FA07DCCE
:10248000C0EE077AB0EE670A7047F7EE007AF9E718
:10249000F2EE047AF6E700BFF3665F3F58A00B4107
:1024A00008B51C3016F01CFAF1EE007AB4EEE70A1B
:1024B000F1EE10FA9DBFF1EE027A37EEC00ADFEDC1
:1024C000047A9FED040A98BF20EE270A08BD00BFDA
:1024D000CDCC4C3ECDCCCC3D08B5836993F9000002
:1024E00038B10CF03BFAFDF7EDFD012894BF002058
:1024F000012008BDF8B52DED028B054603F0CAFC9E
:1025000003F0C6FB0446B8B3FFF7F6F890F80933BA
:1025100093B32846FFF7E0FF064668B30CF01EFAB7
:1025200090F8F432B02707FB030090ED3B7AF0EE11
:10253000087AB4EEE77AF1EE10FA1DD495ED1E8A12
:102540000CF00CFA90F8F432DFED1E7A07FB030072
:1025500090ED3C0A98EE270A14F08EF9DFED1A7A16
:10256000B0EEC00AB4EEE70AF1EE10FA08DC57F05C
:10257000ABFE3446C5F86801BDEC028B2046F8BDC1
:1025800005F5B67016F090FEB0EE408A0CF0E6F954
:1025900090F8F4329FED0D7A07FB0303D3ED3B7AFD
:1025A00067EE877AB4EEE78AF1EE10FADFD557F0DE
:1025B0008BFED5F86841001BB0F5FA6F8CBF002484
:1025C0000124D9E7E02E654200003442CDCC4C3FD7
:1025D00010B50A4B1B68DB6A93F89C3004465BB964
:1025E00057F072FED4F87C31C01A44F61F6398424B
:1025F0008CBF0020012010BD0020FCE784250020B6
:10260000F8B52DED068B04460CF0A8F9054603F04D
:1026100041FC064606F078F9002840F0AB802046E1
:10262000FFF768FF002800F0A8803046FFF784FC21
:10263000D4F8E830984200F01A813046FFF77CFC6D
:10264000D4F8E830DFED8F7AC31A08EE903AF8EE4E
:10265000688A304668EEA78AFFF76EFC94F8BC30B3
:10266000C4F8E800F3B9304603F024FBD0B104F11C
:10267000280796F842233946304603F09DF9D4EDF9
:102680001D0AB0EE401A384694ED1C0A14F06AFD9B
:102690000023C4F89030C4F88C30C4F8883001238B
:1026A00084F8BC3020463146FFF784FE95F8F402EA
:1026B00005EB0015B0EE408AD5F8A030C4F8EC3038
:1026C00004F1B000D4ED129A16F0EEFD6368DFED70
:1026D0006E7A93ED007AB4EEE77AF1EE10FA68EED6
:1026E000299AB0EE40AA01D5C3ED007A2046B0EE9B
:1026F0004A0AFFF7B7FE636820EE299A93ED000AB5
:1027000029EE009AFFF7CCFE29EE009A204684EDD0
:10271000249AFFF75DFF38B1D4ED247AB2EE007A47
:1027200067EE877AC4ED247AF0EE007AF4EEE78A59
:10273000F1EE10FA10D5DFED557AB4EEE7AAF1EE1E
:1027400010FA09D5DFED527A69EEA79AD4ED2A7A0C
:10275000E9EEA87AC4ED2A7A9FED4E0A94ED397A13
:10276000DFED4D7AB0EEC88A28EE008AA7EE278A00
:1027700084ED398ABDEC068BF8BDFEF7BDFF90F8FD
:102780000933002B73D02046FFF7A6FE00286ED039
:1027900095F8F42205EB0213D3F8A010D4F8EC302E
:1027A0008B4264D0B02606FB025292ED3B7AF0EEEB
:1027B000087AB4EEE77AF1EE10FA58DBCB1AC4F8D7
:1027C000EC1008EE903A95F8F4329FED341A94ED3F
:1027D0001E0ADFED337A06FB0353D3ED3C9A69EE14
:1027E000819AF8EE688A39EEC00A68EEA78A14F07A
:1027F000ADF8B0EE409A7BF04BFE94F8BC30B0EEF2
:10280000408AF3B1F3EE047AF4EEE78AF1EE10FABF
:1028100017DC95F8F40206FB005595ED3B7AF2EED5
:10282000027AB4EEE77AF1EE10FAFFF649AFDFED87
:102830001D7AB0EEC99AB4EEE79AF1EE10FAFFF6FF
:102840003FAF9FED198AD4ED1D0A94ED1C0AB0EE3E
:10285000691A04F1280014F085FC012384ED248A10
:1028600084ED238A84ED228A84F8BC3028E7BDEC0D
:10287000068B04F188009FED0D0ABDE8F84016F0C4
:1028800069B900BFBD378635CDCC4C3DC2B8B23E2C
:102890000AD7233CCDCC4C3ECDCC4C3F35FA8E3CB8
:1028A0006F12833A1904863F00000000EC51783F14
:1028B00030B50C2303FB010101F1C003144693E87A
:1028C00007008BB004AD85E8070094E8070083E8B3
:1028D00007002846FFF7E0F907AB58B194E8070076
:1028E00083E807009DED070ADDED080A9DED091A52
:1028F0000BB030BD95E80700F2E70000F0B52DED14
:10290000028BD0F830318B60D0F83431CB6085B099
:1029100004460D4601F012FB06460CF01FF8A369B1
:1029200093F90030022B07464BD1FDF7CBFB022871
:1029300047D997F8F432B02202FB0373D3F8E010C2
:102940000022284602F088FAD4ED500A94ED4F0A8E
:10295000284602F00BFD94F8443163B357F0B4FC01
:102960009FED228A97F8F4128DED018A01AA06469E
:1029700038460BF077F8D4F838019FED1D0A361A67
:1029800007EE906AF8EE677A4FF4876027EE800AC8
:10299000B6EE001AF0EE480A13F0ECFFDDED017A16
:1029A00030EE270A04F584708DED010A15F0F8FE6B
:1029B000284602F0DBFC94F8440105B0BDEC028B24
:1029C000F0BD707C242303FB006696ED0B8AFEF7B6
:1029D00093FED0ED9C7A9FED077AF8EEE77AE8EE69
:1029E000077AFDEEE77A17EE901AA9E700000000DB
:1029F0006F12833A0000C842F8B5036F0B60436F53
:102A00004B60836F8B6000F14C050E46074601F169
:102A10000C040FCD0FC40FCD0FC42B68236007F13A
:102A2000B00207CA06F1300383E8070007F19402F9
:102A300007CA06F13C0383E8070007F11C0207CA36
:102A400006F1480383E8070006F160013846FFF706
:102A500055FF86F87000F8BD30B589B00446684669
:102A60000D4602F0F3F969462046FFF793F818B9CE
:102A70000024204609B030BD04A802F0E7F9204642
:102A800004A9FFF73BFF04460028F1D004A96846DB
:102A900002F0C4FB85ED000AC5ED010A85ED021ABE
:102AA000E7E700001FB500230C4601A9019302933C
:102AB0000393FFF7D1FF08B1039B236004B010BD5F
:102AC00030B585B001AD00230C4629460193029331
:102AD0000393FFF7C1FF034618B195E8030084E8AC
:102AE0000300184605B030BDF8B506460F4615463A
:102AF000FDF770F9044690B13946FDF73BF970B126
:102B000020463946FDF73AF9044640B1FDF762F92F
:102B10003946FDF735F985ED000A2046F8BDFEF788
:102B2000EBFD90F8083343B13046FFF7D5FC04467F
:102B300018B1D6F864312B60EFE7D6F864312B601A
:102B40000024EAE770B52DED048B1646FFF7CCFFA5
:102B5000054670B3FEF7D0FD90F930424CB30BF050
:102B6000FDFEFDF7AFFA012823D9E4B207EE904A43
:102B7000B8EE678A0BF0F2FE90F8F43296ED009A08
:102B8000B02202FB0300D0ED3B8AFEF7A3FF38EE34
:102B9000281A78EEC80A40F2614029EE000A13F0C4
:102BA000E9FEB0EE408AFEF795FFC8EE007AC6ED6A
:102BB000007ABDEC048B284670BD000008B503F018
:102BC00069F9BDE8084003F063B8000010B5044699
:102BD00016F018F850B904F10C0016F013F828B9E3
:102BE00004F11800BDE8104016F00CB8012010BD2B
:102BF00038B500F1280504462846FFF7E7FF28B15D
:102C000020460121BDE83840FFF712BAD4ED107A12
:102C1000B7EE007AF4EEC77AF1EE10FA06D5BFEE01
:102C2000007AF4EEC77AF1EE10FA12DC2046FFF7D4
:102C300059FB2846FFF7CAFF0028E1D1D4ED107AEE
:102C4000B2EE047AF0EEE77AF4EEC77AF1EE10FA1B
:102C5000D6DC38BD10B5044616F026FB2046BDE88C
:102C6000104015F08BBF00002DE9F04F2DED028BC9
:102C7000A3B000270446B0EE408A0A970B970C9742
:102C8000FFF7BEFC13F02AF904F1F00B05465E468F
:102C90004FF0000804F1280A95F8F131022B5FFA91
:102CA00088F1A8BF02238B423AD92846019111F03E
:102CB00055FD019980B310AB13AA284613971497BA
:102CC000159712F03BF89DED100AB5EEC00AF1EE33
:102CD00010FA21DD13A815F0F9FE1CA950468DED60
:102CE0001C0ACDED1D0A8DED1E1A14F06FF816A802
:102CF0008DED160AB0EE480ACDED170A8DED181AC3
:102D000015F0D4FE1CA930468DED1C0ACDED1D0A30
:102D10008DED1E1A15F0EAFE08F101080C36BBE72E
:102D200095F8EC140C2303FB015101F5007150469A
:102D300014F04CF884ED070A94ED450AC4ED080A36
:102D400030EE088A84ED091A84ED458A0BF006FE00
:102D50000646FEF7D1FC90F8093302932046FFF7B0
:102D6000BBFB80B13046FDF7ADF902280BD996F8D0
:102D7000F4226169B02303FB026391F9001093F818
:102D80000201884261DA94ED457ADFEDCC7AB4EE47
:102D9000E77AF1EE10FA62D494ED598AFEF7A0FFBB
:102DA00038B1FDF717F890F84E11FCF7E9FFB0EED7
:102DB000408A236C626BA16A1E93B0EE480A1CA87D
:102DC0001D921C9115F072FE04F5B6710AA88DEDE6
:102DD0000A0ACDED0B0A8DED0C1A15F087FE57F09F
:102DE00073FA0023019084F82C312046FFF774FB1E
:102DF00000286BD096F8F422B02101FB0262D2F8D1
:102E0000E430C4F8303196F8F43201FB0363D3F8B0
:102E1000E830C4F8343157F057FA0123C4F83801C8
:102E2000C4F83C71C4F8407184F84431D4F81831C6
:102E3000002B5ED1019BC4F818310AAB93E8070060
:102E400004F5847484E8070009E006EB0212D2F866
:102E5000A02001920199D4F818218A4204D123B00C
:102E6000BDEC028BBDE8F08F03F5827393E8070099
:102E700094F82C310DF1280C8CE807001BB904F5EF
:102E8000847383E807000123604684F82C3104F53D
:102E9000B67115F0F5FD1CA904F14C008DED1C0A6E
:102EA000CDED1D0A8DED1E1A13F0BEFFB5EEC00A62
:102EB000F1EE10FA8DED1C0AD8BF9FED810ACDED21
:102EC0001D0A8DED1E1A84ED590A8EE794ED457AA0
:102ED000D4ED4F7ADDED0A6AE6EE877ADDED0B6A16
:102EE000C4ED4F7AD4ED507AE7EE267AC4ED507AED
:102EF0009CE7D4ED457A734B0D97F5EEC07AF1EE71
:102F000010FA0E970F93AAD99FED6F7A94F82C318F
:102F100067EE877AB7EE007AC7EE278A1BB9029B65
:102F2000002B00F0C380E36804F584710AA893EDD8
:102F3000008A15F0A5FD28EE888A8DED1C0A1CA8D4
:102F4000B0EE480ACDED1D0A8DED1E1A15F0AEFD4E
:102F500016A90DA88DED160ACDED170A8DED181ADC
:102F600015F0C4FD0DA8FFF775FE0DA815F064FE61
:102F700020B157F0A9F9C4F8780170E701231822AD
:102F8000002116A803937DF035FD182200211CA80E
:102F90007DF030FD9FED4A8A05F20E530DF1700869
:102FA0004FF000094FF0FF37059395F8F131022BF0
:102FB0001A465FFA89F1A8BF02228A4240F296803F
:102FC0008B4204916BD9059B13F80930002B66D016
:102FD000B0EE680A584615F0BDFDDDE90331002B5F
:102FE00066D00C2222AB02FB0933A3F11802049233
:102FF00020465A460693FFF75BFC069B03ED060A44
:10300000049BC3ED010A83ED021A4046FEF744FE1D
:10301000002844D14046FFF71DFE404615F00CFE47
:1030200000283CD10C2303FB09F222AB1344079286
:103030000DA9A3F1300240460492069315F0C6FD97
:10304000069B03ED0C0A049B0DA9C3ED010A83ED59
:10305000021A404615F0A6FD22AB079A03EB89033E
:1030600003ED1A0A16AB981816F01EF97A1C04D054
:10307000B4EEC08AF1EE10FA03DD4FFA89F7B0EE34
:10308000408A22AB03EB870353ED1A7AF5EE407AC0
:10309000F1EE10FAF7EE007A48BFB0EE678A09F158
:1030A000010908F10C080BF10C0B7EE7029B66E7A7
:1030B0009BE8070088E80700A7E700BFCDCC4C3E9F
:1030C00000000000000080BF0AE81C41CDCC4C3E4F
:1030D000CDCC4C3FCDCC4C3D920A06BF920A063F68
:1030E000C2B8B23E728A0E3C5B8218397B1C3FF438
:1030F00040AF84F81C712046FFF7FCF960B1204610
:10310000FFF7EAF9002840F0348122AA0C2303FBE0
:103110000723002243F8282C16AA07EB470895F846
:10312000EB3402EB880895F8F0219A4240F23C819A
:103130002B4493F80C35002B00F0368195F8EC34D5
:1031400095F8F1219A4240F22F812B4493F80E35E5
:10315000002B00F029810C2322AA4146504603FB94
:10316000072713F061FE07ED0C0A47ED0B0A07ED88
:103170000A1A404615F046FD002840F021814046DD
:1031800015F05AFD002840F01B815FED307A94ED78
:10319000387A28EE278A5FED327AA7EE278A04F183
:1031A000B00084ED388A16F07FF8A3685FED377AB7
:1031B00093ED007AB4EEE77AF1EE10FAB0EE408AC1
:1031C00000F102812046B0EE480AFFF74BF9404675
:1031D00015F06CFCA3688DED130ACDED140A8DED8E
:1031E000151A93ED000A13A815F060FC204684ED33
:1031F0001F0AC4ED200A84ED211AFFF7E9F928B16E
:10320000B2EE000A04F17C0015F0A4FC029BB3B3FB
:103210003046FCF757FF012831D996F8F402B02365
:1032200003FB006696ED3B7AF0EE087AB4EEE77A9F
:10323000F1EE10FA23D595F8EC040C2303FB0055AE
:1032400095ED807AF1EE0C7AB4EEE77AF1EE10FAB1
:1032500015DBD4ED1D7A1FED607AF4EEC77AF1EE3E
:1032600010FA0CDD1FED637AF4EEC77AF1EE10FA76
:1032700005D5B6EE000A04F17C0015F06BFC5FED9D
:10328000687AB4EEE78AF1EE10FA22D51FED6B0AE8
:10329000404615F00BFC10A88DED100A94ED450A80
:1032A000CDED110A8DED121A15F000FC13A904F1F1
:1032B000A0008DED130ACDED140A8DED151A15F051
:1032C00015FCD4ED2B7A94ED457A77EE877AC4ED30
:1032D0002B7A94ED2B7AF1EE047AB4EEE77AF1EEE4
:1032E00010FA4FF000053BDB12F0F8FD5FED827A3B
:1032F00094ED2B1A94ED280A21EE271A40F2C530DE
:10330000F1EE410A8DED031ACDED020A13F032FB06
:103310009DED031ADDED020A84ED280A40F2C63065
:1033200094ED290A13F026FB9DED031ADDED020A48
:1033300084ED290A40F2C73094ED2A0A13F01AFBF3
:1033400004F1A00184ED2A0A04F1940015F0CEFBEB
:10335000C4F8A850C4F8A450C4F8A050C4F8AC50A5
:103360001822002104F1F0007DF044FBC4F8145150
:1033700060E5E368F7EE000A93ED000A13F0F8F950
:1033800000283FF4C2AE94ED1C0AB0EEC00A7BF0F8
:103390007FF80C2322AA03FB072353ED0A7A27EEBA
:1033A000800A03ED0A0AB7E60C2322AA03FB0727CB
:1033B000002347F8283C47F82C3C47F8303CD8E637
:1033C0002046FFF715FCD4E5C3ED007AFAE600BF0E
:1033D0002DE9F04D2DED048B9EB0044612F07EFDDC
:1033E00000F59F63D3ED007A90ED7F8AF4EE487A82
:1033F000F1EE10FA48BFB0EE678ADFED5C7AB4EE0A
:10340000E78AF1EE10FA0DDD1822002104F1F00038
:103410007DF0F0FA0023C4F814311EB0BDEC048B2B
:10342000BDE8F08D2046FEF7A1FD2046FEF75AFFCD
:10343000B0EE480A2046FFF717FC2046FFF7D8FBFE
:10344000FEF75AF914AD00F5347204F1280114A8FE
:1034500013F03AFD0FCD04F14C060FC60FCD0FC689
:103460002B68336004F1740204F1780304F17001F5
:1034700004F14C0013F0D6FE94ED1E8AB0EE480A1B
:103480007AF0B0FE84ED6B0AB0EE480A7BF000F8EB
:10349000204684ED6A0AFEF75DFDFEF72DF904F57E
:1034A000C071FDF72FFF56F00FFFD4F8B031C31AEB
:1034B000632BB2D9C4F8B00136F082FC9FED2C9A90
:1034C000054656F009FFD4ED1C7A67EE897A074667
:1034D00017EE900A0E46F9F717F8D4ED1D7A67EE4D
:1034E000897A824617EE900A8B46F9F70DF894ED2B
:1034F0001E0A20EE090A41EC180B13F0A7F9D4F8C4
:10350000740110EE108AF8F7FFFFCDE91201D4F82C
:103510007001F8F7F9FFCDE91001D4F86C01F8F764
:10352000F3FFCDE90E01D4F8E400F8F7EDFFCDE9A3
:103530000C01D4F8E000F8F7E7FFCDE90A014046B6
:10354000F8F7E2FF0B4B01930B4B0093CDE9080119
:103550008DED068BCDE904ABCDE90276074B084A29
:103560000849284636F0B8F957E700BFCDCC4C3EA5
:10357000E02E6542258F09082F8F0908EC8E090877
:10358000F68E0908788D090808B52DED048BB0EE8C
:10359000609AF0EE408A00F011F9B0EE408A89EEB0
:1035A000280A7BF0ABF8DFED0B7A20EE270A7BF0E0
:1035B0003DF8DFED097A38EE278ADFED087A28EE4C
:1035C000278AF7EE007A37EEC00A28EE000ABDEC33
:1035D000048B08BD41D3423E33938843A1D819439D
:1035E000FFF7D2BF08B52DED048B9FED189AF0EED2
:1035F000E07AF4EEC97AF1EE10FAF0EE408AB0EE1D
:10360000608A1ED400F0DAF8DFED117A9FED117AAE
:1036100070EE277A9FED100AE8EEC77A9FED0F7AD9
:1036200027EE800AC8EE007A87EE270AB4EEC90AB0
:10363000F1EE10FA05DBBDEC048BBDE808407BF031
:103640003DB9BDEC048BB7EE000A08BD00000034A4
:1036500033938843F4FDD43B48A18F43CDCC9C3FAA
:10366000427CD0ED257A242101FB020292ED0B0A67
:10367000D2ED090A30EE270AFFF7B4BF38B52DEDB9
:10368000088BDFED21AA9FED21AA9FED21BA054607
:10369000B0EE409AF0EE609AB0EE408A1524013CFC
:1036A000A4B25CB3F0EE490A2846B0EE480AFFF730
:1036B0006BFFF0EE490A70EE698A284638EE2A0A56
:1036C000FFF762FFB0EEE87A70EE697AB4EECA7A7C
:1036D000F1EE10FA77EEE87A10D468EEAA8A40F29A
:1036E000631088EEA70AB0EE4B1A38EE400AF0EEEF
:1036F0004A0A13F03FF9B0EE408AD0E7B0EE480A2C
:10370000BDEC088B38BD00BFCDCCCC3D0AD7233CE7
:1037100000247449002343608360C36003614361F4
:103720008361C361002380F82030704790F8202027
:10373000531CDBB2062B80F8203000EB820288BFDE
:10374000002382ED010A88BF80F820307047000016
:103750004FF0FF3310B543610E4BC0F8A830002383
:10376000044680F8C830A830FFF7D4FF0A4BC4F8ED
:10377000A83004F5867055F003FF084B08491C601B
:10378000204632F0A1FAD4F89030C4F894302046A4
:1037900010BD00BF4C9109085C9109080C5D002028
:1037A000F491090808B5A83037F052FBDFED027A32
:1037B00020EE270A08BD00BF00007A4490ED3C0AC5
:1037C000DFED057AB0EEC07AB4EEE77AF1EE10FAEA
:1037D00048BF90ED3D0A70470000003473B5D0F843
:1037E000A43004460E4663B156F06EFDD4F8A43002
:1037F000C01A42F20F73984203D894ED280A02B01F
:1038000070BD114B1D687DB195F84E112846FCF72F
:10381000B5FA48B195F84E1101AA2846FCF7A4FA6A
:1038200010B19DED010AEAE7242101FB064494ED65
:103830000A0ADFED067AB4EEE70AF1EE10FA58BF95
:10384000B0EE670ADBE700BF045D002000000C4219
:1038500008B561B10378022B02D9064856F002FD83
:103860005A1C027000EB83004160012008BD08462D
:10387000FCE700BF149009082DE9F84305460E4601
:103880009146002400F13C082B78A34211DD00236F
:103890004A46314601200EF0E7FF242363430746E2
:1038A000002158F803000EF0EFFF874204D00134E6
:1038B000EAE70020BDE8F8830120FBE7054B1B6821
:1038C0002BB141694A1C02D0184636F043BA002099
:1038D000704700BFD45F002002290BD8242303FBCC
:1038E000010191F8390030B191F83A0018B191F81E
:1038F0003B007047002070472DE9F047044656F022
:10390000E3FCD4F8F86042F21073861B9E4288BF35
:10391000C4F8F80000274FF0240942F2107A237C03
:10392000FDB2AB421CD929462046FFF7D5FF70B146
:1039300009FB054898ED0D0AD8ED097AD4ED250A62
:1039400030EE270A2046FFF799FE88ED0C0A56450F
:1039500004D909FB0540303032F08EFB0137DEE739
:10396000617C2046FFF73AFF84ED3D0ABDE8F08711
:1039700070B5044686B056F0A7FCD4F89830C31A48
:10398000B3F57A7F05464FD3344B94ED257A1B6807
:10399000DFED336ADB6AD4ED247A93F89C60B0EEF5
:1039A000C76AB4EEE66AF1EE10FA32D5B0EEE76A15
:1039B000B4EEE66AF1EE10FA2BD502A801F046FA51
:1039C00096BBFDF799FE02A9FDF79CFC60B3DDED07
:1039D000037A9FED247AF8EEE77A67EE877AC4EDF2
:1039E000257AC4F89850FDF787FEFDF753FA204674
:1039F000FFF782FF3EF0BAFF0546D4F89400F8F7CF
:103A000083FD194ACDE900010621284638F07EF9E8
:103A10000AE037EE676AF7EE005AB0EEC66AB4EE17
:103A2000E56AF1EE10FA01DC06B070BDB0EEE76AAF
:103A3000B4EEE66AF1EE10FAF6D4002ECFD02046AE
:103A4000903080ED007A32F017FB3EF08FFF074A8E
:103A5000012106B0BDE8704038F058B98425002037
:103A6000000000340AD7233C55900908309009081B
:103A7000F0B52DED048B85B004464FF4537200F57C
:103A8000867103A80FF07CF8D4ED227AD4ED236A76
:103A90009FED796A637C37EEE67A2422B0EEC77A2E
:103AA000B4EEC67AF1EE10FAC1BF9FED747A67EEFC
:103AB000877A9FED737AE6EE877A02FB034300254F
:103AC000C4ED237A93F839602378E9B28B4206D9A2
:103AD00004EB81030135586858F082FDF4E7DFED0F
:103AE000698A9FED698A9FED699A0027237CFDB260
:103AF000AB4264D9242303FB054393F83920002A01
:103B00005BD0D3ED0C7AF4EEE87AF1EE10FA0BDB31
:103B1000F4EE677AF1EE10FA06D6F0EEE77AF4EEFC
:103B2000487AF1EE10FA04DD242303FB05435A6AB8
:103B30001A63242303FB0543D3ED090AD3ED0D7A61
:103B400093F8382070EEA70AA2B993ED0C0A20462C
:103B5000FFF746FDD4ED257A30EE670AB4EE400A51
:103B6000F1EE10FA16D7242303FB0545002385F850
:103B70003A3022E0012A09BFD3ED0C7A93ED0B0A0B
:103B800077EEE00AD4ED3B7A04BF80EE897A87EEC7
:103B9000270AE3E7F0EEC07AF4EE487A2423F1EE48
:103BA00010FA03FB0545E1DC012385F83A30D4ED3A
:103BB000237A37EE800A85ED0B0A013796E7627C9F
:103BC00020461146FFF788FE48B1242101FB02423E
:103BD00092ED0B0AD16904F1A80037F019F994F9B4
:103BE0009C10277C002907DBB94205DACAB21146CE
:103BF0002046FFF771FE68B900226274D5B2AF4269
:103C000009D929462046FFF767FE01320028F5D082
:103C1000657400E062742046FFF7AAFE2046FFF7B5
:103C20004DFE10B1204659F0E3FC637C242505FBD2
:103C3000034393F83930B34216D036F0C1F84FF64B
:103C4000FF7136F087F878B1607C05FB004494F88A
:103C50003930002B14BF00220422019236F0B0F854
:103C6000019A122136F008F803A80EF0ABFF05B058
:103C7000BDEC048BF0BD00BF0AD7233C0AD7A33CA0
:103C800048E17A3F00000034FFFF7F7F00201946A3
:103C90002DE9F04F0446007C0F4687B004F13A034B
:103CA00000220121D5B2A84203F1240305D903F86B
:103CB000231C03F8241C0132F4E76F4B1E68F06AE2
:103CC00003685B68984740B13EF050FE6B4A06219E
:103CD00007B0BDE8F04F38F019B83EF047FE684A2B
:103CE000062138F013F8002303A904F18800039398
:103CF00032F080FD0A2556F0E7FA80462046FFF7AD
:103D0000B7FE56F0E1FAA0EB0800B0F5FA7F02D951
:103D10005C4801F07FF8B06A03680A215B68984745
:103D2000617C2046FFF7D8FD0028E7D0B06A036821
:103D300064215B68013D984715F0FF05DBD1524BCC
:103D400005951B888DF80650CDE90355ADF8043074
:103D5000052556F0B9FA80462046FFF789FE56F051
:103D6000B3FAA0EB0800B0F5FA7FD1D8617C204609
:103D7000FFF7B2FD0028EFD094F810B00DF10C0859
:103D8000A14601AA4FF0000A5FFA8AF18B4516D9C5
:103D90002046FFF7A1FD50B1D8ED007A99ED097AE0
:103DA000137877EE877A0133C8ED007A13700AF141
:103DB000010A08F1040809F124090132E4E7B06AB4
:103DC000036864215B68013D984715F0FF05C0D189
:103DD000A9464FF02408237C5FFA89F6B34226D91E
:103DE00006AB334413F8143C33B908FB064686F897
:103DF0003B3009F10109EEE7002FFAD007EE903AC7
:103E000006AA02EB8602F8EEE77A12ED030AD4ED79
:103E1000250A204680EE270AFFF730FC08FB064003
:103E200002A930308DED020A32F0E4FCE1E7617C5A
:103E3000DFF85C902046FFF7D1FC002684ED3D0AB8
:103E40004FF02408237CF7B2BB420FD908FB07438D
:103E500093F83B3043B13EF089FD7B1C4A46062176
:103E600037F054FF0135EDB20136EBE70DB90748E5
:103E70004FE707B0BDE8F08F842500207090090857
:103E80009B900908B1900908084C0908ED900908B1
:103E9000CB90090808B5037C022B02D9034856F0E1
:103EA000E1F95A1C0274184608BD00BF0C910908BC
:103EB00038B5057C02460024E1B28D4206D9104691
:103EC000FFF70AFD01340028F6D138BD281E18BFBF
:103ED0000120FAE770B50D4609780729044606D88F
:103EE000027E437E22B901228A401343437670BD8D
:103EF000002BFCD000262278F3B29A42F7D904EBCB
:103F00008303294658680368DB6898470136F2E75F
:103F100037B50D460192FFF7CBFF0199044630B942
:103F20000448054B00682A46C06A0FF007F820468F
:103F300003B030BD842500207BD30A08014B1868EC
:103F4000704700BF0C5D002010B50446006810B13A
:103F500003685B689847204610BD000013B5002237
:103F60000B680A6001A9019358F08AFE044601A873
:103F7000FFF7EAFF204602B010BD000013B5002293
:103F80000B680A60022201A901935AF065F8044601
:103F900001A8FFF7D9FF204602B010BD13B50022DB
:103FA0000B680A60012201A901935AF055F80446F2
:103FB00001A8FFF7C9FF204602B010BD13B50022CB
:103FC0000B680A6001A901935AF046F8044601A85B
:103FD000FFF7BAFF204602B010BD000010B504463E
:103FE000006810B103685B689847204610BD000068
:103FF0002DE9F04F8FB0D0F800310893344B354D98
:104000001B6805930446586803689B68984794F9B1
:104010009D300690002BA2BF012606FA03F30693FB
:1040200005F1D80A2B68089A1A420BD000274FF0E6
:10403000010BB946069A0BFA07F3134206D1013772
:10404000202FF7D10C355545ECD12DE0F9B26B6836
:104050002A7A099120460793FFF70EFC09998046BA
:1040600028B3CDE90A990B9B0D930DA9079BCDE9C8
:104070000B992046984701462046FFF7E9FB0DA81B
:10408000FFF762FF0CA8FFF75FFF0BA8FFF7A6FF83
:10409000B8F1000F02D00AA8FFF7A0FF2378032B86
:1040A00002D0237C032BCAD10FB0BDE8F08F059B53
:1040B000586804220368CDE90182074A00921B6810
:1040C0000A461E4601462B7A0BA8B047CBE700BF35
:1040D00084250020E4920908801A060070B5D0ED0E
:1040E000247A9FED657AF0EEE77AF4EEC77A012341
:1040F000F1EE10FA8AB00446037609D4903000231A
:1041000009A90590099332F075FB059831F0B4FFC9
:104110000026E6632666C4F884607622314620468F
:10412000FFF7AAFB054600283FD0CDE90666079AAF
:104130000992002309A92046CDE9073358F062F817
:1041400001462046FFF784FB09A8FFF7FDFE08A8FB
:10415000FFF7FAFE07A8FFF741FF15B106A8FFF722
:104160003DFF2378032B59D0237C032B56D094F9A1
:104170009D10002928DA2046FFF73AFFD4F80031D5
:10418000DA045DD40025637EEB40DB07EAB25DD440
:104190000135082DF7D1237823B1237C13B163684F
:1041A000002B3BD1354800F035FE354B1B68596874
:1041B00004220B68CDE90102324A00921E680246D1
:1041C000762307A8B047B2E77722C9B22046FFF7A7
:1041D00053FB054620B30023CDE90633079B099323
:1041E000002209A92046CDE9072259F035FF0146F2
:1041F0002046FFF72DFB09A8FFF7A6FE08A8FFF74A
:10420000A3FE07A8FFF7EAFE15B106A8FFF7E6FE32
:104210002378032B02D0237C032BACD10AB070BDD2
:10422000174B1B68596804220B68CDE90102154A37
:1042300000921E6894F89D20772307A8B047CDE729
:10424000637E002B9ED1012363769BE73820059285
:1042500001F098F8064618B1059A214659F09AFFE0
:1042600031462046FFF7F4FA2378032BD6D0237C7F
:10427000032B8DD1D2E700BF000000342091090844
:1042800084250020801A060090F86035934207D9F3
:1042900002F5A77250F8220010B103689B6A184714
:1042A000002070472DE9F34105466E4686E80C0074
:1042B000134B45F8043B04460F4600F5C8782846E2
:1042C0002C3500F0CFFCA845F9D196E8030004F2A4
:1042D0006453C4F85C7583E80300089BC4F86C352C
:1042E0000849204631F0F0FC074B1A6812B1074824
:1042F00055F0B8FF20461C6002B0BDE8F08100BF59
:10430000EC950908B4940908105D0020F893090899
:104310002DE9F041A2B00C4607A930F01DFD0028A0
:1043200055D000210D220CA80591ADF818100B9165
:104330007CF060FB2B4B611C1F68C9B20BAD0129DF
:10434000F86A0A9546D1284B062205A90EF0F6FD1B
:10435000264B019305AB0093002411222946244BE0
:10436000F86A8DF819400EF0E9FD04AA0DF10F016D
:1043700028468DF83C40049432F01AF938B31D49B0
:10438000DFF86C80482210A87CF0EAFA062610AC10
:104390002268531E049AC2F3513202EB831223792E
:1043A0008DF82430A368019305AB0093089243462F
:1043B00011222946F86A0EF0C1FD0021B7EE000A6D
:1043C00007A830F079FE013E04F10C04E0D122B0E0
:1043D000BDE8F0810091084B062205A90EF0AEFD64
:1043E000B6E700BF84250020B18209082994090896
:1043F000239409080C4C09081C9409082DE9F04F76
:1044000090F8606585B00446002E59D17F2380F86E
:1044100070350DF10F0104232A308DF80F3032F082
:1044200025FA04F5C87504F5A768271D5FFA86FA12
:104430001822FF2128467CF0DDFA85F85FA097F965
:104440002690B9F10A0F5CD03DDCB9F1040F0FDC06
:10445000B9F1020F0FDD442000F094FF834620B134
:104460003B462A4621465AF0FBF9C8F800B002E064
:10447000B9F1090F39D0D8F8000050B1696EC5F80C
:10448000609031B12C4B43F8261031F02BFE31F007
:1044900021FE58F8040B0AF101095FFA89F940B1CD
:1044A00003689B68984784F8609551462046FFF75B
:1044B0002FFF0136092E05F1680507F12C07B5D14C
:1044C00005B0BDE8F08FB9F1150F28D0B9F1190F7B
:1044D000D1D1482000F056FF83460028C5D03B4686
:1044E0002A4621465BF090FBBFE7382000F04AFFE8
:1044F00083460028B9D03B462A4621465AF016FE8C
:10450000B3E7302000F03EFF83460028ADD0CDF861
:1045100000A03B462A4621465BF0F8FAA5E7782042
:1045200000F030FF834600289FD03B462A462146B4
:104530005AF064FE99E700BF145D002090F86035E2
:104540008B4283BF682303FB010090F8DD0100204C
:104550007047000090F860358B4283BF682303FBEF
:10456000010090ED6A0A9FED010A7047000000000B
:1045700090F860358B4206D901F5A77150F82100FB
:1045800008B15AF00DBB9FED010A70470000000012
:1045900010B490F860458C420A4614D901F5A7740E
:1045A00050F824407CB1E468246A640603D55DF8C1
:1045B000044BFFF7DDBF682101FB020393ED6A0A9C
:1045C0005DF8044B70479FED010AF9E70000000019
:1045D00090F860358B420BD901F5A77150F8210096
:1045E00038B1C3681B6A1A4214BF0120002070470B
:1045F0000020704770B590F86035934204460E462F
:10460000154601D8002070BD02F5A77350F82300AD
:104610000028F7D003689B6998470028F2D06822E9
:1046200002FB0544D4F8AC313360ECE770B590F888
:104630006035934204460E46154601D8002070BDF1
:1046400002F5A77350F823000028F7D003689B6990
:1046500098470028F2D0682202FB0544D4ED6C7A1A
:10466000F4EE677AF1EE10FAE8D6C6ED007AE6E7E6
:1046700070B590F86035934204460E46154601D851
:10468000002070BD02F5A77350F823000028F7D072
:1046900003685B6998470028F2D0682202FB054452
:1046A000D4F8B4313360ECE790F8603593420ED91A
:1046B00002F5A77350F823305BB1682303FB0202B5
:1046C00092F8EC0130B1D2F8E8310B60704700206D
:1046D000704718467047000008299DBF2C2303FB34
:1046E00001004068002070472DE9F04F4B4B2DED45
:1046F000028B1B68DB6A93F89C3089B00446002B60
:1047000000F08680DFF82CB19FED458A4FF000095C
:1047100094F860355FFA89F5AB4279D905F5A7734E
:1047200054F8230000285DD003685B6B984768232A
:1047300003FB0543074693F8DC31834252D203283A
:1047400061D8DFE800F04F025259364E4FF00008B2
:104750003EF00CF994F86025AA4284BF682202FB5F
:1047600005424FF0680105F1010301FB05458CBFCF
:10477000D2F8A82118EE102A8246D5F8B001CDE96A
:104780000632F7F7C1FE079ACDE904011046F7F7A4
:10479000BBFE069B0096CDE902015A460421504615
:1047A00037F0B4FA0123204A84F8713585F8DC71BA
:1047B000D372D4F86C354BB3002255B25957481C0C
:1047C00003D0414502F10102F7D194F97035AB42B3
:1047D00008DBD4F86835D4F864054246314698477A
:1047E00084F8705509F1010992E72C2303FB054376
:1047F0000E4E93F92D80ABE72C2303FB05430C4EA3
:1048000093F92E80A4E70026B046A1E71D46DCE719
:1048100009B0BDEC028BBDE8F08F00BF84250020FD
:10482000000000003D9409088D5D0020B2DF0A08F9
:10483000349409084C94090890F860358B4207D9E4
:1048400001F5A77150F8210010B10368DB69184722
:104850000020704708299CBF682303FB010000F576
:10486000C870704790F86035934207D902F5A77277
:1048700050F8220010B103685B6A184700207047A7
:1048800090F860358B420DD901F5A77350F82330AD
:1048900043B1682303FB0101012081ED730A81F814
:1048A000C801704700207047F8B5002402460E4644
:1048B00025462C2792F86035E1B28B4210D901F5DC
:1048C000A77352F823304BB107FB01239B689E422C
:1048D00004D11046FFF7D4FF2843C5B20134E9E7FD
:1048E0002846F8BD2DE9F04F002493B005460E464A
:1048F000174621462F2206A8059405F5A7697CF0E6
:1049000079F805F12A0A4FF02C0B05F5F8730BFB2B
:1049100004F259F8040B1AF90210E5B230B951B992
:104920000134092CF3D14FF0010813E068226243EF
:104930009A58914212D01548154B006801930135E1
:10494000EDB20095134BC06A324639460EF0F6FAC6
:104950004FF00008404613B0BDE8F08F05A93322A0
:1049600003935AF0FFF9039B804605A90028D7D18D
:10497000064801910135EDB200680095054BC06A0B
:10498000324639460EF0DAFAE4E700BF842500200B
:1049900082940908749409082DE9F04FDFF880909B
:1049A000DFF880A0DFF880B08DB00646002796F8CB
:1049B0006035FCB2A3422ED9682505FB046595F845
:1049C000E43133B395F8E51119BB4FF0010820220B
:1049D000444404A889F819807CF00CF807EE904A4A
:1049E0004AF21043F8EEE77A03AA4C21ADF82830DA
:1049F00050462423CDED037A39F09EF83DF0B6FF02
:104A00009BF80030054A0094042137F07FF985F8BF
:104A1000E5810137CBE70DB0BDE8F08F8C94090834
:104A20008D5D002061600020C52200202DE9F04F3F
:104A30002F4B1E6885B0044646B1D0F85C15304651
:104A400035F088F910B1304634F0D6F855F03CFC1A
:104A50004FF0000801904FF02C0A4FF0680B94F8CB
:104A600060355FFA88F5AB4239D904EB8507D7F892
:104A7000380588B30AFB05430BFB054993F92A2047
:104A8000D9F8F0118A4227D132B30268D268904730
:104A9000D7F838050268126B904799F8DD2112B1FA
:104AA000019BC9F8E031BEB1D4F85C15304635F051
:104AB00051F988B155F010FCCDE9021002460B46C1
:104AC000D7F8380529465AF093FEDDE90232D7F8C7
:104AD000380529465AF00AFF08F10108BFE72046C9
:104AE000FFF702FE204605B0BDE8F04FFFF754BFC8
:104AF000D45F00202DE9F0474FF000082DED028B28
:104B000004468946B0EE408A474601264FF0680ABF
:104B100094F860355FFA88F5AB421AD929FA05F3A3
:104B2000DB070AD505F5A77354F8230078B10368AD
:104B3000B0EE480A9B6B984706400AFB054508F112
:104B4000010895F8DC319F4238BF1F46E0E7064672
:104B5000F3E727B97F23A4F87035034BDF72BDEC70
:104B6000028B3046BDE8F0878D5D002090F86035FF
:104B70008B4207D901F5A77150F8210010B10368E5
:104B8000DB6B1847002070470B46114690F86025F4
:104B90009A4207D903F5A77350F8230010B10368B0
:104BA0001B6C18477047000070B504460E46002580
:104BB00094F86035E9B28B4205D932462046FFF7BA
:104BC000E3FF0135F4E770BD2DE9F84390F8605537
:104BD0000246002400F12A062C2700F5F8784FF051
:104BE0006809E1B28D420FD907FB04F309FB04F019
:104BF000F35658F80000834209D11BB11046FFF765
:104C00009DFC10B10134ECE70120BDE8F8830020E1
:104C1000FBE7000010B590F860258A42044617D9DA
:104C2000682202FB010393F8DC31022B03D004D984
:104C3000032B18BF0023184610BDFFF797FF48B994
:104C40002046FFF7C1FF00280CBF06230123F2E72F
:104C50000023F0E70623EEE7014B1868704700BF1A
:104C6000105D002010B50349044631F02DF82046B0
:104C700010BD00BF6C96090810B50446203047F0FF
:104C80008DFF044B04491C60204631F01DF820467E
:104C900010BD00BF385D0020F0970908F7B5B7EEEA
:104CA000000A00220221044630F01EFB20465AF082
:104CB000FBFF47F0EDFF144B1D680646E86A0368EA
:104CC0005B6A98470B46022102460091304647F046
:104CD0007BFFB4F94A60002E14DDEF6A3B6838466A
:104CE0005B68B4B2984728B197F84D3013B1C92E1C
:104CF000A8BFC824A86A03685B68214603B0BDE862
:104D0000F040184703B0F0BD8425002010B50446DC
:104D10005AF098FF2046BDE810405AF0C3BF00008B
:104D20002DE98048284BDFF8A490DFF8A4A0DFF835
:104D3000A4B01446012293B005460E461A704FF0F7
:104D4000000855F0C1FAD9F800300393A0EB08022F
:104D500041F287339A4207461FD9CDE9005603989E
:104D60005346342205A9C06A0EF0E8F8214605A88A
:104D7000049454F083FCCDE9005603985B4634223A
:104D800005A9C06A0EF0DAF804943DF0EFFD049B2B
:104D900005AA022136F0A0FFB8463DF0E7FD3DF040
:104DA00081F83DF0E3FD3EF045FF0A2105A80DF036
:104DB000CDFE039B986A036805215B68984705A8A8
:104DC0000DF0D0FEBDE700BF3C5D00208425002033
:104DD0006C97090821F80A080FB400B595B016AA17
:104DE000002152F8043B039205A83C220193049150
:104DF0007BF000FE054A019B402104A854F0E6FB2D
:104E0000039A034804A9FFF78BFF00BF74970908B2
:104E10008A9709080FB407B504AA034852F8041B7F
:104E20000192FFF77DFF00BF9C97090808B5044970
:104E300010227BF085FDB0FA80F0400908BD00BF6C
:104E4000405D0020102200217BF0D4BD10B5044647
:104E5000FFF7F8FF204610BD0378416023F00D03F3
:104E6000022A037008D0032A0AD0012A03D1DBB238
:104E700043F0010303707047037843F00803F9E738
:104E8000037823F0050343F00503F3E773B5044605
:104E90000E4615460193FFF7D5FF2046C4E902658B
:104EA000069A0199FFF7D8FF02B070BD007842075B
:104EB00004D4030704D400F00100704703207047B6
:104EC00002207047F0B585B005461646FFF7EEFFA5
:104ED00088420F4605D16B6833600124204605B037
:104EE000F0BD032801D10024F8E70329FBD00128F5
:104EF0000BD0022816D018BB6D68012F22D0022FCC
:104F00002ED0002FEFD13560E7E7FCF7F5FB90F8E6
:104F10007C32DB07E7D56D68FCF7EEFBD0F870322A
:104F20001D44EAE76846FFF78DFFFCF7E5FB69469D
:104F3000FCF7E8F904460028D0D06D68019BEFE744
:104F40000025DAE7FCF7D8FB90F87C4214F0010466
:104F5000C9D0FCF7D1FBD0F87032ED1A3560BDE74F
:104F60006846FFF76FFFFCF7C7FB6946FCF7CAF915
:104F700004460028B2D0019BEFE7000073B501AAF8
:104F800005460E46FFF79EFF044620B101993246C2
:104F90002846FFF761FF204602B070BD13B51446E6
:104FA00001AAFFF78FFF48B1DDED017A9FED047A8A
:104FB000F8EEE77A67EE877AC4ED007A02B010BDAA
:104FC0000AD7233C07EE900A9FED090AF8EEE77A2C
:104FD00008B527EE800A79F005F9DFED067AB4EE20
:104FE000E70AF1EE10FAD8BFB0EE670A08BD00BFBD
:104FF00050E0EF300AD7233C10B50446806811F02A
:105000007BFE20B1E068BDE8104011F089BE10BD04
:105010000D4B83424FF000038B4106DA00F125501F
:1050200000F5311000F5E0507047084B98424FF002
:10503000FF3371EB0303BEBF00F1564000F51300D0
:1050400000F52440704700BF00D2496B002EB69493
:1050500090EA010F01D4401A7047C317401A63EB5E
:10506000E1710D4B83424FF000038B4106DA00F1F2
:10507000255000F5311000F5E0507047074B98427D
:105080004FF0FF3371EB0303BEBF00F1564000F554
:10509000130000F52440704700D2496B002EB694EF
:1050A00070B52DED028B84B0044668460D46FFF7BF
:1050B000C9FEFCF721FB6946FCF724F9064608B354
:1050C000A368029ADFED128A03999B1A07EE903AC1
:1050D000F8EEE77A67EEA87AC5ED007AE068FFF7A8
:1050E000B7FF08EE100AA068024402EBD272B8EED5
:1050F000C88A5010FFF766FF28EE288A28EE000ABB
:1051000085ED010A304604B0BDEC028B70BD00BFD6
:10511000F67C8E3F37B500230C4601AA02210546D6
:105120000193FFF7CFFE10B9002003B030BD214638
:105130002846FFF7B5FF0028F6D0DDED017AF8EE3E
:10514000E77AC4ED027AF0E738B52DED028B0C4614
:105150000246C168E068FFF77BFF9568A46808EE27
:10516000100A601900EBD0704010641BFFF72AFF93
:1051700007EE904AF8EEE77AF8EEC80A87EE807AF2
:10518000BDEEC70A10EE103A5B4200EE103AB8EEE0
:10519000C00A79F049FADFED087A30EE270ABDEC53
:1051A000028BB5EEC00AF1EE10FA44BFDFED037AD0
:1051B00030EE270A38BD00BFDB0FC93FDB0FC94007
:1051C00030B52DED028B0B4685B08C68D0E90251CD
:1051D000D868FFF73DFF08EE100A601900EBD070A9
:1051E0004010FFF7EFFE641B07EE904AF0EE400A16
:1051F000B8EEC88A9FED060AF8EEE77A28EE008A34
:1052000027EE800A68EE200A05B0BDEC028B30BDA7
:105210008262363C82B002B0FFF7D2BFF0B52DED0E
:10522000028B0D4689B08C680646D0E90271E868A9
:10523000FFF70EFF08EE100AE01900EBD0704010E7
:10524000FFF7C0FE73686A689FED0E1A9B1A07EE9F
:10525000903AE41BB8EEE77AF0EE400A07EE904A87
:105260009FED090AB8EEC88AF8EEE77A28EE008AC0
:1052700027EE011A27EE800A68EE200A09B0BDEC7D
:10528000028BF0BD0AD7233C8262363C10B52DED6F
:10529000028B84688A680B46111B08EE901AC1685D
:1052A000D868FFF7D5FE224402EBD27208EE100A4E
:1052B0005010FFF787FEB8EEC88AF8EEE88A28EEAD
:1052C000000A20EE000AA8EEA80A79F0F7FABDEC71
:1052D000028BDFED027A20EE270A10BD8262363C97
:1052E000094B984206DDC0F1D64000F5930000F569
:1052F000A4407047054B9842BEBFC0F1144000F572
:10530000360000F53850704700E9A43500175BCA35
:10531000F8B52DED028BDFED148A076820EE280A20
:105320000646FDEEC07A0D4617EE904A04EBD470A7
:1053300007EB6000B0EE608AFFF744FE28EE288A93
:105340003819C8EE007AFFF7CBFF306017EE900AED
:10535000F7F704FE2B68C01841EBE371FFF758FE26
:10536000BDEC028B2860F8BD02AAB34200F10C012B
:105370000830FFF7CDBF00000148FFF763BD00BF55
:10538000405D00200121884238BF084677F0C4B84C
:10539000FFF7F8BF08B177F0C3B87047FFF7FABF5F
:1053A00000214FF0FF3310B5002203630446016073
:1053B0000171C0F80510417280F8251000F13C031E
:1053C00000F50B70D9709A60DA601A615A619A61BF
:1053D000DA611A625A629A62DA631A645A649A64E7
:1053E000DA641A655A659A65DA65DA661A675A6781
:1053F0007C339842E6D1214604F5167007F026FC6E
:10540000044B1A6822B904491C60204630F05CFC49
:10541000204610BD505D0020449A090873B5D0F8AD
:105420003C3201919942044613D0D0F8403299425F
:1054300018D0D0F844328B4216D102200AE0D4F8BA
:10544000343253B3D4F838324BB34FF0030002B0C8
:1054500070BD002094F822308342F8D8431C84F8B1
:105460002230F4E70120F5E7D0F83062002EE6D1D3
:1054700094F841233546B6009AB1A319C3F8301207
:10548000A319019AC3F83C2294F82230AB429CBF86
:105490006B1C84F822302846D9E70126E8E702266B
:1054A000E6E704F50C7001A9304431F0B1FAE7E702
:1054B00038B504460D4631F021FA291D201D31F082
:1054C0001DFA05F1080104F1080031F0F1FA05F1C7
:1054D000140104F1140031F0EBFA05F1200104F19C
:1054E000200031F0E5FA05F12C0104F12C0031F037
:1054F00099F905F1300104F1300031F0A1FA05F11C
:105500003C0104F13C0031F0D3FAAB6BA3636B6B4D
:10551000636338BD2DE9F043A1B00023002500F1FD
:105520003C0706468DF807500393049305930693B2
:105530000793089309930A930B9310931193129373
:105540001393149315931693179318931C931D9309
:105550001E9300F50F78B94658F8043BF3B1F26E8C
:10556000934223D0D6F8E820934221D0D6F8642184
:10557000934213D10221EBB299420FD0C1EB4111FA
:1055800009EB8104214601A8FFF792FF3946204626
:10559000FFF78EFF01A93846FFF78AFF0135032D7B
:1055A00007F17C07D8D121B0BDE8F0830021E2E704
:1055B0000121E0E72DE9F04706460F4615468046F3
:1055C00004464FF0000A39463046FFF727FF626F66
:1055D000BA425FFA8AF90ED1C3B2022B0BD87C22F1
:1055E00002FB0A66012086F83E0086F83F3085F807
:1055F0000090BDE8F0870AF1010ABAF1030F04F147
:105600007C04E0D1002439463046FFF707FFD8F884
:105610006C205FFA84F912B9C3B2022B22D901348B
:10562000032C08F17C08EED100244FF07C0906F130
:105630003E0A39463046FFF7F1FE034609FB04F007
:105640005FFA84F81AF8002012B9DBB2022B12D9E3
:105650000134032CEDD196F82300042814D91948FD
:1056600054F000FE7C2000FB0464012084F83E001E
:1056700084F83F30BBE70644012086F83E0086F8F8
:105680003F3085F80080B4E706F54371002251F8F9
:10569000043BBB42D4B208D1A04202D8631C86F8B6
:1056A000233003342C700020A3E73BB9421C06EBE7
:1056B000800086F82320C0F80C73F2E70132052A37
:1056C000E5D1F0E780980908C9B200EB8101D1F873
:1056D0003C3253B1026F93420AD0D0F8EC2093428F
:1056E00008D0D0F86821934206D04FF003007047ED
:1056F00000207047012070470220704759B190F890
:105700002030032B07D05A1C80F8202000EB8300A8
:105710004161012070470020704700002DE9F843E7
:105720000F469146044600F5BA7894F83E5035B9D4
:105730007C344445F9D100252846BDE8F883002390
:105740004A46394601200DF08FF800210646E06EEA
:105750000DF09AF88642EBD1EEE700002DE9F04318
:10576000DFF87C8085B0044600F50F7600257C27A5
:10577000B14656F80C3CD9F800209342E9B206F144
:10578000040619D1C3B12046FFF79EFFC0B207FB44
:10579000004090F83E307BB903A9A9F10C000393B7
:1057A00031F036F93DF0E2F856F8043C00934246F9
:1057B0002B46012136F0AAFA0135032DD8D104F188
:1057C0006C0504F5F074296821B9AB6813B128465B
:1057D0002FF0DEFA7C35A542F5D105B0BDE8F083A7
:1057E0009C98090838B504461546FFF76DFFC0B20E
:1057F000022808D87C2303FB004029465030BDE82E
:10580000384031F045B938BD38B504461546FFF784
:105810005BFFC0B2022808D87C2303FB0040294666
:105820005C30BDE8384031F033B938BD37B50D468E
:1058300004468DED010AFFF747FF022D07D8C0B2DD
:105840007C2303FB004001A9683030F0D3FF03B094
:1058500030BD000038B50546FFF736FFC4B2022C54
:1058600013D8C4EB4414A4003C3504F108002844C8
:1058700000212FF08DFA04F1340104F130002944A5
:105880002844BDE8384031F0C3B838BD70B505468E
:105890000E461446FFF718FFC3B2022B0DD87C202A
:1058A00000FB035394E80700443383E807003146C4
:1058B0002846BDE87040FFF7CDBF70BD37B5044640
:1058C0001546FFF701FFC0B2022809D87C2303FB6D
:1058D00000400DF1070140308DF8075031F00EF80F
:1058E00003B030BD10B500210446FFF7B3FF2046DA
:1058F0000121FFF7AFFF20460221BDE81040FFF76E
:10590000A9BF00001FB590F92C30044623B390F9CD
:1059100021300BB36846FFF799FAFBF7EDFE6946B5
:10592000FBF7ACFCC0B1DDED037A9FED0C0AF8EE9D
:10593000E70ADDED027AF8EEE77A0123C0EE800A8D
:1059400084F83D3387EE800A07F0C2FBDFED047A6E
:1059500020EE270A84ED0A0A04B010BD8096184B89
:1059600035FA8E3C024690F9210058B192F8400376
:1059700040B1114491F92C0220B192F9240003386E
:1059800018BF01207047000038B590F82230054656
:105990005BB100242346E1B22846FFF7E3FF08B1DC
:1059A0000133DBB20134032CF5D1184638BD0000B9
:1059B00090ED0A0A7047000038B50C46D1ED066A32
:1059C00011460546FFF780FEC3B27C2000FB03535F
:1059D000D4ED087AD3ED260A94ED076AD3ED255A63
:1059E00093ED245A26EE600A67EEA00AA5EEA70AF8
:1059F000F0EE607AE5EE867AB7EE007AA6EEE67A09
:105A000067EEE60AB1EE400AE5EE070A78F00CFE12
:105A10009FED071ADFED070A40F61C0010F0AAFF01
:105A2000D5ED0A7ABDE8384030EE270A10F08EBF77
:105A3000DB0F4940DB0F49C02DE9F04190F82230DF
:105A40008B4204460D4602D20020BDE8F081FFF7EC
:105A50003BFEC0B204F13C06C0EB401006EB8000F8
:105A6000083013F021FCDFED157AB0EEC00AB4EE79
:105A7000E70AF1EE10FAE7D429462046FFF724FEA4
:105A8000C5B27C2000FB05473B6F002BDCD0032D0B
:105A9000DAD000FB05603030D7F86C8030F0EAF9DE
:105AA000D7E91B32934201D1984505D07C2000FBF9
:105AB0000544C4F86C80C7E70120C6E70000003445
:105AC0002DE9F74F04460E46174600F50F7A4FF0C2
:105AD000000B5AF8049B5FFA8BF8B9F1000F26D03F
:105AE00041462046FFF73EFF08B341462046FFF7F8
:105AF000EBFD7C23C0B203FB004090F83E505DB943
:105B000008F101031B4ADBB23946304653F05EFD13
:105B1000284603B0BDE8F08F5AF8102C914506D006
:105B2000154A3946304653F051FD0025F0E70BF198
:105B3000010BBBF1030FCCD14FF0000894F82230D9
:105B40005FFA88F18B420DD920460191FFF774FF6F
:105B5000054620B901992046FFF704FF20B908F156
:105B60000108EBE70125D3E7044A3946304653F0F4
:105B70002DFDCDE7C4980908D9980908FE980908B1
:105B80002DE9F0412DED048B90F842139FED348AFE
:105B9000DFED348A9FED349A82B00646FFF794FD1C
:105BA00006F13C07C5B27C2000FB057554354FF06B
:105BB000000896F822205FFA88F39A424ED91946D7
:105BC0003046FFF7CFFE10B908F10108F1E719469A
:105BD0003046FFF779FDC4B27C2000FB0474D4ED9D
:105BE000157AF0EEE77AF4EEC87AF1EE10FA04F1E5
:105BF00054040ED5D4ED017AF0EEE77AF4EEC87ACB
:105C0000F1EE10FA05D5002002B0BDEC048BBDE822
:105C1000F0812946204613F05FFBB4EEE80AF1EE6E
:105C200010FAF0DC2946204612F06EFEB4EEC90AE6
:105C3000F1EE10FAE7DC2146284612F0A1FD684695
:105C40008DED000ACDED010A12F04AFEDFED077A74
:105C5000B4EEE70AF1EE10FAB6DDD4E70120D3E79F
:105C600000000034DB0FC93F920A863F0000484322
:105C7000022910B5044608D8FFF726FD7C23C0B2E0
:105C800003FB004494F83D0010BD0020FCE7000039
:105C900013B590F8421301910446FFF7E9FF30B1C4
:105CA0000199204602B0BDE81040FFF75BBE02B08C
:105CB00010BD0000F7B590F921500446002D73D0B7
:105CC00090F84053002D6FD090F84213FFF7D0FFAB
:105CD00094F83D33064613B92046FFF713FE00251E
:105CE00094F82020EBB29A4207D904EB83030135E4
:105CF000586903689B689847F2E754F0E5FA002773
:105D0000224604F5BA7140F2F315D2F89C30C31A5A
:105D1000AB428CBF0023012382F83D307C3291429C
:105D200047EA0307F1D194F92430032B07D194F803
:105D30003C33002B3BD0D4F83803002849D167B15D
:105D4000236B013309D034F03BF8216B34F002F8B7
:105D500018B134F035F833F063F894F92C32002B95
:105D60003AD194F92D32CBBB94F92E3213B10223E0
:105D700084F8423394F842132046FFF779FF8642B5
:105D8000054611D034F01CF84FF6FF7133F0E2FFF6
:105D900050B1002D14BF00220422019234F010F8FB
:105DA000019A032133F068FF284603B0F0BD0123B8
:105DB00084F83C330420FFF7E5FA054610B121468C
:105DC00006F0DAFF94F92430C4F83853032BB2D02C
:105DD000B5E706F0DFFFB2E70023C9E70123C7E715
:105DE00038B590F921300446D3B190F84053BDB195
:105DF000FFF76AFCC0B2022812D87C2303FB0044E0
:105E0000D4ED1A7A9FED087AF4EEC77AF1EE10FA23
:105E100006D4B7EE087AF4EEC77AF1EE10FA00DD98
:105E20000025284638BD00BFABAA2A3F70B5D0F880
:105E3000085315F4003504460E460DD190F8403352
:105E40005BB90A78072A07D8012303FA02F290F80F
:105E50003F33134380F83F3370BD94F82020EBB2FA
:105E60009A42F9D904EB8303314658690368DB6829
:105E700098470135F1E7000038B505466C242B59E9
:105E80001BB1002128192EF083FF7C34B4F5F07F7C
:105E9000F5D138BD014B1868704700BF505D002038
:105EA0002DE9F04FB24BD3F800800446D8F8040037
:105EB00003688DB09B689847002507464FF001099D
:105EC00009FA05F33B4240F092820135202DF7D1CB
:105ED000D8F804000368DB689847002507464FF0B0
:105EE000010909FA05F33B4240F0C3820135202D38
:105EF000F7D1D8F8040003689B6898470025074647
:105F00004FF0010909FA05F33B4240F0F1820135F7
:105F1000202DF7D1D8F8040003689B689847002526
:105F200007464FF0010909FA05F33B4240F01C8394
:105F30000135202DF7D1D8F80400DFF840B203680E
:105F40009B68984700250490049A0123AB401342B4
:105F500040F046830135202DF6D1D8F80400DFF853
:105F60001CB20368DB68984700250490049A01235B
:105F7000AB40134240F005840135202DF6D1D8F80E
:105F800004000368DB689847002507464FF00109C5
:105F900009FA05F33B4240F0BF840135202DF7D1CB
:105FA000D8F804000368DB689847002507464FF0DF
:105FB000010909FA05F33B4240F0ED840135202D3B
:105FC000F7D1D8F8040003689B6898470025074676
:105FD0004FF0010909FA05F33B4240F01B850135FA
:105FE000202DF7D1D8F8040003689B689847002556
:105FF00007464FF0010909FA05F33B4240F04A8594
:106000000135202DF7D1D8F8040003689B68984724
:10601000002507464FF0010909FA05F33B4240F01D
:1060200079850135202DF7D1D8F804000368DB68A5
:106030009847002507464FF0010909FA05F33B424E
:1060400040F0A4850135202DF7D14A4B089308AFC5
:106050000425D8F8040003689B6898470026834607
:106060000123B34013EA0B0F40F0CB850136202EFD
:10607000F6D1D8F804000368DB6898470026834609
:106080000123B34013EA0B0F40F001860136202EA6
:10609000F6D1013D15F0FF0507F10107D9D1D8F878
:1060A000040003689B6898474FF00109074609FA06
:1060B00005F33B4240F02F860135202DF7D1D8F86B
:1060C00004000368DB689847002507464FF0010984
:1060D00009FA05F33B4240F05A860135202DF7D1ED
:1060E000D8F8040003689B689847002507464FF0DE
:1060F000010909FA05F33B4240F085860135202D60
:10610000F7D1D8F804000368DB68984700250746F4
:106110004FF0010909FA05F33B4240F0B086013522
:10612000202DF7D1144B0793D8F8040003689B681F
:106130009847002583460123AB4013EA0B0F41D05B
:1061400000275FFA85F9D4F8083313F4803A31D187
:1061500007AB4946DB5D04931A462046FFF7DEFA9B
:10616000049B0646002800F0C686CDE908AA07E091
:10617000842500200C0D0E0F20212223801A0600FA
:10618000099B0B93002201210BA8CDE9092204F001
:106190006FFF01462046FFF7B1FA0BA8FDF7D4FECA
:1061A0000AA8FDF7D1FE09A8FDF718FF16B108A847
:1061B000FDF714FF94F82330052B00F048810137D8
:1061C000042FC0D10135202DB5D1D8F804000368C3
:1061D000DB689847002583460123AB4013EA0B0F89
:1061E00038D000275FFA85F9D4F8083313F4803AE1
:1061F00028D107AB4946DB5D04931A462046FFF7DA
:106200008DFA049B0646002800F08486CDE908AA92
:106210000022099B0B9311460BA8CDE9092204F03B
:1062200027FF01462046FFF769FA0BA8FDF78CFE11
:106230000AA8FDF789FE09A8FDF7D0FE16B108A847
:10624000FDF7CCFE94F82330052B00F000810137D8
:10625000042FC9D10135202DBED1D8F80400036820
:106260009B689847002682460123B34013EA0A0F31
:1062700031D010255FFA86F9D4F8083313F0080BF3
:1062800020D12A4649462046FFF748FA074600280B
:1062900000F04F86CDE909BB0A9B002201210BA823
:1062A000CDE90A2301F048FC01462046FFF726FA13
:1062B0000BA8FDF793FE0AA8FDF790FE17B109A8F9
:1062C000FDF78CFE94F82330052B00F0C0800135DB
:1062D000EDB2142DD0D10136202EC5D1D8F804004E
:1062E00003689B689847002682460123B34013EA5F
:1062F0000A0F34D014255FFA86F9D4F8083313F462
:10630000001B24D12A4649462046FFF707FA0746D4
:10631000002800F02186CDE908BB099B0B930022E1
:1063200001210BA8CDE9092202F018F80146204608
:10633000FFF7E4F90BA8FDF707FE0AA8FDF704FE36
:1063400009A8FDF74BFE17B108A8FDF747FE94F822
:106350002330052B7BD00135EDB2182DCDD1013680
:10636000202EC2D1D8F804000368DB6898470026C5
:1063700082460123B34013EA0A0F34D014255FFA92
:1063800086F9D4F8083313F4001B24D12A46494671
:106390002046FFF7C3F90746002800F0ED85CDE958
:1063A00008BB0022099B0B9311460BA8CDE90922DB
:1063B00001F0D4FF01462046FFF7A0F90BA8FDF736
:1063C000C3FD0AA8FDF7C0FD09A8FDF707FE17B138
:1063D00008A8FDF703FE94F82330052B37D00135CC
:1063E000EDB2182DCDD10136202EC2D12FE0D4F838
:1063F000083313F0010A25D15FFA85FB1E225946A6
:106400002046FFF78BF9064620B3CDE908AA099A82
:106410000B920023082201210BA8CDE9093303F0D8
:10642000C7FA01462046FFF769F90BA8FDF78CFD76
:106430000AA8FDF789FD09A8FDF7D0FD16B108A847
:10644000FDF7CCFD94F82330052B7FF43EAD0DB065
:10645000BDE8F08FD8F8041004220B68CDE90102E2
:10646000B84A0092D3F800A05A461E2309A8D04784
:10647000CDE7D4F8083313F0010A24D15FFA85FB85
:106480001E2259462046FFF749F9064608B3CDE9D2
:1064900008AA099B0B93062200210BA8CDE909113C
:1064A00003F086FA01462046FFF728F90BA8FDF70E
:1064B0004BFD0AA8FDF748FD09A8FDF78FFD16B1B1
:1064C00008A8FDF78BFD94F82330052B7FF40EAD63
:1064D000BDE7D8F8041004220B68CDE90102994AFF
:1064E0000092D3F800A05A461E2309A8D047D0E74F
:1064F000D4F8083313F4805A21D15FFA85FB0D22BA
:1065000059462046FFF70AF90646F0B1CDE909AA37
:106510000A9B0022CDE90A23012108220BA804F0DE
:10652000B5FA01462046FFF7E9F80BA8FDF756FD3E
:106530000AA8FDF753FD16B109A8FDF74FFD94F821
:106540002330052B7FF4E3AC81E7D8F80410042254
:106550000B68CDE901027B4A0092D3F800A05A46AD
:106560000D230AA8D047D3E7D4F8083313F4801AD0
:1065700021D15FFA85FB2C2259462046FFF7CEF841
:106580000646F0B1CDE909AA0A9B0022CDE90A230B
:10659000012108220BA804F0A7FB01462046FFF7C3
:1065A000ADF80BA8FDF71AFD0AA8FDF717FD16B107
:1065B00009A8FDF713FD94F82330052B7FF4B8AC40
:1065C00045E7D8F8041004220B68CDE901025D4AC2
:1065D0000092D3F800A05A462C230AA8D047D3E74C
:1065E000D4F8083313F480773FD15FFA85F90C2291
:1065F00049462046FFF792F80646002800F08480BE
:10660000CDE90677079B0A934FF0000A69224946B5
:106610002046CDF81CA0FFF781F80746002800F0BF
:106620008180CDE908AA099B0B9300221A230992C5
:106630000BA901220AA801F007F801462046FFF73E
:106640005DF80BA8FDF7CAFC09A8FDF7C7FC17B158
:1066500008A8FDF7C3FC0AA8FDF7C0FC07A8FDF7D2
:10666000BDFC16B106A8FDF7B9FC94F82330052B44
:106670003FF4EDAED4F8083313F480777FF46AACBE
:106680005FFA85F90C2249462046FFF747F806468F
:10669000002859D0CDE90677079B0A934FF0000AEE
:1066A000682249462046CDF81CA0FFF737F8074678
:1066B000002857D0CDE908AA099B0B9300221A2382
:1066C00009920BA901220AA800F0BEFF014620464C
:1066D000FFF714F80BA8FDF781FC09A8FDF77EFC75
:1066E00017B108A8FDF77AFC0AA8FDF777FC07A800
:1066F000FDF774FC16B106A8FDF770FC94F8233082
:10670000052B7FF427ACA2E6D8F8041004220B680E
:10671000CDF800B0CDE901024A461F6807A80C2356
:10672000B8476FE7D8F8041004220B68CDF800B022
:10673000CDE901024A46D3F800A009A86923D04751
:1067400071E700BF801A0600D8F8041004220B6815
:10675000CDF800B0CDE901024A461F6807A80C2316
:10676000B84799E7D8F8041004220B68CDF800B0B8
:10677000CDE901024A46D3F800A009A86823D04712
:106780009AE7D4F8083313F480773DD15FFA85F99E
:106790000C2249462046FEF7C1FF0646002800F0BD
:1067A0008180CDE90677079B0A934FF0000A6922A2
:1067B00049462046CDF81CA0FEF7B0FF074600284A
:1067C0007ED0CDE908AA099B0B9300221A230BA9BE
:1067D0000AA8099200F038FF01462046FEF78EFF16
:1067E0000BA8FDF7FBFB09A8FDF7F8FB17B108A8FC
:1067F000FDF7F4FB0AA8FDF7F1FB07A8FDF7EEFB98
:1068000016B106A8FDF7EAFB94F82330052B3FF4F8
:106810001EAED4F8083313F480777FF4ADAB5FFA83
:1068200085F90C2249462046FEF778FF06460028E7
:1068300055D0CDE90677079B0A934FF0000A6822EE
:1068400049462046CDF81CA0FEF768FF0746002801
:1068500053D0CDE908AA099B0B9300221A230BA958
:106860000AA8099200F0F0FE01462046FEF746FF16
:106870000BA8FDF7B3FB09A8FDF7B0FB17B108A8FB
:10688000FDF7ACFB0AA8FDF7A9FB07A8FDF7A6FBDF
:1068900016B106A8FDF7A2FB94F82330052B7FF470
:1068A0006BABD4E5D8F8041004220B68CDF800B027
:1068B000CDE901024A461F6807A80C23B84772E7D2
:1068C000D8F8041004220B68CDF800B0CDE901021D
:1068D0004A46D3F800A009A86923D04773E7D8F83F
:1068E000041004220B68CDF800B0CDE901024A463D
:1068F0001F6807A80C23B8479DE7D8F804100422A6
:106900000B68CDF800B0CDE901024A46D3F800A0EB
:1069100009A86823D0479EE7D4F8083313F0200A6B
:1069200024D15FFA85FB1C2259462046FEF7F6FE6D
:10693000064608B3CDE908AA0022099B0B9311462D
:106940000BA8CDE9092203F031FC01462046FEF7F1
:10695000D5FE0BA8FDF7F8FA0AA8FDF7F5FA09A885
:10696000FDF73CFB16B108A8FDF738FB94F823307F
:10697000052B7FF412AB6AE5D8F8041004220B68EB
:10698000CDE90102B84A0092D3F800A05A461C2370
:1069900009A8D047D0E7D4F8083313F0200A24D14F
:1069A0005FFA85FB1E2259462046FEF7B7FE0646D3
:1069B00008B3CDE908AA0022099B0B9311460BA846
:1069C000CDE9092203F0F2FB01462046FEF796FED0
:1069D0000BA8FDF7B9FA0AA8FDF7B6FA09A8FDF762
:1069E000FDFA16B108A8FDF7F9FA94F82330052B43
:1069F0007FF4E4AA2BE5D8F8041004220B68CDE953
:106A00000102994A0092D3F800A05A461E2309A811
:106A1000D047D0E7D4F8083313F0200A25D15FFA25
:106A200085FB1C2259462046FEF778FE064610B329
:106A3000CDE908AA099A0B920023022201210BA892
:106A4000CDE9093303F0B2FB01462046FEF756FEBE
:106A50000BA8FDF779FA0AA8FDF776FA09A8FDF761
:106A6000BDFA16B108A8FDF7B9FA94F82330052B42
:106A70007FF4B5AAEBE4D8F8041004220B68CDE942
:106A80000102794A0092D3F800A05A461C2309A8B3
:106A9000D047CFE7D4F8083313F0200A25D15FFAA6
:106AA00085FB1E2259462046FEF738FE064610B3E7
:106AB000CDE908AA099A0B920023022201210BA812
:106AC000CDE9093303F072FB01462046FEF716FEBE
:106AD0000BA8FDF739FA0AA8FDF736FA09A8FDF761
:106AE0007DFA16B108A8FDF779FA94F82330052B42
:106AF0007FF486AAABE4D8F8041004220B68CDE931
:106B00000102594A0092D3F800A05A461E2309A850
:106B1000D047CFE7D4F8083313F0400A21D15FFA09
:106B200085FB0C2259462046FEF7F8FD0646F0B1DB
:106B3000CDE909AA0A9B0022CDE90A2301210622F8
:106B40000BA800F047FD01462046FEF7D7FD0BA835
:106B5000FDF744FA0AA8FDF741FA16B109A8FDF7B6
:106B60003DFA94F82330052B7FF45BAA6FE4D8F844
:106B7000041004220B68CDE901023B4A0092D3F8CD
:106B800000A05A460C230AA8D047D3E7D4F808330C
:106B900013F0400A20D15FFA85FB0C2259462046AB
:106BA000FEF7BCFD0646E8B1CDE909AA00220A9B22
:106BB00011460BA8CDE90A2300F00CFD0146204642
:106BC000FEF79CFD0BA8FDF709FA0AA8FDF706FAE7
:106BD00016B109A8FDF702FA94F82330052B7FF4CB
:106BE00031AA34E4D8F8041004220B68CDE901027C
:106BF0001D4A0092D3F800A05A460C230AA8D04799
:106C0000D4E7D4F8083313F0800A26D13B78F1B2E8
:106C10001A462046CDE90413FEF780FDDDE9041392
:106C2000814618B3CDE909AA0A9B0022CDE90A23BF
:106C300001210C220BA803F087F901462046FEF73C
:106C40005DFD0BA8FDF7CAF90AA8FDF7C7F9B9F170
:106C5000000F02D009A8FDF7C1F994F82330052BE5
:106C60007FF404AAFFF7F3BB801A0600D8F80400EB
:106C7000B84AD0F800E000924FF0040CCDE9019C36
:106C80000A46DEF800A001460AA8D047CCE7D4F8AF
:106C9000083313F0800A26D13B78F1B21A46204619
:106CA000CDE90413FEF73AFDDDE90413814608B38C
:106CB000CDE909AA0A9B0022CDE90A2300210C2272
:106CC0000BA803F041F901462046FEF717FD0BA87B
:106CD000FDF784F90AA8FDF781F9B9F1000F02D098
:106CE00009A8FDF77BF994F82330052B7FF4CEA992
:106CF000FFF7ADBBD8F80400964AD0F800E0009248
:106D00004FF0040CCDE9019C0A46DEF800A00146D4
:106D10000AA8D047CEE7D4F8083313F4004A20D1AC
:106D20005FFA85FB0C2259462046FEF7F7FC064623
:106D3000F0B1CDE909AA0A9B002201210BA8CDE9F7
:106D40000A2302F077FF01462046FEF7D7FC0BA886
:106D5000FDF744F90AA8FDF741F916B109A8FDF7B6
:106D60003DF994F82330052B7FF4A6A9FFF76FBBFC
:106D7000D8F8041004220B68CDE90102754A00928C
:106D8000D3F800A05A460C230AA8D047D3E7D4F87A
:106D9000083313F4004A20D15FFA85FB0C225946D0
:106DA0002046FEF7BBFC0646F0B1CDE909AA002259
:106DB0000A9B11460BA8CDE90A2302F03BFF0146CE
:106DC0002046FEF79BFC0BA8FDF708F90AA8FDF783
:106DD00005F916B109A8FDF701F994F82330052B40
:106DE0007FF47BA9FFF733BBD8F8041004220B68AB
:106DF000CDE90102574A0092D3F800A05A460C236D
:106E00000AA8D047D3E7D4F8083313F4007A20D186
:106E10005FFA85FB302259462046FEF77FFC064686
:106E2000F0B1CDE909AA0A9B002201210BA8CDE906
:106E30000A2303F087FC01462046FEF75FFC0BA8FF
:106E4000FDF7CCF80AA8FDF7C9F816B109A8FDF7B7
:106E5000C5F894F82330052B7FF450A9FFF7F7BA53
:106E6000D8F8041004220B68CDE90102394A0092D7
:106E7000D3F800A05A4630230AA8D047D3E7D4F865
:106E8000083313F4007A20D15FFA85FB302259468B
:106E90002046FEF743FC0646F0B1CDE909AA0022E0
:106EA0000A9B11460BA8CDE90A2303F04BFC0146CF
:106EB0002046FEF723FC0BA8FDF790F80AA8FDF783
:106EC0008DF816B109A8FDF789F894F82330052B41
:106ED0007FF425A9FFF7BBBAD8F8041004220B6889
:106EE000CDE901021B4A0092D3F800A05A46302394
:106EF0000AA8D047D3E7D8F8041004200A68CDE9DF
:106F0000016014480090D2F800A009A84A46D04772
:106F1000FFF736B9D8F8041004200A68CDE90160FB
:106F20000C480090D2F800A009A84A46D047FFF7C5
:106F30006FB9D8F8041004220B68CDE90102054AA4
:106F40000092D3F800B04A462B460AA8D847FFF76C
:106F5000A3B900BF801A0600D8F8041004220B68F9
:106F6000CDE901020C4A0092D3F800B04A462B4604
:106F700009A8D847FFF7D1B9D8F8041004220B6844
:106F8000CDE90102044A0092D3F800B04A462B46EC
:106F900009A8D847FFF705BA801A060073B504465A
:106FA000FEF77EFF94F82330052B32D0002594F8AD
:106FB0003F33EB40DA07E9B216D40135082DF6D19C
:106FC00094F82330052B24D094F8203013B194F892
:106FD0002230F3B9104B11491B68986903681B688C
:106FE00002B0BDE870401847D4F808339B030CD4B6
:106FF0002C200191FEF7C6F9064610B1019903F065
:1070000019FC31462046FEF779FB94F82330052B16
:10701000D3D102B070BD00BF8425002018990908A3
:107020002DE9F04F90F9213089B00446002B00F093
:107030000481012300F50C7580F84133024600F508
:107040000F712B462E46D06E002859D0002384F8AD
:10705000413394F94030642B5BD094F9BC30642BFD
:1070600000F08D8094F93831642B00F08A80D4F8D8
:1070700030722FBB01A920462DF06EFE00B30C2309
:107080000593012306978DF81830714B07936946D5
:10709000BDF80430049704A8ADF810308DF80070E6
:1070A0002DF0DAFF9DF9001051B1022908DC38B14A
:1070B000C9B27C2303FB01416C3128462FF0C0FC90
:1070C00094F841B3BBF1000F5DD0E36E6367D4F871
:1070D000E830C4F8F030D4F86431C4F86C3194F876
:1070E000233003F1C30204EB82020021042B7CD87D
:1070F00052F8040B1061013342F8041CDBB2F5E7CF
:1071000053F8040B0028A1D18B4202F17C029AD1E2
:107110009FE7002066238DF810307C2303FB00409E
:1071200004A940302FF0D0FB04A920462DF014FE16
:1071300000289CD004238DF818300023CDE90133BA
:10714000039331230593694604A82DF085FF059B21
:1071500028B108AA02EB8302009942F8E01C01332F
:10716000332B0593EFD950F033FF9DED031ADDED7E
:10717000020A9DED010A662150F0E8FE77E7012042
:10718000C8E70220C6E70127A94655F8043B23B10A
:10719000AB600137042FF7D197E7AA46B8465FFAEC
:1071A00088F3022BF5D8DAF8002055F8043C9A420F
:1071B00005D104A95046CDF810B02FF041FC5AF883
:1071C000043B08F101020BB99046E8E704A906EB7D
:1071D00088000193CDF810B02FF032FC019BAB601A
:1071E00001A948462FF02CFCD3E794F8413313B99A
:1071F0002046FEF78FF994F822300BB3154B1B682D
:10720000986A036864215B6898472046FEF752FD40
:1072100094F83E3003B9E36694F8BA300BB9C4F879
:10722000E83094F836310BB9C4F86431FAF764FAEF
:10723000FAF7ECFA0123A4F8403309B0BDE8F08F67
:107240002046FFF7ABFE94F82230002BE0D0D5E7C4
:10725000D0350A08842500207047000001207047BF
:1072600001207047436898687047000010B5054BCF
:1072700003600446806A10B103685B689847204643
:1072800010BD00BFD89D0908406803685B6A1847B5
:1072900033B46C46406884E80C0003689D6A94E847
:1072A0000C00AC4602B030BC6047000010B504468C
:1072B000FFF7DCFF2046FEF76DF8204610BD00000A
:1072C00040680BF003BA0000406801230BF0FEB9E0
:1072D00040680BF0D7B9000040680A220BF07CB977
:1072E00040680BF091B9000040680BF013BA000041
:1072F00090F82E2022B190F82D10002201F06EB9E6
:107300007047000073B5044605250026A06A8DF875
:10731000076003680DF10702DB680121984778B127
:107320009DF807300C2B09D0102B05D0092B07D165
:1073300084F8303002B070BD1523F9E71423F7E765
:10734000013DE3D12846F5E710B4806A03681C6963
:107350000822A44601235DF8044B31216047000058
:1073600010B4806A03681C690122A44600235DF8FA
:10737000044B322160470000F0B50446806A036880
:1073800085B05B6998470546002800F08480A06AB4
:1073900003685B69984703689B689847A06A03681D
:1073A0009B69984760B93D4B3D491B6898690368E4
:1073B0001B6898472B682846DB689847002667E0DB
:1073C0002046FFF7CDFF0028F4D02046FFF79AFFB4
:1073D0000028EFD0A06A03680121DB6A98472046A5
:1073E000FFF7B2FF30B92D4B2E491B68986903682F
:1073F0001B68DEE7A06A0368DB69984730B9274B52
:1074000029491B68986903681B68D2E7A06A94F849
:107410003010012784F82E7003685B6A9847A06AD1
:1074200003689B6A984704F12D020146204601F04B
:1074300023F906460028BDD0A06A94F82D100368F1
:1074400001919B6A984701990246204601F018F97C
:1074500094F82C302BB194F82D103A46204601F0C8
:1074600023F994F82F2094F82D10204601F03EF9CE
:107470002B682846DB689847A06A029403681D6A57
:107480000A4B039304AB13E90C0042F21071A847B6
:10749000304605B0F0BD0646FAE700BF842500205F
:1074A000449D09086A9D0908899D0908A575010878
:1074B00070B5002586B0CDE9005500230446806AEA
:1074C0008DF8085005930393049303686A469E68F9
:1074D00010210923B047A0B19DF8003013F0010638
:1074E00015D194F831300133DBB2052B84F83130FB
:1074F00007D12046FFF734FF2046FFF725FF84F829
:107500003160A06A03681B6B984706B070BD9DF898
:10751000083084F831501B07F3D4BDF901309FEDDA
:107520001F6A06EE903ABDF9033007EE103ABDF936
:107530000530F8EEE66A07EE903ACDED036AF0EE1C
:10754000E66AB8EEC77AF8EEE77AF4EEC66AF1EECC
:1075500010FA8DED047ACDED057A0DD5B0EEC77A2F
:10756000B4EEC67AF1EE10FA06D5F0EEE77AF4EE54
:10757000C67AF1EE10FAC4D49FED090A03A811F0FF
:10758000E9FAB2EE040A03A811F0E4FA94F82D2007
:107590000A2303A9204601F00FF9B2E700000034E6
:1075A0009A99193EFFF784BF10B5044B044640F882
:1075B000043BFCF713FD204610BD00BFF09D0908F9
:1075C00010B50446FFF7F0FF2046FDF7E3FE204626
:1075D00010BD0000F7B503680F4616461BB900241E
:1075E000204603B0F0BD0024046008200193FDF79D
:1075F000C9FE054620B1124B0360019B4360019414
:1076000001A8FCF7EBFC002DE9D03420FDF7BAFE11
:1076100004460028E3D000F0E1FE0A4BA562236097
:1076200084F82C7084F82F602046FFF7A5FE0546ED
:107630000028D5D1236820465B6898472C46CFE7C1
:10764000F09D0908D89D09082DE9F74F0468064602
:107650000D4690469946002C6CD00B68002B49D003
:10766000236820465B6A984703689B689847012314
:1076700028680DEB030200210BF028F898B39DF861
:107680000130EA2B2FD1DFF8F0B04FF0060A28685E
:107690000023802206210AF0F5FF20B3DBF80070FA
:1076A000B86A03680A215B689847002328681A466D
:1076B00006210AF0E7FFB0B1B86A03680A215B68E7
:1076C0009847012328680DEB030206210AF0FEFF0C
:1076D00048B19DF8014014F040042FD00AF1FF3A60
:1076E0001AF0FF0AD3D1306803685B6A98470368D1
:1076F000DB68984700241DE0022223460F212868FA
:107700000AF0C0FFB86A036801215B6898473068D7
:1077100003685B6A98470368DB689847336834609E
:107720004A46414601A80193FFF754FF044601A8C9
:10773000FCF754FC204603B0BDE8F08F22462346F8
:107740000F2128680AF09EFFB86A036801215B6870
:1077500098470223214630680DEB03020AF0B6FF7A
:1077600004460028C8D0B869024903681B689847D6
:10777000B9E700BFB09D09088425002090F82C10BF
:10778000002200F02BBF000070B504468CB0042628
:10779000013E76B2731C4AD0A06A15236A465D2169
:1077A0000AF094FF0028F3D0A06A152306AA5D21F1
:1077B0000AF08CFF05460028EAD0152206A9684683
:1077C00079F0BEF80028E3D19DF8003084F82E301F
:1077D0009DF8073084F830309DF8143084F83A3042
:1077E0009DF813309DF8102084F83B309DF80F3041
:1077F00043EA0223A3879DF8013084F82F309DF8D7
:10780000083084F83130039B9DF80C20C3F30F231C
:1078100063869DF80B3043EA0223A386049BC3F3DF
:107820000F23E386019BC3F30F23238707E0054B58
:1078300005491B68986903681B6898470025284616
:107840000CB070BD84250020249E09082DE9FF415D
:1078500004460023806A8DF807300368DFF86881EA
:107860005B6A984703689B689847A06A03680A2187
:107870009B6C9847A06A0A2204210AF0ADFE0425F9
:10788000013D6DB26B1C32D000234B21A06A8222D5
:107890000AF0F8FED8F800600746B06A03680221D3
:1078A0005B689847002FEBD001231A464B21A06A52
:1078B0000AF0E8FE0746B06A036802215B68984751
:1078C000002FDDD0A06A01230DF1070240210AF04C
:1078D000FDFE0028D4D09DF80720322A10D0002DBC
:1078E000CED1B069364903681D683223A847A06A23
:1078F00003685B6A98470368DB68984700255BE08C
:107900002046FFF741FF0028F1D0A06A012317228B
:1079100051210AF0B7FE0028E9D05222A06A0123C3
:1079200011460AF0AFFE0028E1D0A06A01233822F8
:107930004C210AF0A7FE0028D9D0A06A03685B6A30
:1079400098470368DB689847A06A05210AF05CFE47
:10795000A36A04F12C029968204600F08DFE0546CA
:1079600050B3A36A94F82C109A68204600F088FE61
:1079700094F8442094F82C10204600F0B7FE94F8B8
:1079800045302BB194F82C100122204600F08CFEDB
:10799000A06A036802219B6C9847A06A029403685E
:1079A0009E6A084B039304AB13E90C0044F21B11CD
:1079B000B04752F089FC2064284604B0BDE8F0814D
:1079C0004C9E0908357B01088425002070B5858F01
:1079D00090F93B60AD03B5FBF2F2A2F5804404FBE5
:1079E00004F2D51190F83A200498D201624306FBC4
:1079F00005225212A03002F58012424312134A436C
:107A0000DB0003EB623000B270BD000010B5448EA5
:107A100053005C43B0F93830C91A838FD31AB0F9D8
:107A20003620B0F93400534304F500449B10C3EBF7
:107A3000C13300EB2440044993FBF0F04FF40042C3
:107A40000EF0C6FF00B210BD0080FFFF10B52DED97
:107A5000028B8AB004460823806A05AA42210AF0F4
:107A600035FE18B1BDF81A20D30719D4A06A0AF060
:107A700051FE52F029FC236CC31AFA2B0CD9206456
:107A8000002382224B21A06A0AF0FCFD0123A06A98
:107A90001A464B210AF0F6FD0AB0BDEC028B10BD70
:107AA000BDF9141094F930300093920894F92E30F7
:107AB0000392C9102046FFF789FFBDF9161094F90B
:107AC0003130039A009308EE900A94F92F30C910D0
:107AD0002046FFF77BFFBDF91810039A491008EE06
:107AE000100A2046FFF792FF07EE900AF8EEE88AA8
:107AF000F8EEE77AB8EEC88AB3EE000A07A8CDED33
:107B0000097ACDED078A8DED088A11F037F8B2EECB
:107B1000040A07A811F01EF852F0D6FB94F82C20A6
:107B200020640A23204607A900F046FEA06A0AF056
:107B3000F1FDB1E7FFF78ABFF7B503680D461646BA
:107B40001BB90024204603B0F0BD00270760482081
:107B5000CDE90073FDF716FC044650B100F03EFC81
:107B60000E4B2360019BA362019784F8446084F864
:107B7000455001A8FCF7E8F96846FCF7E5F9002C48
:107B8000DFD02046FFF762FE05460028DAD12368E1
:107B900020465B6898472C46D4E700BF849E0908BE
:107BA00010B5044B044640F8283BFCF7CDF92046BD
:107BB00010BD00BF849E090810B50446FFF7F0FF12
:107BC0002046FDF7E7FB204610BD000090F82C1082
:107BD000002200F003BD0000F8B504460D4617462C
:107BE0001E4600F0FBFB094B23602B68A3620022BA
:107BF00000232A6084F82D7084F82E602365636565
:107C0000A365E365236663662046F8BD9C9E09086C
:107C1000F8B51C4609331646DB086A46A2EBC303D7
:107C200000AF9D46806AA31C6A460AF04FFD0546D8
:107C300028B122460DF10201304678F091FE284627
:107C4000BD46F8BD2DE9F34106460F46144652F0F5
:107C50003BFB114BD3F800800546D8F82800036899
:107C600001215B68984701230DF107020721304687
:107C7000FFF7CEFF60B19DF80730DA0702D4B7EB0B
:107C8000531F05D052F020FB431BA342E5D3002035
:107C900002B0BDE8F08100BF842500202DE9F0414D
:107CA000DFF8608292B0044602AF002646F0200260
:107CB000A06A0023D2B250210AF0E4FC002800F0B0
:107CC0000C810325013D6DB26A1C00F00681D8F8D5
:107CD0000030986A03684FF496719B6898470123B7
:107CE0000DF1060255212046FFF792FF002800F013
:107CF000F4809DF8063013F0E00F40F0EE80DB07D3
:107D0000E0D502230DF1060252212046FFF780FF45
:107D1000002800F0E280BDF8063001365BBA202E64
:107D200027F8023BC2D1BDF824309DF826109FED04
:107D30006D7ADFED6D6A9FED6D6A43F30B0207EE1E
:107D4000902A1B0903F47063BDF82620F8EEE77A49
:107D50000B4343F30B03C4ED0C7A07EE903A02F4A5
:107D600070639DF82820F8EEE77A134343F30B0382
:107D7000C4ED0D7A07EE903A9DF92230F8EEE77ADD
:107D8000C4ED0E7A07EE903A9DF92930F8EEE77AC5
:107D900067EE877A07EE103AB8EEC77A9DF92A3077
:107DA000C4ED0F7A27EE267ADFED517A84ED107A52
:107DB00007EE103AB8EEC77A9DF92B30E7EE267A37
:107DC000C4ED117A07EE903AF8EEE77A9DF9233088
:107DD00067EEA67ADFED476AC4ED127A07EE903AB5
:107DE0009DF92C3007EE103AB8EEC77A9DF92E3087
:107DF00027EE267AF8EEE77A84ED147A67EE867A33
:107E000007EE103A9DF93030C4ED137A07EE903A40
:107E1000F8EEE77A9DF92D3067EEA67AB8EEC77ACC
:107E2000C4ED167A27EE267A07EE903A84ED157A9D
:107E3000F8EEE77A9FED307A9DF92F3067EE877A7A
:107E4000C4ED177A07EE903A9DF93130F8EEE77AF3
:107E500006EE903A67EE877AF8EEE66AC4ED187A95
:107E6000DFED267ABDF93830E6EE877A07EE103A74
:107E70009DF93230C4ED197AB8EEC77AF3EE077A7D
:107E8000E7EE067A07EE103ADFED1D6AC4ED1A7AC6
:107E9000B8EEC77A27EE267A84ED1B7A9DF9333047
:107EA00007EE103AB8EEC77A9DF9343027EE267AFD
:107EB00084ED1C7A07EE103A9DF9353007EE903AC2
:107EC000B8EEC77AF8EEE77A27EE267A67EEA67A5A
:107ED00084ED1D7AC4ED1E7A00E0002012B0BDE8EA
:107EE000F08100BFCDCC4C3E0000803B0000003B49
:107EF0000AD7233C0000003D0000803817B7D1B8F6
:107F00000AD7A33A8425002073B501230E460DF14C
:107F1000070206210446FFF77BFE18B90025284614
:107F200002B070BD9DF80730013B012B0CD8002337
:107F3000A06A1A4606210AF0A5FB0028EED0062208
:107F400000212046FFF77EFEA06A0023324606216C
:107F50000AF098FB05460028E0D02622314620464C
:107F6000FFF770FEDBE7000013B501230DF10702F8
:107F700007210446FFF74CFE10B9002002B010BDE7
:107F80009DF807301B070CD50023A06A1A4606216E
:107F90000AF078FB0028F0D0062200212046FFF7E7
:107FA00051FEA06A0023072206210AF06BFB00287D
:107FB000E3D0132207212046FFF744FE0028DCD03F
:107FC000A06A0023052206210AF05CFB0028D4D019
:107FD000172205212046FFF735FE0028CDD00121CC
:107FE0002046FFF791FFC9E7F7B50446806A5B4F6B
:107FF00003685B6A984703689B689847A06A0368B0
:108000000A219B6C9847A06A0A2204210AF0E4FA2C
:108010000525013D6DB26B1C00F09680A06A00231F
:10802000B6227E210AF02EFB0028F2D03B68986A27
:10803000036818215B686E46984701233246002189
:108040002046FFF7E5FD0028E3D09DF80030332BF4
:10805000DFD12046FFF722FE002875D0A06A00235A
:10806000802250210AF00EFB00286DD02046FFF739
:108070007BFF002868D0A06A002386222E210AF008
:1080800001FB002860D0A06A0023242204210AF00A
:10809000F9FA002858D0A06A0023022206210AF02B
:1080A000F1FA002850D0142202212046FFF7CAFD21
:1080B000A06A0023072205210AF0E4FA002843D031
:1080C00001212046FFF720FF00283DD0A06A036869
:1080D00003219B6C9847A06A03685B6A9847036812
:1080E000DB689847A06A17210AF08EFAA36A04F1A8
:1080F0002C029968204600F0BFFA054608B3A36A2F
:1081000094F82C109A68204600F0BAFA94F82E20C1
:1081100094F82C10204600F0E9FA94F82D302BB199
:1081200094F82C100122204600F0BEFAA06A0368E1
:108130009F6A0B4B0094019396E80C0042F2107179
:10814000B847284603B0F0BDA06A03685B6A984749
:108150000368DB6898470025F3E700BF842500200B
:108160005983010810B586B00C236A4631210446B4
:10817000FFF74EFD002800F0DF809DF801309DF8EC
:108180000020DFED717ADFED715A1B0403EB02234F
:108190009DF8022003EB02631B1206EE903A9DF855
:1081A00004309DF803201B0403EB02239DF80520F7
:1081B00003EB02631B1207EE103A9DF807309DF89F
:1081C00006201B0403EB02239DF8082003EB026347
:1081D0001B1206EE103A9DF80A309DF809201B0488
:1081E00003EB0223F8EEE66AB8EEC77A9DF80B209F
:1081F00066EEA76A27EE277AB8EEC66ADFED547AF4
:1082000003EB02631B1226EE276A07EE903AF8EEA4
:10821000E77A67EEA57AF5EEC07AF1EE10FA40F350
:108220008D80DFED4C5A77EEE57AD4ED134A94ED6C
:108230000F5A94ED1C4AD4ED1D3A94F82C20F7EE19
:10824000005A74EEA54AF0EE632AA4EEA75A0A2358
:1082500003A9D4ED107AD4ED0C4A77EEA57A204626
:10826000E7EEA64AD4ED1A7A75EE677A94ED145AC1
:10827000F0EE646AD4ED174AE5EE276AB0EE655A6F
:10828000A7EEA45AC6EE854A94ED115AD4ED0D6AB4
:1082900035EE255AE5EE076A94ED157AE7EE876A22
:1082A00094ED187AB0EE655AA7EE875A86EE857A75
:1082B00094ED125AD4ED0E6A35EE255AE5EE066AB3
:1082C00094ED166A94ED195AE7EE866AB0EE656A87
:1082D000A7EE856AF0EE657A86EE863A94ED1B6A23
:1082E000F0EE646AE6EE447AE6EE476A86EEA75A56
:1082F000F0EE476AE4EE646AC6EEA75AD4ED1E6A51
:10830000D4EE262AE6EE636AB2EE046A27EE667AB7
:1083100065EE066AA2EEA47ACDED036A65EE866A82
:10832000CDED046AC7EE276A76EE837A67EE867A29
:10833000CDED057A00F040FA06B010BD44BFDFED88
:10834000055A77EEA57A70E747ABE73B5B9E803A2C
:10835000F61BEB3B85EBCB41FFF704BF30B5134673
:10836000026885B00D461AB90024204605B030BD1C
:10837000002101607C2001930392FDF703F804467D
:1083800020B1019B2A4603A9FFF726FC03A8FBF7AF
:10839000DBFD002CE8D02046FFF726FE054600282E
:1083A000E3D1236820465B6898472C46DDE7000050
:1083B00010B5044B044640F8283BFBF7C5FD2046AA
:1083C00010BD00BF9C9E090810B50446FFF7F0FFE2
:1083D0002046FCF7DFFF204610BD0000064B10B51D
:1083E00003600446FDF756FD606004F1080051F09B
:1083F000C7F8204610BD00BFB49E090873B50646F5
:10840000144675687C2303FB0253C4EB441405EB4C
:108410008404084693F8A410019010F031FC94F9FC
:108420003C3001983BB9736893F8251002B0BDE861
:10843000704010F025BC94F84010F7E737B5446859
:1084400001917C2505FB024595F83F3004EB830440
:10845000D4F84C325BB151F037FFC5F89C0001995C
:10846000D4F84C0203B0BDE8304003F0A7BF03B01E
:1084700030BD00002DE9F04FC2EB421447684FEACF
:10848000840881460E4607F13C0B08F108018BB0C9
:1084900015465944304610F029FBD9F80400294606
:1084A0000BEB8404FDF79CFC38B17C2303FB0573C4
:1084B00093ED1A0A304610F04DFB7C2303FB057345
:1084C00093ED146ADFED3A7AD3ED156AB0EEC67A11
:1084D000B4EEE77AF1EE10FA0FD5B0EEE67AB4EE2C
:1084E000E77AF1EE10FA08D594ED077AB0EEC77A84
:1084F000B4EEE77AF1EE10FA1BD47C2303FB05738C
:10850000D86D196E5A6E9B6D02900391049007917D
:1085100001A831468DED016ACDED056A06920892FB
:1085200009930EF053FC86ED000AC6ED010A86EDB4
:10853000021A7C2303FB05770023C7F88C30C7F8A9
:108540008830C7F88430D9F8040090F95C3208F11B
:108550003C0A08F14808DA44D84463B15DB94146A1
:1085600000F5167004F0E2FB414630460BB0BDE862
:10857000F04F10F0BBBA90F93430012B0BD190EDD5
:108580000E0A504610F092FA84ED120AC4ED130A56
:1085900084ED141AE8E7022BE6D1FCF75DFB00221C
:1085A00001A9FCF727F80028DED09DED010AE8E7D5
:1085B0000000003410B543687C2404FB023407C972
:1085C00004F1900383E8070051F07EFEC4F89C009C
:1085D00051F06EFEC4F8A00010BD0000F0B50746D3
:1085E00085B00D46164600F10801A92203A80AF03D
:1085F000C7FA7C687C2303FB0543D3F8B42022B977
:1086000003A80AF0DFFA05B0F0BDBEB196ED007A1E
:10861000D3ED2A7A67EE877AC3ED2A7A96ED017A4E
:10862000D3ED2B7A67EE877AC3ED2B7A96ED027A3B
:10863000D3ED2C7A67EE877AC3ED2C7A7C2607EE91
:10864000902A06FB0541A831B8EE670A0846019159
:1086500010F094FA01992A463846FFF7ABFF06FB63
:1086600005410023C1F8B030C1F8AC30C1F8A830E2
:108670000023C1F8B430C3E74068FCF79BBF00009B
:10868000F7B50646406801927C2707FB01000D46BE
:108690006C3001A914462EF0B3F9716807FB05157B
:1086A0002C6703B0F0BD000007B540687C2303FBD6
:1086B000010393F93C30022B0BD000F13C03C1EBDA
:1086C000411003EB80000DF107018DF807202EF01B
:1086D000F1F803B05DF804FB43687C2202FB013132
:1086E00091F93C00003818BF0120704743687C2096
:1086F00000FB013181F8A42070470000F8B5054661
:1087000008460F4610F098FA10B100242046F8BD34
:10871000384610F077FA04460028F6D16B6893F9D2
:1087200034637EB1384610F0BFFD95ED087ADFED79
:108730001F7AF0EEC76AF4EEE76AF1EE10FA03D59D
:1087400085ED080A0124E1E777EE407A30EE076A0A
:10875000F0EEE77AC7EE866AF6B207EE906A9FED12
:10876000146AF8EE677A26EE866AF4EEC67AF1EEBF
:1087700010FA48BFB2EE046ADFED0E7A45BF6B6AAD
:1087800066EE866AB0EE676A87EEA66A46BF013378
:108790006B620124F7EE007A77EEC67A20EE060AC5
:1087A000A7EE270A85ED080AB0E700BF00000034F5
:1087B00000004843CDCCCC3D2DE9F74304460E469E
:1087C00015461F46FFF71AFE2A4631462046FFF798
:1087D00035FE314620462A46FFF74CFE31462046FC
:1087E000FFF78CFF28B39B2204F1080101A80AF0CF
:1087F000C7F964684FF07C0909FB054808F1A8082F
:108800003146404610F072F909FB0542D2F8B41027
:108810000131C2F8B4104FB1B94207D34908C2F8C8
:10882000B410B0EE000A404610F0A8F901A80AF012
:10883000C9F903B0BDE8F08310B50446FCF744FF66
:10884000C0B23C34C0EB401004EB800010BD00000F
:10885000F8B50A4E044600F5167704F5137555F879
:10886000040B08B104F0DEF8BD42F8D13368986A11
:10887000036801215B689847EFE700BF842500206B
:1088800008B5FFF7E5FF0000F0B5144E00EB8107D7
:1088900073780446D7F84C026FF3410387B00D4656
:1088A0007370C8B102F0ACFC68B1737843F0100388
:1088B00073702C440023A372D7F84C0207B0BDE8B4
:1088C000F04002F021BCD7F84C12684602F0C8FC18
:1088D000009B012BEDD1E8E707B0F0BDAC5D0020B7
:1088E00070B506460D46002445FA04F3DB07E1B2F5
:1088F00002D53046FFF7C8FF0134032CF4D170BD18
:10890000FF21FFF7EDBF000030B500F5137587B00C
:1089100000F5167455F8041B21B9A542FAD10020C0
:1089200007B030BD684602F09BFC009B013B022B68
:10893000F3D80120F4E700002DE9F0472DED028B7C
:1089400088B004460D469046B0EE408AFDF790F997
:1089500030B90026304608B0BDEC028BBDE8F08788
:1089600029462046FCF7FEFF06460028F1D004EB1E
:108970008507D7F83C22D7F830329A4206D039F032
:10898000F5FF5C4A032133F0C1F9E2E7D7F84C3236
:1089900083B94FF49870FCF7F5FC814608B103F0F9
:1089A00045F9C7F84C92B9F1000F03D139F0DEFF59
:1089B000514AE7E7B4F84A32D90711D505F0CEFF9E
:1089C00090F8382390F8F43232B9B02202FB030059
:1089D00090F8D130012B03D839F0C8FF474AD1E7CE
:1089E0002046FFF791FF20B9454A537843F0020330
:1089F000537094F9353053B329462046FFF71CFFD6
:108A000090F90030002B53D029462046FFF714FF81
:108A100090F80490B9F12B0F19D829462046D7F8C1
:108A20004CA2FFF709FF94F9353090F90020022B92
:108A3000D4BF00210121012BD4BF00230123003A20
:108A4000009118BF01224946504602F071FB63199C
:108A500000229A7275B3D4EDC10AB4F84822D7F84F
:108A60004C0270EEA00A2B46B0EE480A414602F0D6
:108A70007FFB94F83E33002B31D1224A06941268D2
:108A80000127E773906A0268156D1F4A07920293E7
:108A900009224FF40063CDE9003208AA12E906006A
:108AA0001A4BA847C8B939F061FF194A02216AE791
:108AB0009946B2E729462046FFF7BEFE90F90030FE
:108AC000002BC8D0D4EDC10AB4F84822D4F84C0227
:108AD0002B46B0EE480A4146C9E784F83E730023AE
:108AE0000DF1170104F124008DF817302DF0ECFE84
:108AF00030E700BFC49E0908F69E0908199F0908BF
:108B0000AC5D00208425002081880108379F09087A
:108B1000429F09082DE9F0412DED028B002443739B
:108B20009DF82030837305460F469046B0EE408A8C
:108B3000264647FA04F3DB07E1B210D5B0EE480A47
:108B400042462846FFF7F8FE064640B93946284611
:108B5000FFF7C6FEBDEC028B3046BDE8F081013464
:108B6000032CE6D1F6E70000F8B500242DED028BCA
:108B700005460F46B0EE408A427383732646E1B243
:108B8000B0EE480A3A462846FFF7D6FE01340028E0
:108B900018BF0646032CF2D1BDEC028B3046F8BD5F
:108BA000F0B500EB81030D46D3F84C129BB00446A0
:108BB00011B900201BB0F0BD0BA802F035FB631902
:108BC000987A0028F6D10B9A002A48D0042AF0D1CE
:108BD00001229A720DAA07CA02AB83E8070010AA05
:108BE00007CA05AF87E8070013AA07CA9DED180A50
:108BF00008AE86E807001A46294620468DED010A90
:108C0000FCF744FE3A4629462046FCF7EBFD324687
:108C100029462046FCF7F8FD9DED010A294620462D
:108C2000FCF704FE9DF8643083B129462046FFF727
:108C300003FE90F900304BB194F93530012B05DD7E
:108C40009DF85D2029462046FCF738FE2046FFF7B8
:108C50005BFE20B9034A537843F0040353700120AC
:108C6000A8E700BFAC5D00202DE9F041054688462D
:108C700000F513770024012657F8043BE1B26BB1ED
:108C800048FA04F3DB0709D52846FFF789FF0028D7
:108C900057F8040C08BF002602F036FA0134032C02
:108CA000EAD13046BDE8F0812E4B2DE9F04F1F6828
:108CB000FB6A93F89C8087B00446B8F1000F38D166
:108CC000DFF8A8A000F5137600F1030B054656F86F
:108CD000040BA5EB04095FFA89F9E8B102F07CFA0C
:108CE00028B19AF8013043F008038AF8013056F8A9
:108CF000040C02F085FAF8B9637B6BB1AB7A5BB90F
:108D000056F8041C684602F0ABFA009B042B03D112
:108D100049462046FFF744FF01355D45D7D1124B48
:108D2000204683F81280FFF7EFFD054630B101239E
:108D3000237407B0BDE8F08F8046EDE7237C002B5D
:108D4000F7D0A37B002BF4D0B86A03684FF47A7194
:108D50005B689847B86A03689B6B294607B0BDE813
:108D6000F04F1847842500208D5D0020AC5D002069
:108D7000F0B5002587B000F513762C46012756F88C
:108D8000041B41B1684602F06BFA009B1BB107FA65
:108D900005F31C43E4B20135032DF0D1204607B0A2
:108DA000F0BD00002DE9F04F2DED028B03270E7C66
:108DB0009FED348A91B005468846B946AC5D0134D2
:108DC000E4B2B4FBF9F303EB4303E41AE4B205EBBA
:108DD0008403D3F84C1209B9AC554CE003A802F057
:108DE0003FFADDF80CB00BF1FF33022BF4D830461C
:108DF00033F030FF8246304634F030FE00F11B0382
:108E00009A4508D2304633F0A1F9002011B0BDECEC
:108E1000028BBDE8F08FAC55284698F810A0FFF7FC
:108E2000A7FFDDED057A8DF83100FCEEE77A9DF8BD
:108E300010208DF8332017EE903A8DF8343006ABC1
:108E400003CB1B88ADF83D305C221B23CDE90032FB
:108E5000CDF83500CDF8391009AABF2150468DED67
:108E6000098A8DED0A8A8DED0B8A8DF830408DF8D8
:108E700032B033F059FF013F17F0FF079ED10120B8
:108E8000C4E700BF000000002DE9F04F0F7CA1B047
:108E900006468846032500EB070999F8054001348A
:108EA000E4B20323B4FBF3F303EB4303E41AE4B2A9
:108EB00006EB8403D3F84C1211B989F805400AE097
:108EC00011A802F0B1F9DDF844A0BAF1030F08DCF3
:108ED000BAF1000FF1DA013D15F0FF05DDD10120F7
:108EE00012E0AAF10402032AF5D8384633F0B2FEA4
:108EF0008346384634F0B2FD00F13602934506D27F
:108F0000384633F023F9002021B0BDE8F08F89F80E
:108F10000540304698F810B0FFF72AFFDDF848E02A
:108F2000CDF80CE0DDF84CE0CDF810E0DDF850E0D5
:108F3000CDF814E0DDF854E0CDF818E0DDF858E0A5
:108F4000CDF81CE0DDF85CE0CDF820E0DDF860E075
:108F5000CDF824E03219DDF864E01C9BCDF828E060
:108F6000DDF868E092F80AC09DF874109DF875204D
:108F7000CDF82CE00E93DDF86CE01E9B8DF83500EB
:108F80008DF83C108DF83D20CDF830E08DF8344060
:108F90008DF836A08DF837C02422CDF83E30362328
:108FA000CDE90032C0212C2303AA584633F0BCFE81
:108FB00091E700007FB58A8B0B464AF2B9518A428D
:108FC00005465FD04AF2BA518A4274D04AF2B8518B
:108FD0008A420BD1474A1268D26A92F89C203AB171
:108FE00039F0C4FC444A052132F090FE042479E0B3
:108FF000D3ED007AF5EEC07AF1EE10FAF6D49FEDDB
:109000003F7AF4EEC77AF1EE10FAEFDC93ED017AD5
:10901000DFED3B6A1C6993ED030AB0EEC77AB4EE4C
:10902000E67A93ED027AFCEEE77AB0EEC77AF1EEDB
:1090300010FAB4EEE67A17EE903A54BF01260026F5
:10904000F1EE10FA54BF01220022003C18BF0124A7
:1090500013F0FF0110D18DED030A0292FCF77EFBA5
:109060009DED030A029A234631462846FFF77CFD10
:109070000028BBD0002435E0134600943246FFF7A9
:1090800049FDF5E7D3ED007AF5EEC07AF1EE10FA7E
:10909000ACD49FED1A7AF4EEC77AF1EE10FAA5DCA3
:1090A000FCEEE77A17EE903A13F0FF0108BFFF21BC
:1090B000FFF7DAFDDCE7D3ED007AF5EEC07AF1EEEA
:1090C00010FA93D49FED0D7AF4EEC77AF1EE10FA10
:1090D0008CDCFCEEE77A17EE904A14F0FF0404D122
:1090E000FFF70EFC204604B070BD2146FFF7F8FBE9
:1090F000C0E700BF84250020749F090800007F435B
:1091000000000034F0B58BB00E4614460746FFF75A
:1091100093FB543007C884E8070031463846FFF710
:109120008BFB90ED057ADFED267AB0EEC77AB4EED0
:10913000E77AF1EE10FA054611D590ED067AB0EE19
:10914000C77AB4EEE77AF1EE10FA08D590ED077A17
:10915000B0EEC77AB4EEE77AF1EE10FA24D43146D5
:109160003846FFF769FB016A426A836AE869D5F805
:1091700014E0D5F818C0099001A8CDF804E00291D8
:1091800003920491CDF814C00693079208930DF052
:10919000C9FF98B1214601A80DF018FE84ED000A20
:1091A000C4ED010A84ED021A31463846FFF744FB4C
:1091B00000F1080120460FF0B3FC01200BB0F0BD18
:1091C000000000342DE9F0472DED048BACB0B0EE7B
:1091D000608A0546B0EE409A0F46F0EE418A90460E
:1091E000FCF7BCFADFED8B7AB0EEC87AB4EEE77A22
:1091F000F1EE10FA4BD5B0EEE87AB4EEE77AF1EE84
:1092000010FA44D523AC2046FBF720FEF8F774FA99
:109210002146F8F733F8064658BB05F09FFB90F857
:10922000383390F8F42233B1B02303FB020393F8F0
:10923000D130012B07D84FF0B00909FB020090F89C
:10924000D130022B0BD839F091FB734A032132F055
:109250005DFD30462CB0BDEC048BBDE8F08705F019
:109260007DFB90F8F43209FB0300DC300FC884E882
:109270000F00DDED257A9FED691AB8EEE78ADDED86
:10928000267AF8EEE78A28EE018A68EE818A04AA37
:1092900003A902A8F0EE680AB0EE480A03F002FE45
:1092A000064618B939F062FB5D4ACFE79FED5D7A5B
:1092B000DDED027A9FED5C8ADFED5C8A8DED068A3A
:1092C00067EE877A2422002111A8CDED057A8DED75
:1092D000078A77F08FFB9DED031ADDED040ADFF8B6
:1092E00058A121EE281A68EEE00AB0EE480A11A84B
:1092F0000DF038FF05A911A80DF068FD242200210A
:109300001AA8CDED060A8DED071A8DED050A77F046
:1093100071FBF8F7F1F990ED810A8DED010AF8F78C
:10932000EBF929EE281AD0ED820A9DED010A1AA860
:109330000DF018FF1AA923A80DF036FE05A923A8E1
:109340000DF044FD4FF000098DED050ACDED060A44
:109350008DED071A95F822305FFA89F4A3427FF663
:1093600078AF1FB127FA04F3DB071AD52B1993F94D
:109370002C32B3B1B8F1000F0DD021462846FCF7CE
:1093800077FC88B939F0F2FA294A2346032132F0F2
:10939000BDFC00265DE721462846FCF7E3FA0028DD
:1093A000EBD109F10109D5E708AA214628468DED40
:1093B000088A8DED098A8DED0A8AFFF7A3FE20B990
:1093C00039F0D4FA1B4A2346E0E708A905A80FF0B4
:1093D00057FB0BAA214628468DED0B0ACDED0C0A52
:1093E0008DED0D1AFCF752FA9AE807000EAB83E8F0
:1093F00007001A4621462846FCF7F4F923AA21461D
:1094000028468DED238A8DED248A8DED258AFCF783
:10941000FBF9C6E700000034989F090895BFD633D2
:10942000B39F090800007A440000000035FA8E3C22
:10943000C89F0908DC9F0908544C0908012070479F
:1094400001207047436898687047000040680368CF
:109450009B6C184710B5054B03600446806A10B139
:1094600003685B689847204610BD00BFC4A0090888
:10947000406803685B6A184733B46C46406884E808
:109480000C0003689D6A94E80C00AC4602B030BC46
:109490006047000010B50446FFF7DCFF2046FBF7ED
:1094A00079FF204610BD0000406809F0ADB800000B
:1094B000406809F00BB900004068012309F006B9C3
:1094C0004068002309F0DEB890F84420D20705D5A3
:1094D00090F8421000F12C02FFF780B870470000AE
:1094E000F8B504461E460F461546FEF777FF084BB3
:1094F00023600023E3622363636394F84430A7622C
:1095000065F3410384F8436084F844302046F8BD95
:10951000C4A0090810B50D4B83630446806A036834
:1095200098221B690021984770B1A06A0368202225
:109530001B690121984738B1A06A0368BDE8104053
:109540001B69012202211847002010BDC5DC6A3FBB
:1095500037B50446806A03686A469D68032106237E
:10956000A847D0B1BDF80020BDF8041052BA95B29A
:1095700049BAB5F5704F0BB211D013F5805F0ED01C
:10958000BDF802305BBA9DB2B5F5704F07D05242BC
:109590005B42A287E187A4F8403003B030BD0020D1
:1095A000FBE70000806A036801221B69022118475B
:1095B00030B585B00446FFF7CBFF05462046FFF7E0
:1095C000F1FF6DB3B4F93C3094ED0E0A06EE903A1B
:1095D000B4F93E3007EE103AB4F9403007EE903A55
:1095E000F8EEE66AB8EEC77AF8EEE77A01A8CDEDB4
:1095F000016A8DED027ACDED037A0FF0ABFA94F8A3
:1096000042102046FFF768F818B1022101A80FF0B8
:1096100037FB94F842200E2301A92046FFF7CCF82F
:1096200005B030BDFFF7C4BF13B5806A036801AA57
:109630009C680A210323A04738B10549032201A8E9
:1096400077F07EF9B0FA80F0400902B010BD00BF9B
:10965000FC9F09082DE9F84300252DED028BDFF86A
:1096600088819FED5D8A04462E462F46A06A0368D6
:1096700011221B6900210137984700287BD0D8F8B8
:109680000090D9F82800036832215B689847A06AE7
:10969000036860221B690121984700286BD0A06AEB
:1096A000036801221B6902219847002863D0D9F87A
:1096B0002800036832215B6898472046FFF748FF7F
:1096C000002858D00135022FEDB256DDB4F93C30F8
:1096D0009FED425A9FED426A07EE903AF8EEE77A24
:1096E000C5EE276AF0EEE66AF4EEC66AF1EE10FA0D
:1096F00041DDF4EEC86AF1EE10FA3CD5B4F93E3023
:10970000DFED385A07EE903AF8EEE77A85EEA77A61
:10971000B0EEC77AB4EEC67AF1EE10FA2BDDB4EEF5
:10972000C87AF1EE10FA26D5B4F9403005EE903A39
:10973000F8EEE55AC5EE257AF0EEE77AF4EEC67A51
:10974000F1EE10FA17DDF4EEC87AF1EE10FA12D548
:1097500094ED0B6A76EE266A0136C4ED0B6AD4ED01
:109760000C6A36EE877A84ED0C7A94ED0D7A77EEFA
:10977000277AC4ED0D7A192F02D0052E7FF476AF2B
:10978000A06A036810221B6900219847052E18D192
:10979000D4ED0B6AF1EE047A86EEA77A0120D4EDBF
:1097A0000C6A84ED0B7A86EEA77AD4ED0D6A84ED0F
:1097B0000C7A86EEA77A84ED0D7ABDEC028BBDE8BB
:1097C000F8834FF07E53052DE3622363636394BFF8
:1097D00000200120F1E700BFCDCCAC3F00002E44BB
:1097E0003333333F0000224484250020F0B5044683
:1097F000806A036885B05B699847054648B9504B55
:1098000050491B68986903681B689847284605B04B
:10981000F0BD03689B689847A06A03680A21DB6A69
:109820009847A06A03689B69984760B9444B4649CA
:109830001B68986903681B6898472B682846DB6893
:1098400098470025E2E72046FFF7EEFE0028F4D017
:109850002046FFF7FFFE30B9394B3C491B68986939
:1098600003681B68E8E72046FFF754FE0028E4D0B1
:10987000A06A0368DB69984730B9314B34491B68EB
:10988000986903681B68D7E794F84430A06A43F0EE
:10989000010384F8443003680321DB6A98472B688E
:1098A0002846DB689847236820469B689847A06A4B
:1098B000036807215B6A9847A06A03689B6A984718
:1098C00004F1420201462046FEF7D6FE0546002876
:1098D0009CD0A06A94F84210036801919B6A984753
:1098E000019902462046FEF7CBFE94F8432094F8F7
:1098F00042102046FEF7FAFE94F844309B0705D547
:1099000094F8421001222046FEF7CEFEA06A02948F
:1099100003681E6A0F4B039304AB13E90C0043F278
:109920001541B047064BA06A1B689E6933681F68E3
:1099300003689B6A9847084902463046B84765E77E
:109940008425002000A0090826A009084CA00908C9
:1099500071A00908259601089FA0090810B5084BB9
:10996000036004460023086860600B60037A03F01C
:109970000703022B02D1C02108F074FF204610BD5E
:10998000DCA0090810B5044B044640F8043BFAF784
:10999000DBFA204610BD00BFDCA0090810B5044664
:1099A000FFF7F0FF2046FBF7F5FC204610BD000056
:1099B000F7B503680E4617461BB90024204603B0CE
:1099C000F0BD0022026008200193FBF7DBFC054696
:1099D00010B101A9FFF7C2FF01A8FAF7B5FA002DEF
:1099E000EBD04820FBF7CEFC04460028E5D0294602
:1099F0003B463246FFF774FD2046FFF7F7FE05466B
:109A00000028DBD1236820465B6898472C46D5E7C1
:109A100090F82D100022FEF7E1BD0000F0B50446DD
:109A2000806A036889B05B6A984703689B689847B7
:109A3000A06A03680A219B6C9847A06A01230DF174
:109A40001702002108F042FE002838D09DF8173098
:109A5000082B34D14E4F052500230122A06A322164
:109A600008F010FE3B689B6A1A68526840B90A21E8
:109A700018469047013D15F0FF05EDD145481CE023
:109A800018461421904706AEFF238DF81830A06ABF
:109A900001233246322108F019FE0028EAD09DF851
:109AA000183013F00103E5D1A06A03930822322194
:109AB00008F0E8FD039B58B937484FF0EFFDA06A66
:109AC00003685B6A98470368DB68984700255CE099
:109AD000A06A03931A46342108F0D4FD0028EBD085
:109AE000039BA06A2422412108F0CCFD0028E3D08A
:109AF000039BA06A0822312108F0C4FD0028DBD0B6
:109B0000A06A036803219B6C9847A06A03685B6A9C
:109B100098470368DB689847A06A102108F074FD35
:109B2000A36A04F12D0299682046FEF7A5FD0546BB
:109B300058B3A36A94F82D109A682046FEF7A0FD4A
:109B4000A36A16481A7A597A00919B681449D20878
:109B50004FF0A4FD94F82C2094F82D102046FEF729
:109B6000C5FD94F82E302BB194F82D10012220461B
:109B7000FEF79AFDA06A03689F6A0A4B0694079352
:109B800096E80C0042F21071B847284609B0F0BDC3
:109B9000842500206CA109080CA1090843A109082B
:109BA0003BA10908319C010810B586B00446012389
:109BB000806A0DF10302102108F088FD98B39DF82A
:109BC0000330DB072FD5A06A062301AA112108F074
:109BD0007DFD40B3BDF904309FED146A94F82D204B
:109BE00006EE903ABDF9063007EE103ABDF808309F
:109BF0005B421BB207EE903AF8EEE66AB8EEC77A1F
:109C0000F8EEE77A66EE866A27EE067A67EE867ADF
:109C10000A2303A92046CDED036A8DED047ACDED2C
:109C2000057AFEF7C9FD06B010BD00BF85EBC13F48
:109C3000FFF7BABFF7B503680D4616461BB90024F7
:109C4000204603B0F0BD002707603020CDE9007347
:109C5000FBF798FB044650B1FEF7C0FB0E4B2360A8
:109C6000019BA362019784F82C6084F82E5001A810
:109C7000FAF76AF96846FAF767F9002CDFD0204650
:109C8000FFF7CCFE05460028DAD1236820465B6842
:109C900098472C46D4E700BF98A1090810B5044B9B
:109CA000044640F8283BFAF74FF9204610BD00BFA4
:109CB00098A1090810B50446FFF7F0FF2046FBF70E
:109CC00069FB204610BD000090F831100022FEF71D
:109CD00085BC000010B5002304460122806A0A21D9
:109CE00008F0D0FC10B9012384F8323010BD000018
:109CF000F0B50446806A036889B05B6A98470368D8
:109D00009B689847A06A03680A219B6C98470122C8
:109D100000230B21A06A08F0B5FC514B1F68B86AFC
:109D200003680A215B689847A06A01230DF11702B6
:109D3000002108F0CBFC002835D09DF81730102BFF
:109D400031D10525002301220B21A06A08F09AFCDD
:109D5000BB6A1A680A21526838B918469047013D13
:109D600015F0FF05EED13F481BE01846904706AEC0
:109D7000FF238DF81830A06A012332460B2108F02A
:109D8000A5FC0028EBD09DF8183013F00103E6D1B4
:109D9000A06A03932422412108F074FC039B58B964
:109DA00031484FF07BFCA06A03685B6A9847036800
:109DB000DB68984700254FE0A06AC022422108F0E6
:109DC00061FC0028ECD0A06A036803219B6C9847D3
:109DD0002046FFF77FFFA06A03685B6A9847036825
:109DE000DB689847A06A0A2108F00EFCA36A04F118
:109DF000310299682046FEF73FFC054660B3A36A2E
:109E000094F831109A682046FEF73AFCA36A174886
:109E10001A7A597A00919B681549D2084FF03EFC96
:109E200094F8302094F831102046FEF75FFC94F847
:109E300033302BB194F8311001222046FEF734FC68
:109E4000A06A03689F6A0B4B0694079396E80C0080
:109E500042F21071B847E062284609B0F0BD00BF79
:109E600084250020DFA10908A8A1090843A1090849
:109E7000D7A10908459F010830B590F8323087B066
:109E800004463BB1002380F8323007B0BDE83040D3
:109E9000FFF720BF806A062301AA032108F016FC01
:109EA000002849D02046FFF715FFA06AE16A036841
:109EB00042F21072DB6A9847BDF8042041F2D640A6
:109EC00013189BB242F6AC118B4235D8BDF906107F
:109ED000814231DC194B99422EDBBDF90800BDF8F7
:109EE000083042F28E05A84226DC154DA84223DB3D
:109EF00012B207EE102AB8EEC77AF0EE086A07EE43
:109F0000901A27EE267A5B421BB28DED037AB8EEEB
:109F1000E77A07EE903AF8EEE77A27EE267A67EED0
:109F2000A67A94F831208DED047A0A2303A92046FD
:109F3000CDED057AFEF740FC07B030BD2AEBFFFF00
:109F400072DFFFFFFFF798BFF7B503680D461646AF
:109F50001BB90024204603B0F0BD00270760342061
:109F6000CDE90073FBF70EFA044650B1FEF736FA5E
:109F70000E4B2360019BA362019784F8306084F844
:109F8000335001A8F9F7E0FF6846F9F7DDFF002C30
:109F9000DFD02046FFF7ACFE05460028DAD1236863
:109FA00020465B6898472C46D4E700BF08A2090802
:109FB00010B5044B044640F8283BF9F7C5FF20468E
:109FC00010BD00BF08A2090810B50446FFF7F0FF56
:109FD0002046FBF7DFF9204610BD000090F82C105A
:109FE0000022FEF7FBBA00007FB50446806A0368D2
:109FF0005B6A984703689B689847A06A037A03F0F6
:10A000000703022B02D1C02108F02CFCA06A0368D0
:10A010000A219B6C9847A06A01230DF107020F21CA
:10A0200008F054FB00286BD09DF807303D2B67D11A
:10A030000A220521A06A08F0CFFA0123FC22202180
:10A04000A06A08F01FFB012300222121A06A08F06A
:10A0500019FB012300222221A06A08F013FB01232F
:10A060000C222321A06A08F00DFB402201232421A9
:10A07000A06A08F007FBA06A036803219B6C98475D
:10A08000A06A03685B6A98470368DB689847A06A20
:10A09000082108F0B9FAA36A04F12C029968204655
:10A0A000FEF7EAFA0546002832D0A36A94F82C108D
:10A0B0009A682046FEF7E4FAA36A94F82C2099687F
:10A0C00015484FF0EBFA94F82E2094F82C10204607
:10A0D000FEF70CFB94F82D302BB194F82C100122D4
:10A0E0002046FEF7E1FAA06A029403689E6A0B4BD1
:10A0F000039304AB13E90C0043F2D401B04707E02B
:10A10000A06A03685B6A98470368DB689847002584
:10A11000284604B070BD00BF18A20908A9A1010813
:10A1200010B586B004460123806A0DF10302272191
:10A1300008F0CCFA88B39DF803301B072DD5A06A30
:10A14000062301AA282108F0C1FA30B3BDF9043072
:10A150009FED146A94F82C2006EE903ABDF9063073
:10A1600007EE103ABDF9083007EE903AF8EEE66ACD
:10A17000B8EEC77AF8EEE77A66EE866A27EE067AD8
:10A1800067EE867A0A2303A92046CDED036A8DED9A
:10A19000047ACDED057AFEF70FFBA06A08F0BAFA53
:10A1A00006B010BDF1A9153EFFF7BABFF7B50368B9
:10A1B0000E4615461BB90024204603B0F0BD00270B
:10A1C000076030200193FBF7DDF8044650B1FEF73D
:10A1D00005F90D4B2360019BA362019784F82D6064
:10A1E00084F82E5001A8F9F7AFFE002CE3D02046EA
:10A1F000FFF7FAFE05460028DED1236820465B689B
:10A2000098472C46D8E700BF48A2090810B5044B70
:10A21000044640F8283BF9F797FE204610BD00BFE2
:10A2200048A2090810B50446FFF7F0FF2046FBF7E7
:10A23000B1F8204610BD000090F82D100022FEF766
:10A24000CDB90000F8B504460D4617461E46FEF788
:10A25000C5F8084B23602B68A362002200232A6004
:10A2600084F82E7023636363A36384F84E602046F2
:10A27000F8BD00BF88A20908F0B50446806A0368EB
:10A2800085B05B6A984703689B689847A06A036833
:10A290000A219B6C9847A06A01230DF10702202137
:10A2A00008F014FA002866D09DF80730062B62D11A
:10A2B000802200230821A06A08F0E4F9334B1E68CD
:10A2C000B06A03680A215B68984700231A46072191
:10A2D000A06A08F0D7F900231A460821A06A08F0FE
:10A2E000D1F9A06A03685B6A98470368DB689847FE
:10A2F000A06A0C2108F088F9A36A04F12D0299687C
:10A300002046FEF7B9F9054600283CD0A36A94F828
:10A310002D109A682046FEF7B3F9A36A94F82D2011
:10A3200099681B484FF0BAF994F84E2094F82D1014
:10A330002046FEF7DBF994F82E302BB194F82D105F
:10A3400001222046FEF7B0F9A06A036801219B6C48
:10A350009847A06A029403689F6A0E4B039304AB6C
:10A3600013E90C0042F21071B847B06A0368FA2191
:10A370005B68984707E0A06A03685B6A98470368D0
:10A38000DB6898470025284605B0F0BD84250020ED
:10A3900058A2090841A7010830B5044699B04FF00A
:10A3A00093FF636CC31AB3F5FA7F12D9002384F8C4
:10A3B0002C306064A06A00238022072108F062F933
:10A3C00028B1012384F82C304FF07EFF206419B0AF
:10A3D00030BD94F82C30052BF9D801A252F823F0A7
:10A3E000B5A30108F9A3010843A4010883A4010847
:10A3F000CDA4010865A601084FF066FF236CC01AC2
